:020000040800F2
:1000000000060020A10200084910000801100008A5
:10001000291000080110000821100008A3020008A0
:10002000A3020008A3020008A3020008252A000872
:10003000A3020008A3020008A3020008A30200080C
:10004000A3020008A3020008A3020008A3020008FC
:10005000A3020008A3020008AD3E0008D93E000834
:10006000053F0008313F00085D3F0008A30200087B
:10007000A3020008A3020008A3020008A3020008CC
:10008000A3020008A3020008A3020008A3020008BC
:10009000A3020008A3020008A3020008893F000889
:1000A000A3020008A3020008A3020008A30200089C
:1000B000A3020008A3020008A3020008A30200088C
:1000C000A3020008A3020008A3020008A30200087C
:1000D000A3020008A3020008A30200086140000870
:1000E000ED3F0008A3020008A3020008A3020008D5
:1000F000A3020008A3020008A3020008A30200084C
:10010000A3020008A30200089D400008A302000803
:10011000A302000875400008A3020008A30200081B
:10012000A3020008A3020008A3020008A30200081B
:10013000A3020008A3020008A3020008A30200080B
:10014000A3020008A3020008A3020008A3020008FB
:10015000A3020008A3020008A3020008A3020008EB
:10016000A3020008A3020008A3020008A3020008DB
:10017000A302000891350008A3020008A3020008AA
:10018000A3020008A302000889400008A302000897
:10019000A3020008A3020008A3020008A3020008AB
:1001A000A3020008A3020008A3020008A30200089B
:1001B000A3020008A3020008A3020008A30200088B
:1001C000A3020008A3020008A3020008A30200087B
:1001D000A30200087D350008A3020008A30200085E
:1001E000A3020008A3020008A3020008A30200085B
:1001F000A3020008A3020008A3020008A30200084B
:10020000A3020008A3020008A3020008A30200083A
:10021000A3020008A3020008A3020008A30200082A
:10022000A3020008A3020008A3020008A30200081A
:10023000A3020008A3020008A3020008A30200080A
:10024000A3020008A3020008A3020008A3020008FA
:10025000A3020008A3020008A3020008A3020008EA
:10026000A3020008A3020008A3020008A3020008DA
:10027000A3020008A3020008A3020008A3020008CA
:10028000A3020008A3020008A3020008A3020008BA
:10029000A3020008A3020008A3020008A3020008AA
:1002A00002E000F000F8FEE772B63A4880F30888F2
:1002B000394880F3098839484EF60851CEF20001DA
:1002C000086040F20000CCF200004EF63471CEF22D
:1002D00000010860BFF34F8FBFF36F8F40F2000043
:1002E000C0F2F0004EF68851CEF200010860BFF374
:1002F0004F8FBFF36F8F4FF00000E1EE100A4EF604
:100300003C71CEF200010860062080F31488BFF330
:100310006F8F02F045FC02F0E7FB03F081FB4FF02A
:1003200055301F491B4A91423CBF41F8040BFAE784
:100330001C49194A91423CBF41F8040BFAE71A499B
:100340001A4A1B4B9A423EBF51F8040B42F8040B69
:10035000F8E700201749184A91423CBF41F8040BC6
:10036000FAE702F0FFFB03F0DFFB144C144DAC4244
:1003700003DA54F8041B8847F9E700F041F8114C00
:10038000114DAC4203DA54F8041B8847F9E702F038
:10039000E7BB00000006002000220020000000084B
:1003A0000000002000060020D044000800220020A9
:1003B0006C22002070220020E44F0020A0020008E0
:1003C000A0020008A0020008A00200082DE9F04FDA
:1003D0002DED108AC1F80CD0D0F80CD0BDEC108AED
:1003E000BDE8F08F002383F311882846A047002042
:1003F00001F000FFFEE701F07BFE00DFFEE70000FA
:1004000038B502F0CFFA054602F002FB0446D0B937
:100410000F4B9D4219D001339D4241F2883512BFE6
:10042000044600250124002002F0C6FA0CB100F0B9
:1004300077F800F085FD00F029FC284600F01EF951
:1004400000F06EF8F9E70025EDE70546EBE700BFA1
:10045000010007B008B500F0E5FBA0F12003584209
:10046000584108BD07B541F21203022101A8ADF8B9
:10047000043000F0F5FB03B05DF804FB38B5202331
:1004800083F311881748C3680BB101F039FF0023CB
:10049000154A4FF47A71134801F0F6FE002383F3F6
:1004A0001188124C236813B12368013B23606368F1
:1004B00013B16368013B63600D4D2B7833B96368FA
:1004C0007BB9022000F0AEFC322363602B78032B53
:1004D00007D163682BB9022000F0A4FC4FF47A73B3
:1004E000636038BD702200207D0400088C2300204A
:1004F00084220020084B187003280CD8DFE800F095
:1005000008050208022000F07DBC022000F06ABC51
:10051000024B00225A607047842200208C23002066
:10052000F8B5504B504A1C461968013100F09980CB
:1005300004339342F8D162684C4B9A4240F2918066
:100540004B4B9B6803F1006303F500339A4280F044
:100550008880002000F0B4FB0220FFF7CBFF454B62
:100560000021D3F8E820C3F8E810D3F81021C3F82D
:100570001011D3F81021D3F8EC20C3F8EC10D3F805
:100580001421C3F81411D3F81421D3F8F020C3F8C0
:10059000F010D3F81821C3F81811D3F81821D3F8A4
:1005A000802042F00062C3F88020D3F8802022F03F
:1005B0000062C3F88020D3F88020D3F8802042F076
:1005C0000072C3F88020D3F8802022F00072C3F8B4
:1005D0008020D3F8803072B64FF0E023C3F8084D86
:1005E000D4E90004BFF34F8FBFF36F8F224AC2F8E4
:1005F0008410BFF34F8F536923F480335361BFF3EB
:100600004F8FD2F8803043F6E076C3F3C905C3F3C9
:100610004E335B0103EA060C29464CEA8177013927
:10062000C2F87472F9D2203B13F1200FF2D1BFF35C
:100630004F8FBFF36F8FBFF34F8FBFF36F8F536930
:1006400023F4003353610023C2F85032BFF34F8FBD
:10065000BFF36F8F202383F31188854680F30888CA
:100660002047F8BD0000020820000208FFFF010833
:10067000002200200044025800ED00E02DE9F04F78
:1006800093B0B44B2022FF2100900AA89D6800F08F
:1006900001FCB14A1378A3B90121B0481170C360BD
:1006A000202383F31188C3680BB101F029FE0023D6
:1006B000AB4A4FF47A71A94801F0E6FD002383F3B9
:1006C0001188009B13B1A74B009A1A60A64A1378B1
:1006D000032B03D000231370A24A53604FF0000A8B
:1006E000009CD3465646D146012000F08BFB24B136
:1006F0009C4B1B68002B00F02682002000F092FA31
:100700000390039B002BF2DB012000F06BFB039BAB
:10071000213B1F2BE8D801A252F823F09D070008C7
:10072000C507000859080008E9060008E90600089E
:10073000E9060008EB080008BB0A0008D509000814
:10074000370A00085F0A0008850A0008E906000861
:10075000970A0008E9060008090B00083D08000890
:10076000E90600084D0B0008A90700083D0800082D
:10077000E9060008370A0008E9060008E90600084B
:10078000E9060008E9060008E9060008E90600088D
:10079000E9060008E9060008590800080220FFF7EA
:1007A00059FE002840F0F981009B022105A8BAF10A
:1007B000000F08BF1C4641F21233ADF8143000F0B0
:1007C0004FFA91E74FF47A7000F02CFA071EEBDB3A
:1007D0000220FFF73FFE0028E6D0013F052F00F280
:1007E000DE81DFE807F0030A0D101336052304212C
:1007F00005A8059300F034FA17E004215548F9E7FD
:1008000004215A48F6E704215948F3E74FF01C0841
:10081000404608F1040800F055FA0421059005A8A7
:1008200000F01EFAB8F12C0FF2D101204FF00009B0
:1008300000FA07F747EA0B0B5FFA8BFB00F076FB39
:1008400026B10BF00B030B2B08BF0024FFF70AFEA9
:100850004AE704214748CDE7002EA5D00BF00B0353
:100860000B2BA1D10220FFF7F5FD074600289BD0F6
:100870000120002600F024FA0220FFF73BFE5FFA79
:1008800086F8404600F02CFA0446B0B10399404681
:100890000136A1F140025142514100F031FA0028E5
:1008A000EDD1BA46044641F21213022105A83E4694
:1008B000ADF8143000F0D4F916E725460120FFF713
:1008C00019FE244B9B68AB4207D9284600F0FAF981
:1008D000013040F067810435F3E70025224BBA462A
:1008E0003E461D701F4B5D60A8E7002E3FF45CAFD5
:1008F0000BF00B030B2B7FF457AF0220FFF7FAFD31
:10090000322000F08FF9B0F10008FFF64DAF18F07B
:1009100003077FF449AF0F4A08EB0503926893423F
:100920003FF642AFB8F5807F3FF73EAF124BB84578
:10093000019323DD4FF47A7000F074F90390039A69
:10094000002AFFF631AF039A0137019B03F8012B10
:10095000EDE700BF00220020882300207022002045
:100960007D0400088C230020842200200422002023
:10097000082200200C22002088220020C820FFF737
:1009800069FD074600283FF40FAF1F2D11D8C5F1B0
:1009900020020AAB25F0030084494245184428BFD1
:1009A0004246019200F050FA019AFF217F4800F080
:1009B00071FA4FEAA803C8F387027C4928460193DD
:1009C00000F070FA064600283FF46DAF019B05EB7E
:1009D000830533E70220FFF73DFD00283FF4E4AE36
:1009E00000F0ACF900283FF4DFAE0027B846704BAA
:1009F0009B68BB4218D91F2F11D80A9B01330ED018
:100A000027F0030312AA134453F8203C05934046F1
:100A1000042205A9043700F019FB8046E7E73846B1
:100A200000F050F90590F2E7CDF81480042105A8F4
:100A300000F016F902E70023642104A8049300F0F3
:100A400005F900287FF4B0AE0220FFF703FD00286F
:100A50003FF4AAAE049800F067F90590E6E700239A
:100A6000642104A8049300F0F1F800287FF49CAE00
:100A70000220FFF7EFFC00283FF496AE049800F048
:100A800055F9EAE70220FFF7E5FC00283FF48CAEB9
:100A900000F064F9E1E70220FFF7DCFC00283FF4F6
:100AA00083AE05A9142000F05FF9074604210490E5
:100AB00004A800F0D5F83946B9E7322000F0B2F8C2
:100AC000071EFFF671AEBB077FF46EAE384A07EB28
:100AD0000903926893423FF667AE0220FFF7BAFC23
:100AE00000283FF461AE27F003074F44B9453FF4B7
:100AF000A5AE484609F1040900F0E4F80421059088
:100B000005A800F0ADF8F1E74FF47A70FFF7A2FC0A
:100B100000283FF449AE00F011F9002844D00A9BA8
:100B200001330BD008220AA9002000F0BBF90028ED
:100B30003AD02022FF210AA800F0ACF9FFF792FC7E
:100B40001C4801F05DFB13B0BDE8F08F002E3FF4B0
:100B50002BAE0BF00B030B2B7FF426AE002364218E
:100B600005A8059300F072F8074600287FF41CAE34
:100B70000220FFF76FFC804600283FF415AEFFF718
:100B800071FC41F2883001F03BFB059800F016FA49
:100B900046463C4600F0CAF9A6E506464EE64FF04A
:100BA000000901E6BA467EE637467CE68822002048
:100BB00000220020A08601002DE9F84F4FF47A733F
:100BC00006460D46002402FB03F7DFF85080DFF8ED
:100BD000509098F900305FFA84FA5A1C01D0A34271
:100BE00010D159F824002A4631460368D3F820B0C2
:100BF0003B46D847854205D1074B012083F800A02A
:100C0000BDE8F88F0134042CE3D14FF4FA7001F001
:100C1000F7FA0020F4E700BFD823002010220020BC
:100C200014220020002307B5024601210DF1070020
:100C30008DF80730FFF7C0FF20B19DF8070003B023
:100C40005DF804FB4FF0FF30F9E700000A4604218D
:100C500008B5FFF7B1FF80F00100C0B2404208BD07
:100C6000074B0A4630B41978064B53F82140014629
:100C700023682046DD69044BAC4630BC604700BFAA
:100C8000D823002014220020A086010070B50A4E4F
:100C900000240A4D01F05EFD3080286833888342CD
:100CA00008D901F053FD2B6804440133B4F5003F2B
:100CB0002B60F2D370BD00BFDA2300209423002004
:100CC00001F026BE00F1006000F5003000687047BA
:100CD00000F10060920000F5003001F09DBD0000C1
:100CE000054B1A68054B1B889B1A834202D9104496
:100CF00001F02CBD0020704794230020DA2300204F
:100D000038B50446074D29B128682044BDE838406D
:100D100001F034BD2868204401F01EFD0028F3D006
:100D200038BD00BF942300200020704700F1FF5021
:100D300000F58F10D0F8000870470000064991F8C0
:100D4000243033B100230822086A81F82430FFF7E9
:100D5000BFBF0120704700BF98230020014B1868D7
:100D6000704700BF0010005C1B4B0246F0B51868CE
:100D70001A4BC0F30B06000C1F885C68BE4293F947
:100D8000085003D09F89BE4203D10C335C6893F9AD
:100D900008500426124B1F880433874208BF13F9FA
:100DA000025C013EF7D1013A013C0B460A449342F2
:100DB00007D214F9016F581C2EB1034600F8016CDC
:100DC000F5E7184605E02C2482421C7001D9981CD6
:100DD0005D70401AF0BD00BF0010005C24220020AE
:100DE000A0410008022804D1054B4FF000629A612F
:100DF00070470128FCD1024B4FF08062F7E700BF3B
:100E0000000C0258022804D1054B4FF400629A618D
:100E100070470128FCD1024B4FF48062F7E700BF16
:100E2000000C0258022805D1064A536983F4006376
:100E3000536170470128FCD1024A536983F48063EF
:100E4000F6E700BF000C0258002310B5934203D010
:100E5000CC5CC4540133F9E710BD0000013810B573
:100E600010F9013F3BB191F900409C4203D11AB106
:100E70000131013AF4E71AB191F90020981A10BD36
:100E80001046FCE703460246D01A12F9011B00295E
:100E9000FAD1704702440346934202D003F8011B83
:100EA000FAE770472DE9F8431F4D14460746884678
:100EB00095F8242052BBDFF870909CB395F824304D
:100EC0002BB92022FF2148462F62FFF7E3FF95F858
:100ED00024004146C0F1080205EB8000A24228BF71
:100EE0002246D6B29200FFF7AFFF95F82430A41B3C
:100EF00017441E449044E4B2F6B2082E85F82460EC
:100F0000DBD1FFF71BFF0028D7D108E02B6A03EBEA
:100F100082038342CFD0FFF711FF0028CBD10020FE
:100F2000BDE8F8830120FBE798230020024B1A78E4
:100F3000024B1A70704700BFD823002010220020F7
:100F4000F8B5184C184800F05DFC2146164800F032
:100F500085FC24681548D4F89020154ED2F8043842
:100F6000144D43F00203104FC2F8043801F048F961
:100F70002046114900F080FDD4F890200424D2F8D6
:100F8000043823F00203C2F804384FF4E13333602D
:100F900055F8040BB84202D0314600F091FB013CF9
:100FA000F6D1F8BDB0420008D832002040420F0010
:100FB000C023002014220020B84200080C4B70B55A
:100FC0000C4D04461E780C4B55F826209A420DD045
:100FD0000A4B002118221846FFF75CFF0460014607
:100FE00055F82600BDE8704000F06ABB70BD00BF38
:100FF000D823002014220020D8320020C023002053
:1010000000B59BB0EFF3098168226846FFF71CFF2B
:10101000EFF30583014B9B6BFEE700BF00ED00E0A3
:1010200008B5FFF7EDFF000000B59BB0EFF30981B5
:1010300068226846FFF708FFEFF30583014B5B6BFF
:10104000FEE700BF00ED00E0FEE7000030B50A4417
:10105000084D91420DD011F8013B5840082340F350
:101060000004013B2C4013F0FF0384EA5000F6D14A
:10107000EFE730BD2083B8ED02684368114301609B
:1010800003B1184770470000024A136843F0C003D9
:101090001360704700480040024A136843F0C003E1
:1010A0001360704700500040024A136843F0C003C9
:1010B000136070470078004037B5274C274D204615
:1010C00000F0F2FA04F11400009400234FF40072CF
:1010D000234900F0B3F94FF40072224904F13800BB
:1010E0000094214B00F02CFA204BC4E91735204C1A
:1010F000204600F0D9FA04F11400009400234FF4C4
:1011000000721C4900F09AF94FF400721A4904F178
:1011100038000094194B00F013FA194BC4E9173545
:10112000184C204600F0C0FA04F1140000234FF4DC
:1011300000721549009400F081F9144B4FF40072CD
:10114000134904F13800009400F0FAF9114BC4E996
:10115000173503B030BD00BFDC23002000E1F505EA
:1011600020250020202B0020891000080048004086
:101170004824002020270020202D0020991000085E
:1011800000500040B424002020290020A9100008AD
:10119000202F002000780040037C30B5334C00291C
:1011A00018BF0C46012B18D1314B98420FD1314B4F
:1011B000D3F8E82042F48022C3F8E820D3F81021C5
:1011C00042F48022C3F81021D3F8103105E02A4BF5
:1011D00098422FD0294B984238D02268036EC16DB7
:1011E00003EB52038466B3FBF2F36268150442BF5B
:1011F00023F0070503F0070343EA4503CB60A36828
:1012000043F040034B60E36843F001038B6042F41A
:10121000967343F001030B604FF0FF330B625105EF
:1012200005D512F010221DD0B2F1805F1CD080F8DD
:10123000643030BD0F4BD3F8E82042F48012C3F87D
:10124000E820D3F8102142F48012BBE7094BD3F811
:10125000E82042F08042C3F8E820D3F8102142F0A1
:101260008042AFE77F23E2E73F23E0E7B041000899
:10127000DC2300200044025848240020B42400202D
:101280002DE9F047C66D05463768F46921073462D9
:1012900019D014F0080118BF8021E20748BF41F0BF
:1012A0002001A3074FF0200348BF41F04001600731
:1012B00048BF41F4807183F31188281DFFF7DCFEDD
:1012C000002383F31188E2050AD5202383F31188D4
:1012D0004FF40071281DFFF7CFFE002383F3118820
:1012E0004FF020094FF0000A14F0200838D13B06D7
:1012F00016D54FF0200905F1380A200610D589F3DC
:101300001188504600F050F9002836DA0821281DCF
:10131000FFF7B2FE27F080033360002383F31188C8
:10132000790614D5620612D5202383F31188D5E9F6
:1013300013239A4208D12B6C33B127F040071021B8
:10134000281DFFF799FE3760002383F31188E30619
:1013500018D5AA6E1369ABB15069BDE8F0471847BC
:1013600089F31188736A284695F86410194000F0D3
:10137000B5F98AF31188F469B6E7B06288F3118889
:10138000F469BAE7BDE8F087F8B515468268044607
:101390000B46AA4200D28568A1692669761AB54231
:1013A0000BD218462A46FFF74FFDA3692B44A361D1
:1013B0002846A3685B1BA360F8BD0CD9AF1B184679
:1013C0003246FFF741FD3A46E1683044FFF73CFD05
:1013D000E3683B44EBE718462A46FFF735FDE36830
:1013E000E5E7000083689342F7B50446154600D24E
:1013F0008568D4E90460361AB5420BD22A46FFF755
:1014000023FD63692B4463612846A3685B1BA360CB
:1014100003B0F0BD0DD93246AF1B0191FFF714FDAB
:1014200001993A46E0683144FFF70EFDE3683B441A
:10143000E9E72A46FFF708FDE368E4E710B50A4448
:101440000024C361029B8460C16002610362C0E941
:101450000000C0E9051110BD08B5D0E9053293427E
:1014600001D1826882B98268013282605A1C42616D
:1014700019700021D0E904329A4224BFC368436145
:1014800000F0DAFE002008BD4FF0FF30FBE700005F
:1014900070B5202304460E4683F31188A568A5B1D4
:1014A000A368A269013BA360531CA361157822695C
:1014B000934224BFE368A361E3690BB120469847D8
:1014C000002383F31188284607E03146204600F0C8
:1014D000A3FE0028E2DA85F3118870BD2DE9F74FED
:1014E00004460E4617469846D0F81C904FF0200A46
:1014F0008AF311884FF0000B154665B12A46314634
:101500002046FFF741FF034660B94146204600F000
:1015100083FE0028F1D0002383F31188781B03B0E9
:10152000BDE8F08FB9F1000F03D001902046C84705
:10153000019B8BF31188ED1A1E448AF31188DCE7B6
:10154000C160C361009B82600362C0E90511114460
:10155000C0E9000001617047F8B504460D46164623
:10156000202383F31188A768A7B1A368013BA36078
:1015700063695A1C62611D70D4E904329A4224BF27
:10158000E3686361E3690BB120469847002080F36C
:10159000118807E03146204600F03EFE0028E2DADE
:1015A00087F31188F8BD0000D0E9052310B59A42F1
:1015B00001D182687AB982680021013282605A1CA6
:1015C00082611C7803699A4224BFC368836100F07A
:1015D00033FE204610BD4FF0FF30FBE72DE9F74FFB
:1015E00004460E4617469846D0F81C904FF0200A45
:1015F0008AF311884FF0000B154665B12A46314633
:101600002046FFF7EFFE034660B94146204600F052
:1016100003FE0028F1D0002383F31188781B03B068
:10162000BDE8F08FB9F1000F03D001902046C84704
:10163000019B8BF31188ED1A1E448AF31188DCE7B5
:10164000026843681143016003B118477047000006
:101650001430FFF743BF00004FF0FF331430FFF7A3
:101660003DBF00003830FFF7B9BF00004FF0FF3337
:101670003830FFF7B3BF00001430FFF709BF000098
:101680004FF0FF311430FFF703BF00003830FFF791
:1016900063BF00004FF0FF323830FFF75DBF00003E
:1016A00000207047FFF708BD044B03600023436030
:1016B000C0E9023301230374704700BFC84100082A
:1016C00010B52023044683F31188FFF765FD02233C
:1016D0002374002383F3118810BD000038B5C3695B
:1016E00004460D461BB904210844FFF7A9FF29460B
:1016F00004F11400FFF7B0FE002806DA201D4FF4B5
:101700008061BDE83840FFF79BBF38BD0268436881
:101710001143016003B118477047000013B5406BD7
:1017200000F58054D4F8A4381A681178042914D12B
:10173000017C022911D11979012312898B401342AE
:101740000BD101A94C3002F06BF8D4F8A448024642
:10175000019B2179206800F0DFF902B010BD000084
:10176000143001F0EDBF00004FF0FF33143001F0F2
:10177000E7BF00004C3002F0BFB800004FF0FF336D
:101780004C3002F0B9B80000143001F0BBBF0000CB
:101790004FF0FF31143001F0B5BF00004C3002F0C3
:1017A0008BB800004FF0FF324C3002F085B80000DB
:1017B0000020704710B500F58054D4F8A4381A689A
:1017C0001178042917D1017C022914D159790123F8
:1017D00052898B4013420ED1143001F04DFF024666
:1017E00048B1D4F8A4484FF4407361792068BDE84B
:1017F000104000F07FB910BD406BFFF7DBBF000069
:10180000704700007FB5124B012504260446036093
:101810000023057400F1840243602946C0E90233C5
:101820000C4B0290143001934FF44073009601F07A
:10183000FFFE094B04F69442294604F14C00029441
:10184000CDE900634FF4407301F0C6FF04B070BDF2
:10185000F0410008F91700081D1700080A68202346
:1018600083F311880B790B3342F823004B79133340
:1018700042F823008B7913B10B3342F8230000F5B3
:101880008053C3F8A41802230374002383F3118840
:101890007047000038B5037F044613B190F8543008
:1018A000ABB90125201D0221FFF730FF04F1140020
:1018B0006FF00101257700F0CBFC04F14C0084F8B7
:1018C00054506FF00101BDE8384000F0C1BC38BD94
:1018D00010B5012104460430FFF718FF00232377D9
:1018E00084F8543010BD000038B50446002514308B
:1018F00001F0B6FE04F14C00257701F085FF201DB4
:1019000084F854500121FFF701FF2046BDE838401C
:10191000FFF750BF90F8803003F06003202B06D112
:1019200090F881200023212A03D81F2A06D80020FE
:101930007047222AFBD1C0E91D3303E0034A426706
:1019400007228267C3670120704700BF3C22002046
:1019500037B500F58055D5F8A4381A6811780429F0
:101960001AD1017C022917D11979012312898B40E0
:10197000134211D100F14C04204602F005F858B191
:1019800001A9204601F04CFFD5F8A4480246019B6E
:101990002179206800F0C0F803B030BD01F10B03DD
:1019A000F0B550F8236085B004460D46FEB1202303
:1019B00083F3118804EB8507301D0821FFF7A6FE8D
:1019C000FB6806F14C005B691B681BB1019001F0DC
:1019D00035FF019803A901F023FF024648B1039B9C
:1019E0002946204600F098F8002383F3118805B0BB
:1019F000F0BDFB685A691268002AF5D01B8A013BCA
:101A00001340F1D104F18002EAE70000133138B548
:101A100050F82140ECB1202383F3118804F5805362
:101A2000D3F8A4281368527903EB8203DB689B691F
:101A30005D6845B104216018FFF768FE294604F18E
:101A4000140001F023FE2046FFF7B4FE002383F3C9
:101A5000118838BD7047000001F016B901234022FB
:101A6000002110B5044600F8303BFFF713FA0023BD
:101A7000C4E9013310BD000010B52023044683F3F0
:101A800011882422416000210C30FFF703FA204620
:101A900001F01CF902232370002383F3118810BD89
:101AA00070B500EB8103054650690E461446DA60B6
:101AB00018B110220021FFF7EDF9A06918B110222A
:101AC0000021FFF7E7F931462846BDE8704001F0F4
:101AD0000FBA000083682022002103F0011310B523
:101AE000044683601030FFF7D5F92046BDE810406A
:101AF00001F08ABAF0B4012500EB810447898D40DA
:101B0000E4683D43A469458123600023A2606360CB
:101B1000F0BC01F0A7BA0000F0B4012500EB81048D
:101B200007898D40E4683D43646905812360002393
:101B3000A2606360F0BC01F01DBB000070B5022321
:101B400000250446242203702946C0F888500C3032
:101B500040F8045CFFF79EF9204684F8705001F0CD
:101B60005BF963681B6823B129462046BDE87040D5
:101B7000184770BD037880F88C30052303704368E4
:101B80001B6810B504460BB1042198470023A360DD
:101B900010BD000090F88C20436802701B680BB1E8
:101BA000052118477047000070B590F87030044662
:101BB00013B1002380F8703004F18002204601F058
:101BC00047FA63689B68B3B994F8803013F06005F6
:101BD00035D00021204601F0F1FC0021204601F023
:101BE000E1FC63681B6813B1062120469847062371
:101BF00084F8703070BD204698470028E4D0B4F8CF
:101C00008630A26F9A4288BFA36794F98030A56F8F
:101C1000002B4FF0200380F20381002D00F0F280B2
:101C2000092284F8702083F3118800212046D4E92A
:101C30001D23FFF771FF002383F31188DAE794F87F
:101C4000812003F07F0343EA022340F202329342F1
:101C500000F0C58021D8B3F5807F48D00DD8012B86
:101C60003FD0022B00F09380002BB2D104F1880208
:101C700062670222A267E367C1E7B3F5817F00F0E4
:101C80009B80B3F5407FA4D194F88230012BA0D182
:101C9000B4F8883043F0020332E0B3F5006F4DD062
:101CA00017D8B3F5A06F31D0A3F5C063012B90D83E
:101CB0006368204694F882205E6894F88310B4F834
:101CC0008430B047002884D0436863670368A36703
:101CD0001AE0B3F5106F36D040F6024293427FF41B
:101CE00078AF5C4B63670223A3670023C3E794F8D4
:101CF0008230012B7FF46DAFB4F8883023F00203FB
:101D0000A4F88830C4E91D55E56778E7B4F8803059
:101D1000B3F5A06F0ED194F88230204684F88A3053
:101D200001F0D8F863681B6813B101212046984779
:101D3000032323700023C4E91D339CE704F18B03C4
:101D400063670123C3E72378042B10D1202383F397
:101D500011882046FFF7BEFE85F3118803216368D2
:101D600084F88B5021701B680BB12046984794F87B
:101D70008230002BDED084F88B300423237063681C
:101D80001B68002BD6D0022120469847D2E794F852
:101D9000843020461D0603F00F010AD501F04AF9F0
:101DA000012804D002287FF414AF2B4B9AE72B4B69
:101DB00098E701F031F9F3E794F88230002B7FF4D3
:101DC00008AF94F8843013F00F01B3D01A06204600
:101DD00002D501F00BFCADE701F0FCFBAAE794F89B
:101DE0008230002B7FF4F5AE94F8843013F00F01AD
:101DF000A0D01B06204602D501F0E0FB9AE701F0D7
:101E0000D1FB97E7142284F8702083F311882B46C6
:101E10002A4629462046FFF76DFE85F31188E9E63C
:101E20005DB1152284F8702083F3118800212046CB
:101E3000D4E91D23FFF75EFEFDE60B2284F8702037
:101E400083F311882B462A4629462046FFF764FE75
:101E5000E3E700BF20420008184200081C420008C7
:101E600038B590F870300446002B3ED0063BDAB20D
:101E70000F2A34D80F2B32D8DFE803F0373131087E
:101E8000223231313131313131313737856FB0F86C
:101E900086309D4214D2C3681B8AB5FBF3F203FB64
:101EA00012556DB9202383F311882B462A46294603
:101EB000FFF732FE85F311880A2384F870300EE0B4
:101EC000142384F87030202383F3118800232046E4
:101ED0001A461946FFF70EFE002383F3118838BD1A
:101EE000C36F03B198470023E7E70021204601F0C4
:101EF00065FB0021204601F055FB63681B6813B1A8
:101F00000621204698470623D7E7000010B590F831
:101F100070300446142B29D017D8062B05D001D8D1
:101F20001BB110BD093B022BFBD80021204601F05C
:101F300045FB0021204601F035FB63681B6813B1A7
:101F4000062120469847062319E0152BE9D10B23DB
:101F500080F87030202383F3118800231A46194635
:101F6000FFF7DAFD002383F31188DAE7C3689B6982
:101F70005B68002BD5D1C36F03B19847002384F869
:101F80007030CEE7024B0022C3E900339A607047FD
:101F900020310020002382680374054B1B68996878
:101FA0009142FBD25A6803604260106058607047EB
:101FB0002031002008B5202383F31188037C032BF4
:101FC00005D0042B0DD02BB983F3118808BD4369CC
:101FD00000221A604FF0FF334361FFF7DBFF00235D
:101FE000F2E7D0E9003213605A60F3E70023826819
:101FF0000374054B1B6899689142FBD85A680360CB
:10200000426010605860704720310020054B19690C
:1020100008741868026853601A6018610123037419
:10202000FEF7D4B9203100204B1C30B5044687B0F0
:102030000A4D10D02B6901A8094A00F025F9204665
:10204000FFF7E4FF049B13B101A800F059F92B69D5
:10205000586907B030BDFFF7D9FFF8E720310020FD
:10206000B51F000838B50C4D044641612B698168E5
:102070009A68914203D8BDE83840FFF78BBF1846F5
:10208000FFF7B4FF01232C61014623742046BDE80D
:102090003840FEF79BB900BF20310020044B1A687E
:1020A0001B6990689B68984294BF0020012070478C
:1020B0002031002010B5084C236820691A6854604C
:1020C0002260012223611A74FFF790FF0146206904
:1020D000BDE81040FEF77AB92031002008B5FFF7BF
:1020E000DDFF18B1BDE80840FFF7E4BF08BD000000
:1020F000FFF7E0BFFEE7000010B50C4CFFF742FF12
:1021000000F0B4F880220A49204600F03BF8012391
:1021100044F8180C037400F095FC002383F3118835
:1021200062B60448BDE8104000F04CB848310020C9
:10213000244200083442000800F01CB9EFF311807B
:1021400020B9EFF30583202282F311887047000045
:1021500010B530B9EFF30584C4F3080414B180F36B
:10216000118810BDFFF7BAFF84F31188F9E700006A
:10217000034A516853685B1A9842FBD8704700BF06
:10218000001000E082600222028270478368A3F19F
:102190007C0243F80C2C026943F83C2C426943F85A
:1021A000382C074A43F81C2CC268A3F1180043F8E6
:1021B000102C022203F8082C002203F8072C704789
:1021C000E503000810B5202383F31188FFF7DEFF35
:1021D00000210446FFF746FF002383F311882046C1
:1021E00010BD0000024B1B6958610F20FFF70EBFA6
:1021F00020310020202383F31188FFF7F3BF000074
:1022000008B50146202383F311880820FFF70CFF4F
:10221000002383F3118808BD49B1064B42681B694E
:1022200018605A60136043600420FFF7FDBE4FF052
:10223000FF307047203100200368984206D01A68AA
:102240000260506018465961FFF7A4BE7047000055
:1022500038B504460D462068844200D138BD036875
:1022600023605C604561FFF795FEF4E7054B4FF096
:10227000FF3103F11402C3E905220022C3E907126A
:10228000704700BF2031002070B51C4E05460C463B
:10229000C0E9032301F0AEFB334653F8142F9A42F2
:1022A0000DD130620A2C2CBF00190A302A60C5E912
:1022B0000124C6E90555BDE8704001F085BB316ACF
:1022C000431AE31838BF1C469368A34202D9081981
:1022D00001F08AFB73699A6894420CD85A68AC6022
:1022E0002B606A6015609A685D60121B9A604FF0FF
:1022F000FF33F36170BDA41A1B68ECE720310020A6
:1023000038B51B4C636998420DD08168D0E9003222
:1023100013605A600022C2609A680A449A604FF0C3
:10232000FF33E36138BD03682246002142F8143FC1
:1023300093425A60C16003D1BDE8384001F04EBB02
:102340009A688168256A0A449A6001F053FB6369C0
:10235000411B9A688A42E5D9AB181D1A206A092DDB
:1023600098BF01F10A02BDE83840104401F03CBBBF
:10237000203100202DE9F041184C002704F114060B
:10238000656901F037FB236AAA68C11A8A4215D829
:102390001344D5F80C802362D5E9003213605A60EB
:1023A0006369EF60B34201D101F018FB87F3118834
:1023B0002869C047202383F31188E1E76169B142AE
:1023C00009D013441B1ABDE8F0410A2B2CBFC018DA
:1023D0000A3001F009BBBDE8F08100BF20310020C8
:1023E00000207047FEE70000704700004FF0FF300C
:1023F0007047000002290CD0032904D001290748A6
:1024000018BF00207047032A05D8054800EBC2001A
:102410007047044870470020704700BF144300080D
:102420004C220020C842000870B59AB00546084604
:10243000144601A900F0C2F801A8FEF723FD431CD1
:102440000022C6B25B001046C5E9003423700323A6
:10245000023404F8013C01ABD1B202348E4201D8FF
:102460001AB070BD13F8011B013204F8010C04F816
:10247000021CF1E708B5202383F311880348FFF716
:1024800067FA002383F3118808BD00BFD83200200B
:1024900090F8803003F01F02012A07D190F88120C4
:1024A0000B2A03D10023C0E91D3315E003F06003BC
:1024B000202B08D1B0F884302BB990F88120212A44
:1024C00003D81F2A04D8FFF725BA222AEBD0FAE74F
:1024D000034A426707228267C3670120704700BF33
:1024E0004322002007B5052917D8DFE801F01916A7
:1024F00003191920202383F31188104A0121019028
:10250000FFF7CEFA019802210D4AFFF7C9FA0D48EC
:10251000FFF7EAF9002383F3118803B05DF804FBA9
:10252000202383F311880748FFF7B4F9F2E720234B
:1025300083F311880348FFF7CBF9EBE76842000803
:102540008C420008D832002038B50C4D0C4C2A467D
:102550000C4904F10800FFF767FF05F1CA0204F116
:1025600010000949FFF760FF05F5CA7204F1180071
:102570000649BDE83840FFF757BF00BFB04B002009
:102580004C2200204C420008544200085F420008E0
:1025900070B5044608460D46FEF774FCC6B22046E8
:1025A000013403780BB9184670BD32462946FEF750
:1025B00055FC0028F3D10120F6E700002DE9F04793
:1025C00005460C46FEF75EFC2A49C6B22846FFF7D0
:1025D000DFFF08B10936F6B227492846FFF7D8FFD2
:1025E00008B11036F6B2632E0BD8DFF88880DFF81A
:1025F0008890224FDFF890A02E7846B92670BDE86B
:10260000F08729462046BDE8F04701F0B3BD252EEE
:102610002CD1072241462846FEF720FC60B9184B12
:10262000224603F1100153F8040B8B4242F8040BCD
:10263000F9D107351034DFE7082249462846FEF76E
:102640000DFC98B9A21C0F4B197802320909C95D1B
:1026500002F8041C13F8011B01F00F015345C95D7A
:1026600002F8031CF0D118340835C5E7013504F829
:10267000016BC1E7344300085F4200084D43000886
:102680003C43000800E8F11F0CE8F11FBFF34F8F37
:10269000044B1A695107FCD1D3F810215207F8D125
:1026A000704700BF0020005208B50D4B1B78ABB936
:1026B000FFF7ECFF0B4BDA68D10704D50A4A5A60E2
:1026C00002F188325A60D3F80C21D20706D5064AA7
:1026D000C3F8042102F18832C3F8042108BD00BF09
:1026E0000E4E0020002000522301674508B5114B13
:1026F0001B78F3B9104B1A69510703D5DA6842F019
:102700004002DA60D3F81021520705D5D3F80C2126
:1027100042F04002C3F80C21FFF7B8FF064BDA681D
:1027200042F00102DA60D3F80C2142F00102C3F852
:102730000C2108BD0E4E0020002000520F289ABF29
:1027400000F5806040040020704700004FF4003026
:1027500070470000102070470F2808B50BD8FFF70E
:10276000EDFF00F500330268013204D104308342EA
:10277000F9D1012008BD0020FCE700000F2870B54A
:10278000054645D8FFF7DAFC224CFFF77FFF0646E7
:10279000FFF78AFF4FF0FF33072D6361C4F8143150
:1027A00020D82361FFF772FF2B0243F02403E3607C
:1027B000E36843F08003E36023695A07FCD42846AA
:1027C000FFF764FF4FF40031FFF7B8FF00F002F9A4
:1027D0003046FFF78BFFFFF7BBFC2846BDE8704093
:1027E000FFF7BABFC4F81031FFF750FFA5F1080397
:1027F0001B0243F02403C4F80C31D4F80C3143F02D
:102800008003C4F80C31D4F810315B07FBD4D6E751
:10281000002070BD002000522DE9F84F40EA02036D
:1028200005460C461746D80602D00020BDE8F88FB2
:1028300027F01F07DFF8D4B0FFF736FF2744BC426C
:1028400003D10120FFF752FFF0E72022294620465E
:1028500001F080FC10B920352034F0E72B4605F15B
:1028600020021E68711CE0D104339A42F9D1FFF7AF
:1028700065FC05F17843234AB3F5801F224B28BF3E
:102880009A4603F1040338BF9046A2F1080228BF1C
:102890009846A3F108033ABF9146DA469946FFF7F6
:1028A000F5FEC8F80060A5EB040CD9F8002004F18F
:1028B0001C0142F00202C9F80020221FDAF8006071
:1028C00016F00506FAD152F8043F8A424CF802305D
:1028D000F4D1BFF34F8FFFF7D9FE4FF0FF32C8F8A6
:1028E0000020D9F8002022F00202C9F80020FFF7EA
:1028F0002FFC20222146284601F02CFC0028AAD0DB
:1029000030469FE714200052102100521020005240
:1029100010B5084C237828B11BB9FFF7C5FE012379
:10292000237010BD002BFCD02070BDE81040FFF7D5
:10293000DDBE00BF0E4E00200244074BD2B210B5E0
:10294000904200D110BD441C00B253F8200041F861
:10295000040BE0B2F4E700BF504000580E4B30B516
:102960001C6F240405D41C6F1C671C6F44F40044C6
:102970001C670A4C02442368D2B243F4807323607C
:10298000074B904200D130BD441C51F8045B00B2AB
:1029900043F82050E0B2F4E70044025800480258DF
:1029A0005040005807B5012201A90020FFF7C4FFDD
:1029B000019803B05DF804FB13B50446FFF7F2FF7E
:1029C000A04205D0012201A900200194FFF7C6FF13
:1029D00002B010BD0144BFF34F8F064B884204D3B1
:1029E000BFF34F8FBFF36F8F7047C3F85C02203087
:1029F000F4E700BF00ED00E0034B1A681AB9034A80
:102A0000D2F8D0241A607047104E002000400258BF
:102A100008B5FFF7F1FF024B1868C0F3806008BDEE
:102A2000104E0020EFF30983054968334A6B22F00A
:102A300001024A6383F30988002383F311887047F6
:102A400000EF00E0202080F3118862B60D4B0E4AA3
:102A5000D96821F4E0610904090C0A430B49DA60E2
:102A6000D3F8FC2042F08072C3F8FC20084AC2F878
:102A7000B01F116841F0010111601022DA7783F86C
:102A80002200704700ED00E00003FA0555CEACC50A
:102A9000001000E0202310B583F311880E4B5B6813
:102AA00013F4006314D0F1EE103AEFF309844FF001
:102AB0008073683CE361094BDB6B236684F3098810
:102AC000FFF7ECFA10B1064BA36110BD054BFBE715
:102AD00083F31188F9E700BF00ED00E000EF00E0AC
:102AE000F7030008FA03000870B5BFF34F8FBFF378
:102AF0006F8F1A4A0021C2F85012BFF34F8FBFF3F5
:102B00006F8F536943F400335361BFF34F8FBFF3AB
:102B10006F8FC2F88410BFF34F8FD2F8803043F626
:102B2000E074C3F3C900C3F34E335B0103EA040648
:102B3000014646EA81750139C2F86052F9D2203B5C
:102B400013F1200FF2D1BFF34F8F536943F4803359
:102B50005361BFF34F8FBFF36F8F70BD00ED00E087
:102B6000FEE700000A4B0B480B4A90420BD30B4B7D
:102B7000C11EDA1C121A22F003028B4238BF002257
:102B80000021FEF787B953F8041B40F8041BECE75B
:102B90003C450008E44F0020E44F0020E44F0020B3
:102BA0007047000070B5D0E9244300224FF0FF3594
:102BB0009E6804EB42135101D3F80009002805DA9E
:102BC000D3F8000940F08040C3F80009D3F8000BA7
:102BD000002805DAD3F8000B40F08040C3F8000B62
:102BE000013263189642C3F80859C3F8085BE0D273
:102BF0004FF00113C4F81C3870BD000000EB8103D6
:102C0000D3F80CC02DE9F043DCF814204E1CD0F8AA
:102C10009050D2F800E005EB063605EB41185068FD
:102C200070450AD30122D5F8343802FA01F123EABB
:102C30000101C5F83418BDE8F083AEEB0003BCF821
:102C40001040A34228BF2346D8F81849A4B2B3EBDA
:102C5000840FF0D89468A4F1040959F8047F376010
:102C6000A4EB09071F44042FF7D81C4403449460C5
:102C70005360D4E7890141F02001016103699B069B
:102C8000FCD41220FFF774BA10B50A4C2046FEF7A8
:102C9000E5FE094BC4F89030084BC4F89430084C5A
:102CA0002046FEF7DBFE074BC4F89030064BC4F815
:102CB000943010BD144E00200000084084430008EA
:102CC000B04E0020000004409043000870B5037827
:102CD0000546012B5DD1494BD0F89040984259D11F
:102CE000474B0E216520D3F8D82042F00062C3F88C
:102CF000D820D3F8002142F00062C3F80021D3F8B5
:102D00000021D3F8802042F00062C3F88020D3F87D
:102D1000802022F00062C3F88020D3F8803000F0D9
:102D200071FC384BE360384BC4F800380023D5F809
:102D30009060C4F8003EC02323604FF40413A363E3
:102D40003369002BFCDA01230C203361FFF710FA02
:102D50003369DB07FCD41220FFF70AFA3369002B32
:102D6000FCDA00262846A660FFF71CFF6B68C4F853
:102D70001068DB68C4F81468C4F81C68002B3AD1EA
:102D8000224BA3614FF0FF336361A36843F001035B
:102D9000A36070BD1E4B9842C8D1194B0E214D2027
:102DA000D3F8D82042F00072C3F8D820D3F800211D
:102DB00042F00072C3F80021D3F80021D3F880203C
:102DC00042F00072C3F88020D3F8802022F0007215
:102DD000C3F88020D3F88020D3F8D82022F0806276
:102DE000C3F8D820D3F8002122F08062C3F8002174
:102DF000D3F8003193E7074BC3E700BF144E002020
:102E0000004402584014004003002002003C30C03F
:102E1000B04E0020083C30C0F8B5D0F890400546D0
:102E200000214FF000662046FFF724FFD5F89410EC
:102E300000234FF001128F684FF0FF30C4F8343890
:102E4000C4F81C2804EB431201339F42C2F8006906
:102E5000C2F8006BC2F80809C2F8080BF2D20B687E
:102E6000D5F89020C5F89830636210231361166975
:102E700016F01006FBD11220FFF77AF9D4F80038CB
:102E800023F4FE63C4F80038A36943F4402343F0FD
:102E90001003A3610923C4F81038C4F814380B4B8D
:102EA000EB604FF0C043C4F8103B094BC4F8003B43
:102EB000C4F81069C4F80039D5F8983003F110024D
:102EC00043F48013C5F89820A362F8BD604300085E
:102ED00040800010D0F8902090F88A10D2F8003886
:102EE00023F4FE6343EA0113C2F800387047000080
:102EF0002DE9F84300EB8103D0F890500C46804652
:102F0000DA680FFA81F94801166806F00306731EA5
:102F1000022B05EB41134FF0000194BFB604384E6D
:102F2000C3F8101B4FF0010104F1100398BF06F124
:102F3000805601FA03F3916998BF06F5004600290F
:102F40003AD0578A04F15801374349016F50D5F8F8
:102F50001C180B430021C5F81C382B180127C3F897
:102F60001019A7405369611E9BB3138A928B9B086B
:102F7000012A88BF5343D8F89820981842EA03439F
:102F800001F140022146C8F89800284605EB82026C
:102F90005360FFF76FFE08EB8900C3681B8A43EAA2
:102FA000845348341E4364012E51D5F81C381F4306
:102FB000C5F81C78BDE8F88305EB4917D7F8001B66
:102FC00021F40041C7F8001BD5F81C1821EA0303BF
:102FD000C0E704F13F030B4A2846214605EB830373
:102FE0005A60FFF747FE05EB4910D0F8003923F48B
:102FF0000043C0F80039D5F81C3823EA0707D7E7A3
:103000000080001000040002D0F894201268C0F87C
:103010009820FFF7C7BD00005831D0F89030490123
:103020005B5813F4004004D013F4001F0CBF0220BF
:10303000012070474831D0F8903049015B5813F4B3
:10304000004004D013F4001F0CBF02200120704781
:1030500000EB8101CB68196A0B6813604B68536001
:103060007047000000EB810330B5DD68AA69136882
:10307000D36019B9402B84BF402313606B8A146856
:10308000D0F890201C4402EB4110013C09B2B4FB83
:10309000F3F46343033323F0030343EAC44343F0ED
:1030A000C043C0F8103B2B6803F00303012B0ED183
:1030B000D2F8083802EB411013F4807FD0F8003BBF
:1030C00014BF43F0805343F00053C0F8003B02EBC1
:1030D0004112D2F8003B43F00443C2F8003B30BD3C
:1030E0002DE9F041D0F8906005460C4606EB4113FF
:1030F000D3F8087B3A07C3F8087B08D5D6F814380C
:103100001B0704D500EB8103DB685B689847FA076F
:103110001FD5D6F81438DB071BD505EB8403D96817
:10312000CCB98B69488A5A68B2FBF0F600FB1622CC
:103130008AB91868DA6890420DD2121AC3E90024DD
:10314000202383F3118821462846FFF78BFF84F361
:103150001188BDE8F081012303FA04F26B8923EAA8
:1031600002036B81CB68002BF3D021462846BDE8D3
:10317000F041184700EB81034A0170B5DD68D0F8D3
:1031800090306C692668E66056BB1A444FF4002004
:10319000C2F810092A6802F00302012A0AB20ED10D
:1031A000D3F8080803EB421410F4807FD4F8000928
:1031B00014BF40F0805040F00050C4F8000903EB09
:1031C0004212D2F8000940F00440C2F8000901227E
:1031D000D3F8340802FA01F10143C3F8341870BD82
:1031E00019B9402E84BF4020206020681A442E8ADE
:1031F0008419013CB4FBF6F440EAC44040F00050AE
:10320000C6E700002DE9F041D0F8906004460D4675
:1032100006EB4113D3F80879C3F80879FB071CD5EE
:10322000D6F81038DA0718D500EB8103D3F80CC0B4
:10323000DCF81430D3F800E0DA6896451BD2A2EB34
:103240000E024FF000081A60C3F80480202383F3B5
:103250001188FFF78FFF88F311883B0618D50123EB
:10326000D6F83428AB40134212D029462046BDE898
:10327000F041FFF7C3BC012303FA01F2038923EAFB
:1032800002030381DCF80830002BE6D09847E4E71E
:10329000BDE8F0812DE9F84FD0F8905004466E69F2
:1032A000AB691E4016F480586E6103D0BDE8F84F3C
:1032B000FEF744BC002E12DAD5F8003E9F0705D079
:1032C000D5F8003E23F00303C5F8003ED5F80438D6
:1032D000204623F00103C5F80438FEF75BFC3005F7
:1032E00005D52046FFF75EFC2046FEF743FCB104FF
:1032F0000CD5D5F8083813F0060FEB6823F470539B
:103300000CBF43F4105343F4A053EB60320704D5D1
:103310006368DB680BB120469847F30200F1BA807E
:10332000B70226D5D4F8909000274FF0010A09EB98
:103330004712D2F8003B03F44023B3F5802F11D19C
:10334000D2F8003B002B0DDA62890AFA07F322EA71
:103350000303638104EB8703DB68DB6813B1394641
:10336000204698470137D4F89430FFB29B689F42BB
:10337000DDD9F00619D5D4F89000026AC2F30A1715
:1033800002F00F0302F4F012B2F5802F00F0CC80AF
:10339000B2F5402F09D104EB8303002200F58050E1
:1033A000DB681B6A974240F0B2803003D5F81858AA
:1033B00035D5E90303D500212046FFF791FEAA0386
:1033C00003D501212046FFF78BFE6B0303D50221B5
:1033D0002046FFF785FE2F0303D503212046FFF784
:1033E0007FFEE80203D504212046FFF779FEA902FB
:1033F00003D505212046FFF773FE6A0203D5062197
:103400002046FFF76DFE2B0203D507212046FFF76C
:1034100067FEEF0103D508212046FFF761FE700328
:1034200040F1A980E90703D500212046FFF7EAFE15
:10343000AA0703D501212046FFF7E4FE6B0703D559
:1034400002212046FFF7DEFE2F0703D50321204689
:10345000FFF7D8FEEE0603D504212046FFF7D2FE83
:10346000A80603D505212046FFF7CCFE690603D543
:1034700006212046FFF7C6FE2A0603D5072120466F
:10348000FFF7C0FEEB0576D520460821BDE8F84FD2
:10349000FFF7B8BED4F8909000274FF0010AD4F897
:1034A00094305FFA87FB9B689B453FF639AF09EB89
:1034B0004B13D3F8002902F44022B2F5802F24D117
:1034C000D3F80029002A20DAD3F8002942F09042EC
:1034D000C3F80029D3F80029002AFBDB5946D4F8A9
:1034E0009000FFF7C7FB22890AFA0BF322EA0303D5
:1034F000238104EB8B03DB689B6813B1594620469C
:10350000984759462046FFF779FB0137C7E79107EF
:1035100001D1D0F80080072A02F101029CBF03F814
:10352000018B4FEA18283DE704EB830300F5805038
:10353000DA68D2F818C0DCF80820DCE9001CA1EB3E
:103540000C0C00218F4208D1DB689B699A683A44D1
:103550009A605A683A445A6027E711F0030F01D184
:10356000D0F800808C4501F1010184BF02F8018B85
:103570004FEA1828E6E7BDE8F88F000008B50348D1
:10358000FFF788FEBDE80840FFF784BA144E00201C
:1035900008B50348FFF77EFEBDE80840FFF77ABA9A
:1035A000B04E0020D0F8903003EB4111D1F8003B31
:1035B00043F40013C1F8003B70470000D0F890308E
:1035C00003EB4111D1F8003943F40013C1F800397D
:1035D00070470000D0F8903003EB4111D1F8003B68
:1035E00023F40013C1F8003B70470000D0F890307E
:1035F00003EB4111D1F8003923F40013C1F800396D
:1036000070470000090100F16043012203F56143A6
:10361000C9B283F8001300F01F039A4043099B00CE
:1036200003F1604303F56143C3F880211A607047DA
:1036300030B50433039C0172002104FB0325C160F3
:10364000C0E90653049B0363059BC0E90000C0E981
:103650000422C0E90842C0E90A11436330BD0000FA
:103660000022416AC260C0E90411C0E90A226FF079
:103670000101FEF7EDBD0000D0E90432934201D113
:10368000C2680AB9181D70470020704703691960A5
:103690000021C2680132C260C26913448269934248
:1036A000036124BF436A0361FEF7C6BD38B5044613
:1036B0000D46E3683BB162690020131D1268A362E6
:1036C0001344E36207E0237A33B929462046FEF724
:1036D000A3FD0028EDDA38BD6FF00100FBE7000024
:1036E000C368C269013BC360436913448269934262
:1036F000436124BF436A436100238362036B03B1C8
:103700001847704770B52023044683F31188866AF2
:103710003EB9FFF7CBFF054618B186F3118828465E
:1037200070BDA36AE26A13F8015B9342A36202D3FD
:103730002046FFF7D5FF002383F31188EFE7000051
:103740002DE9F84F04460E46174698464FF02009DB
:1037500089F311880025AA46D4F828B0BBF1000FE0
:1037600009D141462046FFF7A1FF20B18BF3118814
:103770002846BDE8F88FD4E90A12A7EB050B521AC8
:10378000934528BF9346BBF1400F1BD9334601F147
:10379000400251F8040B914243F8040BF9D1A36A9B
:1037A000403640354033A362D4E90A239A4202D31B
:1037B0002046FFF795FF8AF31188BD42D8D289F3DE
:1037C0001188C9E730465A46FDF73EFBA36A5E44BE
:1037D0005D445B44A362E7E710B5029C04330172C9
:1037E00004FB0321C460C0E906130023C0E90A33C7
:1037F000039B0363049BC0E90000C0E90422C0E905
:103800000842436310BD0000026A6FF00101C2600C
:10381000426AC0E904220022C0E90A22FEF718BD6C
:10382000D0E904239A4201D1C26822B9184650F85F
:10383000043B0B607047002070470000C368002104
:10384000C2690133C360436913448269934243618F
:1038500024BF436A4361FEF7EFBC000038B504465D
:103860000D46E3683BB1236900201A1DA262E2699C
:103870001344E36207E0237A33B929462046FEF772
:10388000CBFC0028EDDA38BD6FF00100FBE700004B
:1038900003691960C268013AC260C269134482694F
:1038A0009342036124BF436A036100238362036B75
:1038B00003B118477047000070B520230D46044639
:1038C000114683F31188866A2EB9FFF7C7FF10B13E
:1038D00086F3118870BDA36A1D70A36AE26A013382
:1038E0009342A36204D3E16920460439FFF7D0FF75
:1038F000002080F31188EDE72DE9F84F04460D46CE
:10390000904699464FF0200A8AF311880026B34664
:10391000A76A4FB949462046FFF7A0FF20B187F3B9
:1039200011883046BDE8F88FD4E90A073A1AA8EBA7
:103930000607974228BF1746402F1BD905F14003C1
:1039400055F8042B9D4240F8042BF9D1A36A403668
:103950004033A362D4E90A239A4204D3E1692046A2
:103960000439FFF795FF8BF311884645D9D28AF3C6
:103970001188CDE729463A46FDF766FAA36A3D4429
:103980003E443B44A362E5E7D0E904239A4217D1C1
:10399000C3689BB1836A8BB1043B9B1A0ED0136042
:1039A000C368013BC360C3691A4483699A420261D8
:1039B00024BF436A036100238362012318467047D2
:1039C0000023FBE700F0DAB8034B002258631A61CA
:1039D0000222DA60704700BF000C0040014B002259
:1039E000DA607047000C0040014B5863704700BF1D
:1039F000000C0040014B586A704700BF000C0040AB
:103A00004B6843608B688360CB68C3600B6943611C
:103A10004B6903628B6943620B6803607047000067
:103A200008B53C4B40F2FF713B48D3F888200A436D
:103A3000C3F88820D3F8882022F4FF6222F007021E
:103A4000C3F88820D3F88820D3F8E0200A43C3F8CD
:103A5000E020D3F808210A43C3F808212F4AD3F8FD
:103A600008311146FFF7CCFF00F5806002F11C0120
:103A7000FFF7C6FF00F5806002F13801FFF7C0FFD5
:103A800000F5806002F15401FFF7BAFF00F5806095
:103A900002F17001FFF7B4FF00F5806002F18C01C4
:103AA000FFF7AEFF00F5806002F1A801FFF7A8FF65
:103AB00000F5806002F1C401FFF7A2FF00F580600D
:103AC00002F1E001FFF79CFF00F5806002F1FC01CC
:103AD000FFF796FF02F58C7100F58060FFF790FF0D
:103AE00000F000F90E4BD3F8902242F00102C3F827
:103AF0009022D3F8942242F00102C3F894220522C6
:103B0000C3F898204FF06052C3F89C20054AC3F8D0
:103B1000A02008BD00440258000002589C43000841
:103B200000ED00E01F00080308B500F0F3FAFEF70F
:103B3000E3FA0F4BD3F8DC2042F04002C3F8DC205C
:103B4000D3F8042122F04002C3F80421D3F8043151
:103B5000084B1A6842F008021A601A6842F0040220
:103B60001A60FEF749FFBDE80840FEF7EDBC00BF54
:103B7000004402580018024870470000114BD3F867
:103B8000E82042F00802C3F8E820D3F8102142F000
:103B90000802C3F810210C4AD3F81031D36B43F05C
:103BA0000803D363C722094B9A624FF0FF32DA62EF
:103BB00000229A615A63DA605A6001225A611A60DF
:103BC000704700BF004402580010005C000C004029
:103BD000094A08B51169D3680B40D9B29B076FEA4F
:103BE0000101116107D5202383F31188FEF7A4FAA0
:103BF000002383F3118808BD000C0040384B4FF0C0
:103C0000FF31D3F88020C3F88010D3F88020002241
:103C1000C3F88020D3F88000D3F88400C3F8841060
:103C2000D3F88400C3F88420D3F88400D86F40F020
:103C3000FF4040F4FF0040F43F5040F03F00D867A1
:103C4000D86F20F0FF4020F4FF0020F43F5020F018
:103C50003F00D867D86FD3F888006FEA40506FEA0A
:103C60005050C3F88800D3F88800C0F30A00C3F8A6
:103C70008800D3F88800D3F89000C3F89010D3F8E8
:103C80009000C3F89020D3F89000D3F89400C3F8C4
:103C90009410D3F89400C3F89420D3F89400D3F888
:103CA0009800C3F89810D3F89800C3F89820D3F878
:103CB0009800D3F88C00C3F88C10D3F88C00C3F8AC
:103CC0008C20D3F88C00D3F89C00C3F89C10D3F858
:103CD0009C10C3F89C20D3F89C3000F0E7B900BFDB
:103CE00000440258614B0122C3F80821604BD3F80D
:103CF000F42042F00202C3F8F420D3F81C2142F071
:103D00000202C3F81C210222D3F81C31594BDA609D
:103D10005A689104FCD5584A1A6001229A60574AA1
:103D2000DA6000221A614FF440429A61514B9A695D
:103D30009204FCD51A6842F480721A604C4B1A6FD8
:103D400012F4407F04D04FF480321A6700221A67C1
:103D50001A6842F001021A60454B1A685007FCD5F8
:103D600000221A611A6912F03802FBD10121196090
:103D70004FF0804159605A67414ADA62414A1A61FC
:103D80001A6842F480321A60394B1A689103FCD5E4
:103D90001A6842F480521A601A689204FCD53A4AB2
:103DA0003A499A6200225A6319633949DA6399637E
:103DB0005A64384A1A64384ADA621A6842F0A852D9
:103DC0001A602B4B1A6802F02852B2F1285FF9D121
:103DD00048229A614FF48862DA6140221A622F4ABF
:103DE000DA644FF080521A652D4A5A652D4A9A6559
:103DF00032232D4A1360136803F00F03022BFAD10C
:103E00001B4B1A6942F003021A611A6902F0380268
:103E1000182AFAD1D3F8DC2042F00052C3F8DC2093
:103E2000D3F8042142F00052C3F80421D3F804214E
:103E3000D3F8DC2042F08042C3F8DC20D3F8042120
:103E400042F08042C3F80421D3F80421D3F8DC20E7
:103E500042F00042C3F8DC20D3F8042142F00042D3
:103E6000C3F80421D3F80431704700BF008000512B
:103E7000004402580048025800C000F0020000014F
:103E80000000FF0100889008222040006302090121
:103E90002C02040047040508FD0BFF012000002050
:103EA0000010E00000010100002000524FF0B0427D
:103EB00008B5D2F8883003F00103C2F8883023B186
:103EC000044A13680BB150689847BDE80840FEF7F4
:103ED000E1BD00BF644F00204FF0B04208B5D2F8FA
:103EE000883003F00203C2F8883023B1044A936893
:103EF0000BB1D0689847BDE80840FEF7CBBD00BFC6
:103F0000644F00204FF0B04208B5D2F8883003F07B
:103F10000403C2F8883023B1044A13690BB1506915
:103F20009847BDE80840FEF7B5BD00BF644F0020CC
:103F30004FF0B04208B5D2F8883003F00803C2F859
:103F4000883023B1044A93690BB1D0699847BDE822
:103F50000840FEF79FBD00BF644F00204FF0B04205
:103F600008B5D2F8883003F01003C2F8883023B1C6
:103F7000044A136A0BB1506A9847BDE80840FEF73F
:103F800089BD00BF644F00204FF0B04310B5D3F897
:103F9000884004F47872C3F88820A30604D5124A36
:103FA000936A0BB1D06A9847600604D50E4A136B2A
:103FB0000BB1506B9847210604D50B4A936B0BB19C
:103FC000D06B9847E20504D5074A136C0BB1506CCF
:103FD0009847A30504D5044A936C0BB1D06C98475D
:103FE000BDE81040FEF756BD644F00204FF0B043CF
:103FF00010B5D3F8884004F47C42C3F888206205E9
:1040000004D5164A136D0BB1506D9847230504D59E
:10401000124A936D0BB1D06D9847E00404D50F4A56
:10402000136E0BB1506E9847A10404D50B4A936EE2
:104030000BB1D06E9847620404D5084A136F0BB1D8
:10404000506F9847230404D5044A936F0BB1D06F87
:104050009847BDE81040FEF71DBD00BF644F00202B
:1040600008B50348FDF70CF9BDE80840FEF712BD9E
:10407000DC23002008B50348FDF702F9BDE808403D
:10408000FEF708BD4824002008B50348FDF7F8F8FE
:10409000BDE80840FEF7FEBCB424002008B5FFF7D9
:1040A00097FDBDE80840FEF7F5BC0000062108B505
:1040B0000846FFF7A7FA06210720FFF7A3FA062113
:1040C0000820FFF79FFA06210920FFF79BFA062137
:1040D0000A20FFF797FA06211720FFF793FA062127
:1040E0002820FFF78FFA09217A20FFF78BFA0721A2
:1040F0003220FFF787FA0C212720FFF783FA0C21E3
:104100003520FFF77FFA0C215220BDE80840FFF769
:1041100079BA000008B5FFF771FD00F00DF8FDF762
:10412000C1FAFDF799FCFDF76BFBFFF725FDBDE834
:104130000840FFF747BC00000023054A1946013339
:10414000102BC2E9001102F10802F8D1704700BF3C
:10415000644F002010B501390244904201D1002083
:1041600005E0037811F8014FA34201D0181B10BDE0
:104170000130F2E7034611F8012B03F8012B002A66
:10418000F9D1704753544D333248373F3F3F0053C6
:10419000544D3332483734332F3735330000000065
:1041A00001105A0003105900012058000320560046
:1041B0000096000000000000000000000000000069
:1041C0000000000000000000000000006D16000864
:1041D0005916000895160008811600088D1600086B
:1041E000791600086516000851160008A116000887
:1041F000000000007D17000869170008A5170008D7
:10420000911700089D170008891700087517000806
:1042100061170008B117000800000000010000004D
:10422000000000006D61696E0000000069646C654B
:10423000000000002C42000860310020D83200202D
:1042400001000000F520000800000000486F6C79B4
:1042500062726F0025424F415244252D424C002589
:1042600053455249414C2500020000000000000067
:104270009D1900080D1A000840004000804B0020E6
:10428000904B00200200000000000000030000002E
:1042900000000000551A0008000000001000000097
:1042A000A04B002000000000010000000000000002
:1042B000144E002001010200E5240008F523000847
:1042C000912400087524000843000000D042000833
:1042D00009024300020100C0320904000001020289
:1042E000010005240010010524010001042402023C
:1042F0000524060001070582030800FF09040100E8
:10430000020A0000000705010240000007058102C3
:1043100040000000120000001C43000812011001C0
:10432000020000406231530000020102030100005C
:104330000403090425424F4152442500506978681E
:1043400061776B36432D626473686F74003031326D
:10435000333435363738394142434445460000004E
:1043600000000000A91B0008611E00080D1F0008C6
:10437000400040004C4F00204C4F00200100000046
:104380005C4F002080000000400100000800000099
:104390000001000000040000080000000000802A66
:1043A00000020000AAAAAAAA00000024FFFF000041
:1043B0000000000000A00A00000000000000000053
:1043C000AAAAAAAA00000000FFFF00000000000047
:1043D000000000000000105600000000AAAAAAAACF
:1043E00000000055FFFF0000000000000000080072
:1043F00020015A00000C0000AAAAAAAA1001050078
:10440000FFFF00000008000077000000108002009D
:1044100000000000AAAAAAAA00400100FFFF0000B5
:104420000000007007000000000000000000000015
:10443000AAAAAAAA00000000FFFF000000000000D6
:10444000000000000000000000000000AAAAAAAAC4
:1044500000000000FFFF000000000000000000005E
:104460000000000000000000AAAAAAAA00000000A4
:10447000FFFF00000000000000000000000000003E
:1044800000000000AAAAAAAA00000000FFFF000086
:10449000000000000000000000000000000000001C
:1044A000AAAAAAAA00000000FFFF00000000000066
:1044B000000000000000000000000000AAAAAAAA54
:1044C00000000000FFFF00000000000000000000EE
:1044D000380000000000000000001E000000000086
:1044E000FF000000D8320020B4240020482400201F
:1044F000DC23002000000000844100083F00000091
:10450000500400008F4100083F00000000960000AA
:1045100000000800960000000008000004000000F1
:104520003043000800000000000000000000000010
:10453000000000000000000000000000FFFFFFFF7F
:10454000FFFFFFFFFFFFFFFFFFFFFFFFFFFFFFFF7B
:10455000FFFFFFFFFFFFFFFFFFFFFFFFFFFFFFFF6B
:10456000FFFFFFFFFFFFFFFFFFFFFFFFFFFFFFFF5B
:10457000FFFFFFFFFFFFFFFFFFFFFFFFFFFFFFFF4B
:020000040801F1
:020000040802F0
:1000000000060024BD0D0208099E0A0871030208BB
:10001000919D0A08899D0A088D9D0A08BF0D020856
:10002000BF0D0208BF0D0208BF0D02080DA40F0886
:10003000BF0D0208BF0D0208BF0D0208BF0D020868
:10004000BF0D0208BF0D0208BF0D0208BF0D020858
:10005000BF0D0208BF0D0208E5171008111810089F
:100060003D1810086918100895181008C1B10F083C
:10007000E9B10F0815B20F0841B20F086DB20F08B1
:1000800095B20F08C1B20F08E5AD0F08918E0A08AE
:10009000B98E0A08A58E0A08CD8E0A08C118100864
:1000A000BF0D0208391A1008BF0D02084D1A1008BA
:1000B000511A1008611A1008751A10087DBA0F0835
:1000C000ADBA0F08DDBA0F080DBB0F08F9C40F0851
:1000D0000DC50F08AD191008C1191008D519100861
:1000E00025191008BF0D0208BF0D0208BF0D020838
:1000F000BF0D0208BF0D0208BF0D0208EDB20F08C8
:10010000BF0D0208BF0D0208891A1008BF0D0208B2
:10011000BF0D0208E9191008BF0D0208BF0D020843
:1001200019B30F0841B30F086DB30F0899B30F0847
:10013000C5B30F08BF0D0208BF0D0208BF0D0208AE
:10014000BF0D0208BF0D0208BF0D0208BF0D020857
:10015000EDB30F0819B40F0845B40F08FD191008C6
:10016000BF0D0208BF0D0208BF0D0208BF0D020837
:10017000BF0D020845141008BF0D0208BF0D02088C
:10018000BF0D0208BF0D0208111A1008251A100829
:10019000BF0D0208BF0D0208BF0D0208BF0D020807
:1001A000BF0D0208BF0D0208BF0D0208BF0D0208F7
:1001B000BF0D0208BF0D0208BF0D02083DBB0F08AE
:1001C0006DBB0F08BF0D0208BF0D0208BF0D02086E
:1001D000BF0D020831141008BF0D0208BF0D020840
:1001E000BF0D0208BF0D0208BF0D0208BF0D0208B7
:1001F000BF0D0208BF0D0208BF0D0208BF0D0208A7
:10020000BF0D0208BF0D0208BF0D0208BF0D020896
:10021000BF0D0208BF0D0208BF0D0208BF0D020886
:10022000BF0D0208BF0D0208BF0D0208BF0D020876
:1002300099191008BF0D0208BF0D020805AE0F087E
:10024000BF0D02088DAF0F08B5AF0F08E1AF0F0863
:100250000DB00F0839B00F0865B00F0891B00F0846
:10026000BDB00F08BF0D0208BF0D0208BF0D020888
:10027000BF0D0208BF0D0208BF0D0208BF0D020826
:10028000BF0D0208BF0D0208BF0D0208BF0D020816
:10029000BF0D0208BF0D0208BF0D0208BF0D020806
:1002A000BF0D0208BF0D0208BF0D0208BF0D0208F6
:1002B000BF0D0208BF0D0208BF0D0208BF0D0208E6
:1002C000BF0D0208BF0D0208BF0D0208BF0D0208D6
:1002D000BF0D0208BF0D0208BF0D0208BF0D0208C6
:1002E000C52D020805C30208B9040308698503087F
:1002F00045C20408C5F906088D220708458F07087E
:10030000B5980708059C0708712208080129080804
:10031000CD48080845510808596F080815250908EF
:10032000F931090875910A0885960A0871B20A0818
:1003300085270C08C1660C086DB60C08B9D30C08EB
:10034000B9D00D08BD350E0891500E08D16C0E08BD
:100350006D840E08E5AE0E081DC60E08FDF80E08E9
:1003600015000F08FFFFFFFFFFFFFFFFFFFFFFFF6D
:10037000EFF30383EFF30982EFF30881DFF814D082
:100380002DE9FE4F684600F0E3FFBDE8FE4F8D46C5
:1003900070470000642C0024F1EE101AA0EC200A33
:1003A00001607047A0EC108A704700BF81F00041E7
:1003B00002E000BF83F0004330B54FEA41044FEA4A
:1003C000430594EA050F08BF90EA020F1FBF54EAE5
:1003D000000C55EA020C7FEA645C7FEA655C00F081
:1003E000E2804FEA5454D4EB5555B8BF6D420CDD52
:1003F0002C4480EA020281EA030382EA000083EAD5
:10040000010180EA020281EA0303362D88BF30BD74
:1004100011F0004F4FEA01314FF4801C4CEA1131CA
:1004200002D0404261EB410113F0004F4FEA033329
:100430004CEA133302D0524263EB430394EA050FB4
:1004400000F0A780A4F10104D5F1200E0DDB02FA23
:100450000EFC22FA05F2801841F1000103FA0EF2B7
:10046000801843FA05F359410EE0A5F120050EF17D
:10047000200E012A03FA0EFC28BF4CF0020C43FAAE
:1004800005F3C01851EBE37101F0004507D54FF0BB
:10049000000EDCF1000C7EEB00006EEB0101B1F50B
:1004A000801F1BD3B1F5001F0CD349085FEA300051
:1004B0004FEA3C0C04F101044FEA445212F5800F5C
:1004C00080F09A80BCF1004F08BF5FEA500C50F1F9
:1004D000000041EB045141EA050130BD5FEA4C0CDC
:1004E000404141EB0101013C28BFB1F5801FE9D239
:1004F00091F0000F04BF01460020B1FA81F308BF5C
:100500002033A3F10B03B3F120020CDA0C3208DD27
:1005100002F1140CC2F10C0201FA0CF021FA02F102
:100520000CE002F11402D8BFC2F1200C01FA02F172
:1005300020FA0CFCDCBF41EA0C019040E41AA2BF97
:1005400001EB0451294330BD6FEA04041F3C1CDA5F
:100550000C340EDC04F11404C4F1200220FA04F07F
:1005600001FA02F340EA030021FA04F345EA030129
:1005700030BDC4F10C04C4F1200220FA02F001FAEB
:1005800004F340EA0300294630BD21FA04F029466D
:1005900030BD94F0000F83F4801306BF81F4801106
:1005A0000134013D4EE77FEA645C18BF7FEA655C79
:1005B00029D094EA050F08BF90EA020F05D054EA4B
:1005C000000C04BF1946104630BD91EA030F1EBF50
:1005D0000021002030BD5FEA545C05D14000494154
:1005E00028BF41F0004130BD14F580043CBF01F547
:1005F000801130BD01F0004545F0FE4141F470012D
:100600004FF0000030BD7FEA645C1ABF1946104607
:100610007FEA655C1CBF0B46024650EA013406BF08
:1006200052EA033591EA030F41F4002130BD00BFC7
:1006300090F0000F04BF0021704730B54FF4806484
:1006400004F132044FF000054FF0000150E700BF05
:1006500090F0000F04BF0021704730B54FF4806464
:1006600004F1320410F0004548BF40424FF0000151
:100670003EE700BF42004FEAE2014FEA31014FEA94
:1006800002701FBF12F07F4393F07F4F81F06051E3
:10069000704732F07F4208BF704793F07F4F04BF2E
:1006A00041F40021704730B54FF4607401F000450B
:1006B00021F000411CE700BF50EA010208BF70476B
:1006C00030B54FF000050AE050EA010208BF70475C
:1006D00030B511F0004502D5404261EB41014FF4C5
:1006E000806404F132045FEA915C3FF4D8AE4FF0CD
:1006F00003025FEADC0C18BF03325FEADC0C18BFB0
:10070000033202EBDC02C2F1200300FA03FC20FA00
:1007100002F001FA03FE40EA0E0021FA02F114444D
:10072000BDE600BF80F0004002E000BF81F0004164
:1007300042001FBF5FEA410392EA030F7FEA226C87
:100740007FEA236C6AD04FEA1262D2EB1363C1BF17
:10075000D218414048404140B8BF5B42192B88BF86
:10076000704710F0004F40F4000020F07F4018BFA9
:10077000404211F0004F41F4000121F07F4118BFC9
:10078000494292EA030F3FD0A2F1010241FA03FC71
:1007900010EB0C00C3F1200301FA03F100F0004359
:1007A00002D5494260EB4000B0F5000F13D3B0F121
:1007B000807F06D340084FEA310102F10102FE2A90
:1007C00051D2B1F1004F40EBC25008BF20F0010000
:1007D00040EA03007047490040EB0000013A28BF9F
:1007E000B0F5000FEDD2B0FA80FCACF1080CB2EB22
:1007F0000C0200FA0CF0AABF00EBC25052421843A0
:10080000BCBFD0401843704792F0000F81F4000144
:1008100006BF80F400000132013BB5E74FEA410317
:100820007FEA226C18BF7FEA236C21D092EA030F83
:1008300004D092F0000F08BF0846704790EA010FFD
:100840001CBF0020704712F07F4F04D1400028BF2A
:1008500040F00040704712F100723CBF00F500000C
:10086000704700F0004343F0FE4040F40000704742
:100870007FEA226216BF08467FEA236301464202EE
:1008800006BF5FEA412390EA010F40F48000704701
:100890004FF0000304E000BF10F0004348BF4042A7
:1008A0005FEA000C08BF704743F0964301464FF0E3
:1008B00000001CE050EA010208BF70474FF000033F
:1008C0000AE000BF50EA010208BF704711F0004380
:1008D00002D5404261EB41015FEA010C02BF844650
:1008E0000146002043F0B64308BFA3F18053A3F5AF
:1008F0000003BCFA8CF2083AA3EBC25310DB01FAF6
:1009000002FC634400FA02FCC2F12002BCF1004F79
:1009100020FA02F243EB020008BF20F0010070470A
:1009200002F1200201FA02FCC2F1200250EA4C005E
:1009300021FA02F243EB020008BF20EADC707047A4
:100940007BB972B90029BEBF00204FF0004106E01C
:1009500008BF00281CBF6FF000414FF0FF3000F0CF
:100960002BBAADF1080C6DE904CE002909DB002B90
:100970001ADB00F0B9F8DDF804E0DDE9022304B089
:100980007047404261EB4101002B1BDB00F0ACF8EB
:10099000DDF804E0DDE9022304B0404261EB4101EF
:1009A000524263EB43037047524263EB430300F050
:1009B0009BF8DDF804E0DDE9022304B0404261EB7E
:1009C00041017047524263EB430300F08DF8DDF8BC
:1009D00004E0DDE9022304B0524263EB43037047B5
:1009E00053B94AB9002908BF00281CBF4FF0FF3196
:1009F0004FF0FF3000F0E0B9ADF1080C6DE904CE26
:100A000000F072F8DDF804E0DDE9022304B070477D
:100A1000430803F05533C01A830803F0333300F062
:100A20003330184400EB101000F00F3000EB0020C2
:100A300000EB0040000E704708B502460B4643EC41
:100A4000172BB5EEC07BF1EE10FA03D4BDE80840D9
:100A500000F02AB8B1EE477B51EC170B00F024F8F8
:100A6000404261EB410108BD9FED0B6B07EE900A20
:100A70009FED0B5BB7EEE77A27EE066BBCEEC66B1D
:100A8000B8EE464BA4EE457BFCEEC77B16EE101A83
:100A900017EE900A704700BF000000000000F03D14
:100AA000000000000000F0419FED0B6B41EC170BC4
:100AB0009FED0B5B27EE066BBCEEC66BB8EE464BAC
:100AC000A4EE457BFCEEC77B16EE101A17EE900ADB
:100AD000704700BFAFF30080000000000000F03D51
:100AE000000000000000F0412DE9F047089D044699
:100AF0008E46002B4DD18A42944669D9B2FA82F2D1
:100B000052B101FA02F3C2F1200120FA01F10CFA0C
:100B100002FC41EA030E94404FEA1C48210CBEFB44
:100B2000F8F61FFA8CF708FB16E341EA034306FBCD
:100B300007F199420AD91CEB030306F1FF3080F05C
:100B40001F81994240F21C81023E63445B1AA4B2A9
:100B5000B3FBF8F008FB103344EA034400FB07F74B
:100B6000A7420AD91CEB040400F1FF3380F00A818C
:100B7000A74240F207816444023840EA0640E41B81
:100B800000261DB1D4400023C5E900433146BDE82D
:100B9000F0878B4209D9002D00F0EF800026C5E9CF
:100BA000000130463146BDE8F087B3FA83F6002EE7
:100BB0004AD18B4202D3824200F2F980841A61EB5F
:100BC000030301209E46002DE0D0C5E9004EDDE77D
:100BD00002B9FFDEB2FA82F2002A40F09280A1EB65
:100BE0000C014FEA1C471FFA8CFE0126200CB1FBBA
:100BF000F7F307FB131140EA01410EFB03F08842B3
:100C000008D91CEB010103F1FF3802D2884200F23F
:100C1000CB804346091AA4B2B1FBF7F007FB1011D1
:100C200044EA01440EFB00FEA64508D91CEB04046F
:100C300000F1FF3102D2A64500F2BB800846A4EBCA
:100C40000E0440EA03409CE7C6F12007B34022FAB5
:100C500007FC4CEA030C20FA07F401FA06F31C43E4
:100C6000F9404FEA1C4900FA06F3B1FBF9F8200CF1
:100C70001FFA8CFE09FB181140EA014108FB0EF037
:100C8000884202FA06F20BD91CEB010108F1FF3A87
:100C900080F08880884240F28580A8F10208614493
:100CA000091AA4B2B1FBF9F009FB101144EA0141A1
:100CB00000FB0EFE8E4508D91CEB010100F1FF344C
:100CC0006CD28E456AD90238614440EA0840A0FBE4
:100CD0000294A1EB0E01A142C846A64656D353D0BA
:100CE0005DB1B3EB080261EB0E0101FA07F722FADE
:100CF00006F3F1401F43C5E9007100263146BDE807
:100D0000F087C2F12003D8400CFA02FC21FA03F369
:100D1000914001434FEA1C471FFA8CFEB3FBF7F0EA
:100D200007FB10360B0C43EA064300FB0EF69E420F
:100D300004FA02F408D91CEB030300F1FF382FD2A8
:100D40009E422DD9023863449B1B89B2B3FBF7F650
:100D500007FB163341EA034106FB0EF38B4208D929
:100D60001CEB010106F1FF3816D28B4214D9023E6A
:100D70006144C91A46EA004638E72E46284605E788
:100D80000646E3E61846F8E64B45A9D2B9EB020859
:100D900064EB0C0E0138A3E74646EAE7204694E7E9
:100DA0004046D1E7D0467BE7023B614432E730461C
:100DB00009E76444023842E7704700BF02E000F0F0
:100DC00000F8FEE772B6374880F30888364880F3AB
:100DD000098836483649086040F20000CCF200002D
:100DE0004EF63471CEF200010860BFF34F8FBFF3AF
:100DF0006F8F40F20000C0F2F0004EF68851CEF244
:100E000000010860BFF34F8FBFF36F8F4FF00000FA
:100E1000E1EE100A4EF63C71CEF2000108600620A9
:100E200080F31488BFF36F8FDFF078FDDEF0E4FB12
:100E30004FF055301F491B4A91423CBF41F8040B0B
:100E4000FAE71D49184A91423CBF41F8040BFAE702
:100E50001A491B4A1B4B9A423EBF51F8040B42F8F9
:100E6000040BF8E700201849184A91423CBF41F8AA
:100E7000040BFAE7DFF090FDDEF042FC144C154D58
:100E8000AC4203DA54F8041B8847F9E701F0ECFEA2
:100E9000114C124DAC4203DA54F8041B8847F9E7B1
:100EA000DFF078BD000600240022002400000208C4
:100EB00008ED00E000000024000600241052140891
:100EC000002200246C2A0024702A00245CEA0124F9
:100ED000E0020208640302086403020864030208D3
:100EE0002DE9F04F2DED108AC1F80CD0D0F80CD0C0
:100EF000BDEC108ABDE8F08F002383F311882846EB
:100F0000A0470020DEF0FEF8FEE7DDF067FF00DF1F
:100F1000FEE7000070B54FF0FF0C4CF4E06C1CEAEB
:100F200011541DBF1CEA135594EA0C0F95EA0C0FDF
:100F300000F0DEF82C4481EA030621EA4C5123EA52
:100F40004C5350EA013518BF52EA033541F4801181
:100F500043F4801338D0A0FB02CE4FF00005E1FB34
:100F600002E506F00042E0FB03E54FF00006E1FB7E
:100F700003569CF0000F18BF4EF0010EA4F1FF04C1
:100F8000B6F5007F64F5407404D25FEA4E0E6D4101
:100F900046EB060642EAC62141EA55514FEAC52012
:100FA00040EA5E504FEACE2EB4F1FD0C88BFBCF58E
:100FB000E06F1ED8BEF1004F08BF5FEA500E50F13F
:100FC000000041EB045170BD06F0004646EA010105
:100FD00040EA020081EA0301B4EB5C04C2BFD4EB37
:100FE0000C0541EA045170BD41F480114FF0000E30
:100FF000013C00F3AB8014F1360FDEBF002001F09E
:10100000004170BDC4F10004203C35DA0C341BDC17
:1010100004F11404C4F1200500FA05F320FA04F0E9
:1010200001FA05F240EA020001F0004221F000411D
:1010300010EBD37021FA04F642EB06015EEA430E90
:1010400008BF20EAD37070BDC4F10C04C4F12005C0
:1010500000FA04F320FA05F001FA04F240EA020073
:1010600001F0004110EBD37041F100015EEA430E44
:1010700008BF20EAD37070BDC4F1200500FA05F264
:101080004EEA020E20FA04F301FA05F243EA0203E3
:1010900021FA04F001F0004121FA04F220EA0200F2
:1010A00000EBD3705EEA430E08BF20EAD37070BD38
:1010B00094F0000F0FD101F00046400041EB010118
:1010C00011F4801F08BF013CF7D041EA060195F0FA
:1010D000000F18BF704703F00046520043EB0303B4
:1010E00013F4801F08BF013DF7D043EA06037047A1
:1010F00094EA0C0F0CEA135518BF95EA0C0F0CD0AC
:1011000050EA410618BF52EA4306D1D181EA0301F1
:1011100001F000414FF0000070BD50EA410606BFEB
:101120001046194652EA430619D094EA0C0F02D130
:1011300050EA013613D195EA0C0F05D152EA033675
:101140001CBF104619460AD181EA030101F0004193
:1011500041F0FE4141F470014FF0000070BD41F0DC
:10116000FE4141F4780170BD4FEA410212F50012D0
:1011700015D211D56FF47873B3EB625212D94FEADE
:10118000C12343F0004343EA505311F0004F23FAC8
:1011900002F018BF404270474FF00000704750EA1D
:1011A000013005D111F0004008BF6FF000407047DA
:1011B0004FF00000704700BF4FEA4102B2F1E04338
:1011C00024BFB3F5001CDCF1FE5C0DD901F0004C2E
:1011D0004FEAC0024CEA5070B2F1004F40EB83007E
:1011E00008BF20F00100704711F0804F21D113F1AA
:1011F0003872BCBF01F00040704741F480114FEAE3
:101200005252C2F11802C2F1200C10FA0CF320FA6B
:1012100002F018BF40F001004FEAC1234FEAD32388
:1012200003FA0CFC40EA0C0023FA02F34FEA4303F2
:10123000CCE77FEA625307D150EA01331EBF4FF07B
:10124000FE4040F44000704701F0004040F0FE4096
:1012500040F40000704700BF01F0FF01102A2BDBB3
:1012600010F0070F08D010F8013B013A8B422DD047
:1012700010F0070F42B3F6D1F0B441EA012141EA80
:10128000014122F007047FF000070023F0E8025636
:10129000083C85EA010586EA010685FA47F5A3FAC6
:1012A00087F586FA47F6A5FA87F68EB9EED1F0BC37
:1012B00001F0FF0102F0070232B110F8013B013AE0
:1012C00083EA010313B1F8D1002070470138704759
:1012D000002D06BF35460338073815F0010F07D13A
:1012E000013015F4807F02BF013015F4C03F01309A
:1012F000F0BC0138704700BF10F8012B11F8013B1A
:10130000012A28BF9A42F7D0D01A7047034613F833
:10131000012B002AFBD1181A0138704710B504467A
:1013200020461CB154F80C3B013300D110BD0822FB
:10133000012100F071FB54F80C0C54F8082C14F83F
:10134000041C121AB2FBF1F200F066FBE8E70000A1
:10135000C26AD0E9003112F0040F2DE9F04118BF44
:101360000B46A6B00021594C042601270291CDE975
:101370000003D0064CBF03F1200203F16802039280
:10138000DA690399D2099B6902F004021B880A43B7
:1013900003F47F4303924FF0E022A3F53E41D2F8DD
:1013A000882D02F4A002B2F5A00F04BF0122029220
:1013B0004B424B410493464D03A82C6000F02AFA9F
:1013C00004220121434800F027FB0422012102A846
:1013D00000F022FB10220121019800F01DFB009873
:1013E000202201210C3000F017FB0198042201217A
:1013F000103000F011FB0422012103A800F00CFBC7
:1014000001980C220121143000F006FB0C2201216E
:10141000009800F001FB029BDA071FD5009BDB6AF6
:10142000DB064ED415A8FEF7BDFFDDF804C00DF1B4
:10143000140E0CF120030CF160081868083353F8FF
:10144000041C7246434503C29646F6D1DCF8603070
:1014500025938422012105A800F0DEFA00F0C0F8EF
:10146000FFF75CFF4FF0E023D3F8003D03F4702357
:10147000B3F5402F0ED0184B05A88DF81C600593CE
:1014800014338DF8287006934FF0FF33CDE90833FD
:10149000FFF744FF2B68A34206D0104B0422012122
:1014A00005A8059300F0B8FA00F02AFA002882D0C7
:1014B000049B1BB1019A93690233936126B0BDE886
:1014C000F08105A8FEF768FFC3E700BFED55CEAC7D
:1014D000702A002494A1100828ED00E0ACCE55ED50
:1014E00037B50E4D2A78202A15D10D4C0D482368AA
:1014F0000D4918440192DEF0A5FB23680021019AF2
:101500002033094829702360E4F096FC03B0BDE85D
:101510003040DFF017B903B030BD00BF642C0024A9
:101520008C2C0024805A1408662C002408B5352021
:10153000DBF0C4FE144BD3F8902042F48012C3F8C1
:101540009020D3F8902022F48012C3F89020D3F892
:101550009020D3F8E82042F48012C3F8E820D3F8B2
:10156000102142F48012C3F810216D22D3F81031FB
:10157000064BDA604FF0FF321A620D221A60012228
:10158000034B1A7008BD00BF0044025800500040D1
:101590009C2C0024014B1868704700BFFCFF1F08FB
:1015A000014B0248C01A7047805A140800002008F6
:1015B00000487047805A140807490022074B5B1AFD
:1015C0009A4201D30120704751F8040B013001D138
:1015D0000432F5E700207047805A14080000200804
:1015E0005E4B2DE9F74F1A6802255D4B02F56A58EC
:1015F000DFF894911A7808F118085A4F5A4C904421
:10160000DFF888A1DDF002FBA9EB070B06460EB15F
:101610004E2D49D9A9EB0702B2EB080700F19280E1
:101620004E2D00F28F80DFF868C16B1C4F4E0C21ED
:10163000DBB2ACEB06006943B84273DD60184FF0D3
:10164000010C665090463E4480F808C04660B2EBFC
:10165000080213D44F2B11D0454E19464548AB1CF8
:10166000351ADBB295424FF00C0505FB01F163DD45
:1016700065180126024460502E726A600C22012116
:101680005343E21811724FF0FF31E15051603A4B71
:101690001B782BB1394B1B682360394B1B68636087
:1016A000314803B0BDE8F08F336AF06953450ABF93
:1016B000344BF31AA3EB0A0380B10193DEF0B0FCC4
:1016C000019B58B12A460C2101354A430121EDB254
:1016D000A0180172F169A1500D3141600C20012167
:1016E000984400FB05FCD84504EB0C0244F80C6060
:1016F00006F13C0C1172C2F804C005EB010205F1C1
:101700000205D2B2EDB200FB02F204EB020001725C
:10171000316AA1501944416014D23046DDF086FA96
:10172000064674E767184FF0010E8044665087F84C
:1017300008E0C7F804C08AE76218012560501572F6
:1017400056609BE74F2D01D82B4697E7012384F87D
:10175000BC334FF0FF33C4E9ED3398E78C2C002401
:10176000642C0024805A140804220024702A0024C7
:101770000000082460EA012400220024902C0024A8
:10178000882C0024002200240000200800060024E9
:101790005CEA01240C4B1B7810B50BB9FFF7C6FEB1
:1017A00000230A490A48CA699206FCD54A6A1C5CA9
:1017B000D2B2944205D10133DBB20E2BF3D100201B
:1017C00010BD0023EFE700BF9C2C00240050004018
:1017D00098A1100838B5084B04461B780BB9FFF7E1
:1017E000A5FEE4B2054DAC62EB695B0600D538BDE1
:1017F000DEF0A8FFF8E700BF9C2C0024005000405A
:1018000010B5441E14F8010F00B910BDFFF7E2FF38
:10181000F8E7000070B502680446EFF30581D920AF
:101820005369C9B288F0B6FA294B1B78A3B1294B8A
:1018300094E8030083E803002748FFF7E1FF6368AB
:10184000B3B12648FFF7DCFF2548FFF7D9FFFFF7C4
:10185000A1FF2448FFF7D4FF234D2B783BB1246828
:101860001CB12046DEF0DCFB20B900232B7070BDDC
:101870001E48E7E720461E4EDEF0E6FB00F214505D
:1018800084421FD22046DEF0DFFB30602046194E36
:10189000DEF0EEFB04F5E053834217D92046DEF07C
:1018A000E7FB30600023144A1360144A1370FFF7FB
:1018B00083FE0028D9D0DEF045FF0120BDE870404E
:1018C000DEF048BAA4F214533360DFE73360E9E78F
:1018D000652C0024942C0024A8A11008ADA11008A8
:1018E000BEA110088479110800220024B8A11008B4
:1018F000902C0024882C00248C2C0024642C0024A0
:10190000284B1A7870B542B12748FFF779FF274B6B
:101910005868003818BF012070BD254A107800288B
:101920003CD0244E244C33682448254D1A1D217880
:101930002D1A0A44AA4205D3224A4FF0FF31D16141
:10194000202222702278D2B103F120018D4205D8E5
:101950001F2A9FBF1B4AD3612022227020221949CF
:101960001844DEF06FF932682378002115481344DB
:10197000202221703360E4F05FFADEF0E3FE33688A
:101980009D4207D90F4920220F48CB61DEF05AF95A
:10199000DEF0D8FE0020DEF0DDF9B8E701221A7093
:1019A000BAE700BF652C002404A21008942C002480
:1019B000002200248C2C0024642C0024805A14085B
:1019C00000002008662C0024E0FF1F082DE9F843E2
:1019D00007460E460024DFF83890DFF83880B4421E
:1019E00001D1BDE8F88324B1230702D14846FFF7AF
:1019F00007FF3D5D01342B0905F00F0518F80300C2
:101A0000FFF7E8FE18F80500FFF7E4FEE7E700BF80
:101A10008479110814A21008474B1B782DE9F74F61
:101A200007460E4690465BB1022925D0042938D0DE
:101A3000012902D11146FFF7C9FF4048FFF7E0FE38
:101A40003F4B1B78002B4ED03E4A00253E4BA2EB6D
:101A5000030938E037F81430ADF8043024B16207D8
:101A600002D12846FFF7CCFE0134022101A8FFF77E
:101A7000ADFFA045EED1E0E70024304DF9E757F87F
:101A80002430019324B1A30702D12846FFF7B8FE02
:101A9000042101340DEB0100FFF798FFA045EED1C2
:101AA000CBE70024254DF9E7FFF71AFD022E1DD0E4
:101AB000042E2CD0012E06D12378795D5A1C227079
:101AC000224AD1540135A8450DD0214B214C1B6829
:101AD0002278043313444B45E6D31C4B4FF0FF32BE
:101AE000DA612023237003B0BDE8F08F2378DFF89C
:101AF0005CA05A1C22703A780AF80320FFF7F0FC29
:101B000023785A1C227000220AF80320DAE74FF0EB
:101B1000000ADFF838B022783B78511C23FA0AF328
:101B20000AF1080A21700BF80230FFF7D9FCBAF16C
:101B3000200FF0D1C6E700BF652C0024847911087E
:101B40000022002400002008805A1408662C00247B
:101B50008C2C0024642C0024036800221B68184786
:101B60000120704737B501912021044681F0EAF940
:101B7000E0B10F4B93F9121AB1B1B3F9141A03F58E
:101B80008053019AD3F8B433B3F90C5001F10A032E
:101B90009D4203DD40F28D33994205DC2046054B22
:101BA000202181F0D5F9002003B030BD0120FBE7F2
:101BB000A06C002428A2100808B506F061F80121E5
:101BC000BDE8084005F0D0B82DE9F04300278FB0FC
:101BD0000E46054606F054F880462E22394602A8E5
:101BE0000197E4F029F9322301AA3946404605F06D
:101BF00089FA044648B901AB174A3146284681F0B4
:101C000003FC20460FB0BDE8F083DFF85890D9F808
:101C1000E00003689B6898470028F2D0A9F5C0400F
:101C200003F078FE814630B90C4A314628464C46CE
:101C300081F0EAFBE5E76946404605F087F80028B1
:101C4000DFD09DF801305B06DBD5054A31462846DA
:101C50003C4681F0D9FBD4E73CA2100845A210080D
:101C60005CA21008A08C002408B5064B93F8293616
:101C70009B0704D5044A81F0C7FB002008BD012062
:101C8000FCE700BFA07C00246CA2100870B50C4CCF
:101C900005460E46D4F8E0000368DB68984710B1AB
:101CA0000124204670BDA4F5C04003F051FE044657
:101CB0000028F5D1034A3146284681F0A5FBF0E71C
:101CC000A08C00247CA21008284B2DE97043D3F887
:101CD0002C36814688461D7B5DB9254B1B68986A6A
:101CE00003685B6B984738B9224A4146484681F001
:101CF0008BFB2846BDE8708360F062FD202161F017
:101D0000F7FF38B160F05CFD1F2161F0F1FF08B111
:101D1000194AEAE7484681F00DF938B9D9F8003098
:101D2000414648469B6BBDE87043184741464846CC
:101D3000FFF718FF06464146484682F0E9F906409B
:101D400020214846F5B281F0FDF841464846FFF7AC
:101D50008BFF054041464846FFF798FF0540414646
:101D6000484682F05DFC0540C3E700BFA07C00242C
:101D7000888E002490A21008A7A2100808B5FFF7CB
:101D8000A3FF054A92F8181660F3410182F818166D
:101D9000024A907108BD00BFA07C00242590002459
:101DA0002DE9F04106460F4681F024F8044678B349
:101DB0000221304681F0C6F850B305F061FF4FF4C0
:101DC0008071804604F0D0FF054608BB4FF40071D7
:101DD000404604F0C9FFD8B10F4885F0E1FF0F4B32
:101DE00003F6FC33D3ED007AF8EEE77A30EE670ABB
:101DF000DFED0B7AB0EEC00AB4EEE70AF1EE10FAAE
:101E000006DD2C46074B3A460221304681F0A0F809
:101E10002046BDE8F08100BF94890024A07C002406
:101E20000000C842C4A21008F8B504460F4681F06D
:101E3000ADFC10210546204681F084F858B12046BB
:101E4000FFF7BAFE064630B93546044B3A46102134
:101E5000204681F07DF82846F8BD00BFD8A21008C2
:101E600070B505460E4681F059FA044678B18021D6
:101E7000284681F067F850B1094B93F8F93B43B11C
:101E80000024084B32468021284681F061F8204624
:101E900070BD31462846BDE8704081F059BE00BF94
:101EA000A07C0024ECA210082DE9F04180460E46EB
:101EB0001B4FFFF789FE044610B90024FC710AE0AD
:101EC000184D05F5C043D3F8E00003689B689847B8
:101ED00020B90123FB712046BDE8F081082140466E
:101EE00081F030F80028F4D095F83436B02202FBA7
:101EF000035305F58045B3F83E24B5F9103A9A42EC
:101F000006DD094B32460821404681F021F8D4E72E
:101F10003146404681F030F90028DAD1CDE700BFE4
:101F200025900024A02C002400A3100881F00EBFEF
:101F300070B505460E46FFF747FE084B044631468E
:101F4000D8712846FFF7A2FE00283146284608BF70
:101F5000002482F0C5FA204070BD00BF2590002407
:101F60002DE9F843414F81463B78002B7BD1404C13
:101F70000126D4F82C563E702D7B1DB13B702846AF
:101F8000BDE8F88382F036FC054630B9394A38702E
:101F9000137843F001031370F1E7DFF8F48052F097
:101FA00063FB314651F020FB88F804600B26013EAC
:101FB00049F04EF848F06AFF16F0FF06F7D12E49B7
:101FC000484682F0DFFA05F05BFED0F80C22C4F838
:101FD0003C2690F89432DA0733D405F001F952F038
:101FE00043FB3C2152F0D0F804F2246300221A6033
:101FF000224B01211B68D86A03681B689847D4F8F4
:102000002C26137B1BB90123137388F8043052F07C
:102010002BFB94F81D2694F81C1651F0D9FC4EF0B9
:10202000E5FD4EF015F900233B7087F021FF144BBE
:10203000C3F8D40094F8193643F0200384F8193615
:102040009DE79B07D4D431460E4802F0F9FA0E48BA
:1020500085F0A6FEDFED0D7A04F2246320EE270A58
:1020600083ED000AC4E7002589E700BF9D2C00240A
:10207000A07C00244490002410A31008888E002423
:10208000A08C0024A02C0024948900240AD7233C8F
:10209000259000242DE9F043364D87B006460C46C6
:1020A000D5F82C361B7B002B61D000294BD0214664
:1020B000304682F065FC0446002853D02E49304655
:1020C00082F060FA05F0DCFD07460BF00FF8804661
:1020D000384604F081FAD8B198F92830022B17D18C
:1020E00000264FF00009F1B203AA3846CDF80C9053
:1020F0000191CDF81090CDF8149004F09FFE019955
:1021000018B103AA40460AF0FDFC0136032EEAD1BD
:10211000D5F82C26137B1BB100231373174A1371B8
:1021200052F0A2FA002151F05FFA154B00211B6812
:10213000D86A03681B68984795F819366FF34513FA
:1021400085F819360FE005F580530192D3F8E000C9
:102150000368DB689847019A0028A8D195F81836DB
:10216000DB06A4D40024204607B0BDE8F083012498
:10217000F9E700BFA07C002420A3100825900024CC
:10218000888E002400F5A04008B590F81836C3F3F7
:1021900080028A420BD061F3820380F8183631B195
:1021A00052F062FA0F21BDE8084051F0EDBF08BDC2
:1021B00000F5A04210B592F829360C4603F0010153
:1021C000A14209D064F3000382F82936DB0704D466
:1021D00002F088FC024B9C7210BD02F035FDF9E75D
:1021E0002590002400F5A04090F8293661F34103C2
:1021F00080F82936014B1973704700BF25900024E1
:102200000020704700207047002070470020704772
:102210000020704700207047002070470020704762
:102220000020704700207047002070470020704752
:102230007047000070470000002070470020704782
:102240000020704700207047002070470020704732
:102250000020704700207047002070477047000042
:102260000020704700207047002070470020704712
:102270000020704700207047002070470020704702
:1022800000207047002070470020704700207047F2
:102290000020704700207047704700007047000022
:1022A00000F5944020307047004870472CD4100847
:1022B00000F5A04090F81C06704700000348086035
:1022C0001C21117008221A60704700BFF8A6100880
:1022D0004EF0D8BB1FF000B951F008BB5FF04CBE08
:1022E0005DF0F4BA02F01EBC02F050BB02F076BA08
:1022F00048F0CCBD66F0A6BC60F014B914F0F2B89A
:1023000002F08AB902F056BE02F008BB02F0A6BD88
:1023100003F024B91FF07CBE03F030BB02F036BCE2
:1023200002F0F0BC694B70B5044640F8043B64F021
:10233000AFFE002504F1100004F5934609F02EFAD3
:1023400004F1B00082F08AFB04F51C704EF028F90D
:1023500004F54A7012F06AFA04F5EE6007F0FEFD2B
:1023600004F618100AF01CF804F546601EF006FE8C
:1023700004F5BF502836103064F000FE04F5C65056
:102380004DF0F0FC04F5DF50083051F06DF804F525
:10239000E7501C306EF064FB04F5E850183063F031
:1023A000CFF804F5EA50143078F01AF904F50F501C
:1023B00024307FF071FB04F510504EF0ABFC04F5B7
:1023C0001450143066F050F804F5005304F515501D
:1023D0003F4A83F8585504F51553283018331360D5
:1023E00048F03AFB04F516502946383003F0C8FD92
:1023F00004F532506AF048FA04F53250303075F086
:10240000E1FA04F55C503C3076F08EF804F5735038
:102410007CF09CFB04F5775018307EF097FC04F5B7
:1024200078503C307FF0CCF804F57A50143073F0DB
:1024300095FE04F57C503C3007F0C4FB04F5814068
:10244000203076F0CDF904F58240203080F0C0FCD9
:1024500004F588401F4974304CF022FB04F5894094
:102460000C306EF045FF04F58B40203080F084FB8B
:1024700004F58B40783087F007FD04F58F402C3051
:1024800062F080FB04F5804383F8145804F590450E
:10249000283528460C3554F06FFBAE42F9D104F5CF
:1024A00093400D4D343080F0E7FB04F593405830F5
:1024B00054F0CCF92B6813B1084887F0A9FC2046EA
:1024C00007494CF0EDFA20462C6070BD4888110891
:1024D000FC9C0024A81613082891002478A3100857
:1024E000F086110810B503F013F960F069F903687C
:1024F000BDE810405B681847FFF7F4BF38B500F53A
:10250000AC4504464035284609F012F80AF0EEFDC5
:1025100090F92530D3B190F84433BBB1284600215F
:1025200008F06AFDDFED0A7A04F6743304F6181039
:1025300020EE270ADFED077A93ED287AA7EE270A27
:1025400083ED280ABDE838400AF0DEBC38BD00BF84
:10255000CDCCCC3D6666663FFFF7D0BF10B50121FC
:10256000044603F02FFA10B1204601F0EBF94FF4C6
:102570008051204603F026FA20B12046BDE81040E5
:1025800001F0A2B910BD0000FFF7E8BF38B5022185
:10259000044603F017FA38B10121204603F012FA7D
:1025A00010B9204601F0CEF90221204603F00AFAC4
:1025B00058B3204601F0D4F94021204603F002FA36
:1025C00068B104F5DF550835284650F015FA04F5D2
:1025D000805393F9183D13B1284650F0D9FB4FF4BE
:1025E0008061204603F0EEF920B104F5DF50083099
:1025F00050F0A4FA8021204603F0E4F960B120F005
:1026000065FEBDE838401EF0E1BA0121204603F026
:10261000D9F90028CDD1CFE74FF48021204603F02F
:10262000D1F90028EBD14FF40021204603F0CAF97C
:102630000028E4D138BD0000FFF7A8BF10B5012184
:10264000044603F0BFF910B1204601F089F980215A
:10265000204603F0B7F928B120F038FEBDE810405D
:102660001EF090BA10BD0000FFF7E8BF38B5044671
:102670004FF6FF7103F0A6F904F5A04528B1D5F88F
:1026800018260721204601F073F962F019F961F06C
:10269000EDFD95F81836074A83F01003C3F30013D5
:1026A00053714EF0A3FA4DF0F5FE0348BDE83840F3
:1026B00072F0CEBF25900024808C0024FFF7D6BF97
:1026C0002DE9F04F00F516540546012138342DED63
:1026D000028B2046A1B005F045FA05F5B841204629
:1026E0001C3105F0ADF805F5B8412046343104F051
:1026F00099F804F54B7005F5245105F5A04408310F
:1027000004F5446B04F61C4604F5426826F09EFA74
:1027100005F5B8408BED000A1EA932684830D8F89C
:10272000003004F628471E9204F62C491F9354F0FB
:10273000C9FE05F5B84105F5B940B0EE608A04F56B
:10274000436AF0EE408A24310C3054F04FFD05F519
:10275000B84105F5B940C7ED008A403189ED008ADE
:1027600040308AED000A54F041FD04F6444383ED05
:10277000000A1B9351F078FF054687F081FB2F4A32
:102780001B9B92ED007A04F63C42B7EEC77A8DEDC2
:10279000187B92ED007A04F63842B7EEC77A8DEDD9
:1027A000167B92ED007A04F6344204F62444B7EE28
:1027B000C77A8DED147B92ED007A214AB7EEC77A85
:1027C0008DED127B93ED007A1E4BB7EEC77A8DED3F
:1027D000107B9BED007AB7EEC77A8DED0E7B9AEDFC
:1027E000007AB7EEC77A8DED0C7B94ED007AB7EEE8
:1027F000C77A8DED0A7B99ED007AB7EEC77A8DED39
:10280000087B98ED007AB7EEC77A8DED067B97EDE1
:10281000007AB7EEC77A8DED047B96ED007AB7EEBD
:10282000C77ACDE90001084928468DED027B51F0B9
:102830003BFB21B0BDEC028BBDE8F08F705400244F
:102840009AA310088CA31008C7A31008FFF738BF7D
:1028500010B5044602F0E6FF1021204603F0B2F85E
:1028600050B120F033FD1EF089FA04F5EA50BDE8BE
:102870001040143077F0E8B810BD0000FFF7E8BF53
:1028800000F51650D1ED017A91ED006AD0EDA85A0D
:10289000D0EDAB6A26EEE77A67EEA57AA6EE257A4A
:1028A000E6EE267A81ED007AC1ED017A70470000EC
:1028B00000F51650D1ED017A91ED006AD0EDA85ADD
:1028C000D0EDAB6A27EEA67A67EEA57AA6EE257A5A
:1028D000E6EE667A81ED007AC1ED017A704700007C
:1028E0002DE9F04104464FF001082DED028B86B032
:1028F00004F5A045FFF716FDC14B04F5944004F51F
:10290000A746236004AF5430483601F053FD04F568
:10291000944330461833C5F8BC33062385F8C033DA
:1029200080F074FAB74B301D04F5A8463946C5F857
:10293000C83344368DF810804DF0CEF8B24B06F116
:102940000C00C5F8443486F057FB1E234FF4E160B9
:1029500085F8A885C5F8B0350023A5F8B43509F089
:10296000DDFCC5F8AC0504F5AB40383086F044FB1F
:1029700004F5AB407C3086F03FFBA44B1A6802B9EB
:102980001E60A34930464CF08BF8A24B04F5AC40D6
:10299000F7EE008AC5F8443401231E309FED9E8A6D
:1029A000A5F81C36142682F03FF89C4B04F5AC4089
:1029B0004FF4007105939A4B40300494009397E8CC
:1029C0000C0008F055F903A904F5B840CDED038AD1
:1029D00054F058F904F5B8400C3009F03BF805F60E
:1029E0001C43B0EE083A9FED8F2A83ED008A04F570
:1029F000BA4083ED018AF0EE420A83ED028A05F6C1
:102A00002843F0EE432A103083ED008AB0EE430AEB
:102A100083ED018AF0EE481A83ED028A05F634430D
:102A2000B0EE481A83ED008A83ED018A83ED028AB5
:102A300005F66C4383ED008A83ED018A05F6744345
:102A400083ED008A83ED018A05F67C4383ED008ADD
:102A500083ED018A05F6844383ED008A83ED018AC4
:102A600005F6F44383ED008A83ED018A83ED028A43
:102A700004F5BA4383ED008A83ED018A83ED028A6F
:102A800004F516533833C5F80C3D73F019F8B0EE61
:102A9000083A04F5BB40B0EE682AF0EE481A624DE1
:102AA000F0EE432A4430B0EE481AF7EE080AB1EED1
:102AB0000C0A73F0B3F9B0EE083A04F5BC40F0EE3E
:102AC000481AB0EE481A9FED572AF0EE432ADFED80
:102AD000570AB0EE430A3C3073F0A0F9B0EE083A62
:102AE00004F5BD40F0EE481AB0EE481A9FED502AAA
:102AF000F0EE432ADFED4F0AB0EE680A343072F090
:102B0000DFFFB0EE083A04F5BE40B0EE482AF0EE22
:102B1000481A9FED490AF0EE432A6830B0EE481A91
:102B2000F0EE480A73F07AF9F0EE083A04F5BF4087
:102B3000B0EE485AF0EE684A9FED400AB0EE484ABF
:102B40006030B0EE633AF0EE632AB0EE002AF0EEA9
:102B5000481AB0EE481AF6EE000A72F029FD384B1A
:102B600004F5C1421D6000235C3298B2013306FBBC
:102B70000051097C0029F8D1324B1880324B188063
:102B8000324B196811B1324887F042F904F5C1405F
:102B900004F5C0451A606430C5F8E00002F0C2F9DF
:102BA0002C4B04F5C240C5F8E430143002F0BAF9F9
:102BB000294B04F5C240C5F81431443002F0B2F993
:102BC000264B04F5C240C5F84431743002F0AAF92E
:102BD000234B04F5C34085ED698AC5F8743185ED52
:102BE0006A8A343085ED6B8A02F09CF91D4B2046D1
:102BF000C5F8B43106B0BDEC028BBDE8F08100BF72
:102C000034A910083CA3100800AE1108A4950024B4
:102C100078A911085CAA100800000000212302080E
:102C200028A91008CDCC4C3E38E71008CDCCCC3EBE
:102C3000CDCCCC3DCDCC4C3D3333333F9A99993FED
:102C4000EC900024E8900024B890002484900024A4
:102C5000CCA3100884F01008CCEF100838F110084D
:102C600024F01008D4F0100838B5054B0A46014688
:102C70001C68236820461D68024BA847002038BD09
:102C8000888E0024A02C002438B5037904463BB973
:102C900005682DB128461DF007F9284609F040FBCC
:102CA000204638BD384B70B50360044600F58840B7
:102CB000143008F0B1FE04F5405393F8302E42B9B9
:102CC000D3F82C5E2DB128461DF0EEF8284609F009
:102CD00027FB04F50F5004F5C35504F5C056243006
:102CE00014357EF0EDFE04F5FB5014360830FFF786
:102CF000CBFF04F5FB50FFF7C7FF04F5FA5018307F
:102D0000FFF7C2FF04F5E850183062F031FCB5421D
:102D100004D0183D28461CF0B9FCF8E704F594559A
:102D200004F59256194B0C350436C4F8603CB54294
:102D300004D0083D2846FFF7A7FFF8E704F6B4756E
:102D400004F6A846B5420ED0A5F5827505F17800C7
:102D500054F0BEFE05F14C0054F0BAFE05F120001F
:102D600054F0B6FEEEE70A4BC4F8FC3094F80C328F
:102D700043B9D4F808522DB128461DF095F82846DD
:102D800009F0CEFA204670BD48881108505211084B
:102D9000F8431308094B0A4A10B5036000F5A04335
:102DA0000446D3F8AC05C3F8442408B109F0BCFAD2
:102DB0002046FFF777FF204610BD00BF34A910085A
:102DC00000AE110810B586F055FC064C064B186095
:102DD0002046FFF785FD2046044A0549BDE810401E
:102DE000DFF0A6B9A02C0024888E002428420124FC
:102DF000952D020810B50446018002494BF050FEA3
:102E0000204610BD24AA100800234FF07C524FF03A
:102E10007E5110B5264C0365C0F88030C0F8903064
:102E2000C0F8A030C0F8C0304365C0F88430C0F8A6
:102E30009430C0F8A430C0F8C43083668367C0F80B
:102E40009830C0F8A830C0F8B830C366C367C0F87F
:102E50009C30C0F8AC30C0F8BC304FF03F43026744
:102E6000C0F8B0204267C0F8B420C0F88820C0F88D
:102E7000C820C0F88C20016644668465C1654FF4A3
:102E80007A71C0F8CC30212061F062F94FF47A7188
:102E9000222061F05DF94FF47A71232061F058F936
:102EA0004FF47A712420BDE8104061F051B900BFA1
:102EB000000080BF70B52DED068B037B82B0044609
:102EC0009FED8A8A3BB980ED358A80ED368A80EDA8
:102ED000388A80ED378AD4ED371A04F1100594ED65
:102EE000381AB7EE009AD4ED360A212694ED350A49
:102EF0007F4800F07DFCB7EE001AFFEE000A582074
:102F000094ED350A21F0A4FEB7EE001AFFEE000A98
:102F1000592084ED350A94ED360A21F099FEB7EE7A
:102F2000001AFFEE000A5A2084ED360A94ED380AA2
:102F300021F08EFEB7EE001AFFEE000A5B2084ED52
:102F4000380A94ED370A21F083FE84ED370A86F0C3
:102F500085FF07EE900A9FED677A2946F8EE677ABB
:102F6000DFED659A67EE877AC4ED027AD4ED353AE3
:102F700094ED384AD4ED367A95ED105AD5ED145AC1
:102F800095ED186A23EE855A67EEA55AD4ED374AB7
:102F900024EE066AD5ED1C6A88FE055AB5EEC05AC5
:102FA000C8FE255A64EEA66AB0EEC66A35EE257AEA
:102FB000F0EEE66AF1EE10FA37EE067AF5EEC05A58
:102FC000CCBF0123002337EE267AF1EE10FAB5EEDE
:102FD000C06AA5EC017A95ED233A85ED079A67EE74
:102FE000837A95ED1F3AE3EE837AD5ED273AE4EE46
:102FF000237A95ED2B4AE4EE847AC5ED037A84F8C2
:10300000D030C2BF94F8D030013384F8D030F1EE24
:1030100010FAF5EEC06AC2BF94F8D030013384F8DC
:10302000D030F1EE10FAC2BF94F8D030013384F8FA
:10303000D03094F9D030002BC1BF06EE903AF8EEB4
:10304000E66A87EEA66A85ED036AD5ED038AF0EE9F
:10305000E87A37EE277AB4EEC97AF1EE10FAC4BFF7
:1030600039EE677A05ED017A94F9E83015ED01AA99
:1030700073B1B4EEE9AAF1EE10FA09D89FED1F7A08
:10308000F4EEC77AF1EE10FAA4BF4FF08043EB6183
:1030900094ED390AD5ED077A019120EE270AD4ED97
:1030A000027A20EE270ADFED167A30EE000A20EED3
:1030B000270ADFF043F8EAEE008A30B201369FEDCE
:1030C000110AB6B228EE800AC5ED0B8A61F01CF831
:1030D000252E01997FF44AAF04F12002044802B082
:1030E000BDEC068BBDE8704000F0B4BB00000000F2
:1030F000A02C0024BD3786359A99193FCDCCCC3E03
:10310000DB0F494000007A440022C0F8D420C0F808
:10311000D820C0F8E020C0F8DC20FFF7CBBE0000CC
:1031200000207047002070470120704790F8303031
:103130008B4286BF00EB8100406B0020704700008F
:1031400090F830308B4286BF00EB8100406B00204E
:1031500070470000FA207047D0E9093242F4E0528B
:1031600043F4F8438262C26A436242F4E052C262AC
:1031700070470000014802F03FBC00BFA02C0024B3
:1031800013B54FF45E70019109F0C2F8044620B106
:1031900001995DF099FE024B2360204602B010BDFC
:1031A000A4AA100870470000704700000020704774
:1031B00070470000002070470020704700207047D3
:1031C00000207047002070477047000070470000E3
:1031D0000320704708207047064BD3F82C363BB1CC
:1031E0001B7B002B0CBF5020D02040F0010070470B
:1031F0005020FAE7A07C00247047000070470000D0
:10320000114BD3F82C06F0B1D0ED387A90ED367A28
:10321000F0EEE77AD0ED376AB0EEC77AF0EEE66A04
:10322000C7FE877A90ED357AB0EEC77A87FE267AA8
:10323000C7FE877A9FED057A67EE877AFDEEE77A1B
:1032400017EE903A18B27047A07C00240000C842E4
:1032500057F0D0BA10B5044658F0E8FE054802F021
:10326000CBFB054A034606212046BDE8104058F036
:10327000C5BE00BFA02C002490AA100857F0B8BD0E
:10328000084608B508F008FD00280CBF04200020FF
:1032900008BD0000162A01D057F0E2BA032201202F
:1032A0000A7070475DF008BB08B557F03BFD40F46D
:1032B0001C6040F00D0008BD10B5044609F030F860
:1032C000204610BD08B5094B93F81826D2060BD43A
:1032D00003F58053D3F8E0000368DB6A98470028C1
:1032E0000CBF0220042008BD0120FCE7A07C0024C4
:1032F000044B187820B9044B93F81906C0F38010DA
:10330000704700BFE08E0024A07C002400B500239D
:1033100089B002930393049304F0B2FC02A904F071
:103320006BFAA0B104F0ACFC00F5607005AB07C807
:1033300083E80700184626F02BF8F1EE047A20EE19
:10334000270AFCEEC07ACDED017A9DF8040009B0A1
:103350005DF804FB7FB5002303930493059304F009
:103360008FFC03A904F048FAD8B104F089FCD0ED31
:10337000E00A90EDE10AF1EE600AB1EE400ADFF0FA
:10338000B5FEDFED097A20EE270A21F0BDFBF6EE4F
:10339000007A20EE270AFCEEC07ACDED017A9DF886
:1033A000040007B05DF804FBE02E65421FB5002362
:1033B00001930293039304F063FC01A904F01CFA47
:1033C00028B101A825F0E4FF05B05DF804FB13F077
:1033D000C7F8B02290F80C3302FB030090ED410ACD
:1033E000F2E700000B4B93F8F92B7AB993F82926F2
:1033F00051070BD193F81826D20609D493F8193641
:1034000013F0020F14BF04200120704705207047FD
:1034100003207047A07C00242DE9F04F394D8FB078
:10342000044695F81C26012A5BD9A5F5805705F5B9
:103430005568354E4FF0080905F5845516F901BB5E
:10344000B7F92C3A0BF1FF3A43FA0AF3D90743D5FF
:1034500094F8280055F0BCFB039094F8280056F02F
:10346000AFFB039A00F121039A4206D294F8280098
:103470000FB0BDE8F04F57F06DB8BAF1070F2BD879
:10348000DFE80AF03E04323436383A3C1F4B5A69C2
:10349000D8681969D3F804E0D3F818C0D3F800A0AD
:1034A0000A925A6A1B6ACDF82D206222CDF831307B
:1034B000212308900991C22194F82800CDF814A086
:1034C000CDF818E0CDF81CC08DF82CB0CDE9003255
:1034D000192305AA55F0FAFB09F1FF3313F0FF0990
:1034E000ACD10FB0BDE8F08F094BD0E7094BCEE768
:1034F000094BCCE7094BCAE7094BC8E72B46C6E79F
:103500004346C4E7A07C002484AB10081C8A002436
:10351000948A00240C8B0024948B0024C08B0024FC
:10352000388C0024094BD3F8582A920701D457F05D
:103530008BB903F58053DFED067A03F5416393ED14
:10354000000AB8EEC00A20EE270A7047A06C0024DB
:103550000AD7233C10B594B0044603A808F07AFAC1
:103560001A4B03A9D3F8E00003685B6B984758B384
:1035700094F8284086F07CFC059B9622DDED047AC9
:1035800057210893069BF8EEE77A9FED117A09938D
:10359000002367EE877A07900B9320460C930D93D8
:1035A0000E930F931093119312934FF6F853CDEDA2
:1035B0000A7AADF84C3000238DF84E303323CDE934
:1035C000003207AA55F082FB14B010BDA08C002475
:1035D0000AD7233CF0B5254D95B00E46074603ACFF
:1035E0000FCD0FC42B682360731EDBB2042B2AD8C7
:1035F00014AA02EB830353F8445C2B6828461B6A29
:1036000098472B68044628469B6A98470023052262
:1036100097F82850089009938DF828208DF8296094
:103620008DF82A3094B9232221460DF12B00E2F0C7
:1036300003FC86222E2340F2B3112846CDE9003246
:1036400008AA55F043FB052015B0F0BD20460DF14A
:103650002B0304F1200250F8041B904243F8041B92
:10366000F9D102881A8082789A70E2E7A89F100840
:10367000014802F0BFB900BFA02C0024014B93F811
:103680001C067047A07C0024024B93F81906C0F377
:1036900040007047A07C0024164B30B505460C4610
:1036A0002DED028BD3F8E00085B091ED018A03681F
:1036B000DB69984728B9BDEEC88A18EE103ADB07D7
:1036C00012D5D4E9040121F0A7FD68B1684608F0DD
:1036D000C1F96A46214628465CF0F0F920B1064956
:1036E000684608F0E5FA00B1022005B0BDEC028B97
:1036F00030BD00BFA08C0024AC8800248B8B162B1F
:1037000005D0C02B01D1FFF7C7BF5EF0C3B80020C2
:103710007047000030B5002305462DED028B8DB0BB
:1037200003930493059304F0ABFA03A904F064F83F
:1037300060B304F0A5FA00F5607306AC95F8285064
:1037400093E8070084E80700DDED060A9DED070A0F
:10375000F1EE600AB1EE400ADFF0C8FC2046B0EEA0
:10376000408A25F015FE089B0122DFED0A7AA82188
:103770000B930C2328EE278A28468DED0A0ACDE903
:10378000003209AA8DED098A55F0A0FA0DB0BDEC02
:10379000028B30BDE02E6542242938B5054605D0A0
:1037A00040290DD0BDE838405CF002BD0C2156F038
:1037B000E3FE044610B12846FFF7ACFF204638BDB3
:1037C0000124FBE7F6EE007A08B591ED007AB4EE3D
:1037D000E77AF1EE10FA06DD012205210348FEF733
:1037E00059FC002008BD0420FCE700BF68800024CD
:1037F0002DE9F04188B080461B22002101A810EE7F
:10380000107A10EE906A11EE105A11EE904AE2F022
:1038100013FBA3238DF8043095238DF805300B237B
:103820008DF8063086F02CFBCDF8070008F5DF5048
:10383000CDF80B101B2201A90830CDF80F70CDF880
:103840001360CDF81750CDF81B404FF0E9FE08B0DB
:10385000BDE8F08170B58CB00D46144606462B22AB
:10386000002101A8E2F0E8FAA3238DF804309523A3
:103870008DF805300C238DF8063086F001FB2B689F
:103880002B22CDF8070006F5DF50CDF80F30236866
:103890000830CDF80B1001A9CDF813306B68CDF8C6
:1038A00017306368CDF81B30AB68CDF81F30A368C4
:1038B000CDF82330EB68CDF82730E368CDF82B3016
:1038C0004FF0AEFE0CB070BD70B500F5DF5400F5E2
:1038D000BA4605460E21083406F1500220464FF044
:1038E00053FD06F17C0220460F214FF04DFD05F5FA
:1038F000BB4220461021743205F5BD464FF044FD11
:1039000005F5BC42204611216C324FF03DFD06F119
:10391000740220466C214FF037FD06F1A0022046CC
:103920006D214FF031FD05F5BF4220460D211832C3
:103930004FF02AFD05F5C14220466921BDE87040DF
:103940004FF022BD1FB500F51650002301A93830F5
:1039500001930293039302F011FA05B05DF804FBA2
:1039600008B504F08DF9BDE8084003F017BE00006B
:103970007FB50E464FF6FF710446154602F022F859
:10398000E8B1102200216846E2F056FAA3238DF830
:10399000003095238DF8013004238DF8023086F035
:1039A0006FFACDF8030004F5DF50CDF807101022B0
:1039B000694608308DF80B6003954FF0B1FE04B0F6
:1039C00070BD0000B220704738B500F5DF550446E1
:1039D00002F012F80C490835024628464FF0BCFFA9
:1039E00004F5A043284693F81D2693F81C164FF0C3
:1039F000EFFF04F51650383004F0FAFA04F54A7077
:103A0000BDE8384011F0C6BC90AA100837B5069D35
:103A1000044600B92C7801B9697802B9AA7803B9CB
:103A2000EB78002064F3070061F30F2062F3174086
:103A300063F31F6003B030BD2DE9F04FDC4CF7EEAF
:103A4000006ADFEDDC5A924605460E46DFF89483A5
:103A50002DED0C8B9DB00D93D4EDB99A04F5A044D7
:103A600090ED006AD4F82C36D3ED367A93ED387A9F
:103A7000F0EEE77AB0EEC77A77EE877AF4EEE67A80
:103A8000F1EE10FAC8BF86EEA78ADFEDCB7AD8BF79
:103A9000B0EE668A28EE277AA6EE257A80ED007AC7
:103AA000D4F82C3693ED357A93ED376AB0EEC77AB9
:103AB000B0EEC66A37EE067AB4EEE67AF1EE10FAA8
:103AC000C8BFC6EE878A90ED017AD8BFF7EE008AAC
:103AD00068EEA77AE7EE257AC0ED017A50F0C4FDD2
:103AE000074686F0CDF9B7EEE87AB7EEC88AB34B51
:103AF000B34A8DED087B95ED017AB7EEC77ACDE933
:103B000000018DED047B95ED007A3846AD49B7EEA6
:103B1000C77AAD4F8DED068B8DED027B50F0C4F969
:103B2000AA49304697ED00AA24F0FEFF8DED160A53
:103B30009AED000ACDED170A30EE4A0A8DED181AFB
:103B400021F05AF89DED167A08F64C23B0EEC77AAC
:103B5000D3ED007AA7F5FA63B4EEE77A0B93F1EEB2
:103B600010FA00F12982D4F82C361B7B002B00F0D0
:103B70002382B8F84A9AC9F340099DED177AB0EE4E
:103B8000C77AF4EEC77AF1EE10FA00F31882D4F88F
:103B90002C361B7B002B00F01282B8F84A3A03F057
:103BA00001039DED187A0A93B0EEC77AF4EEC77A56
:103BB000F1EE10FA00F30582D4F82C361B7B002BB3
:103BC00000F0FF81B8F84A3AC3F38007B0EEC00AAC
:103BD000F4EEC07AF1EE10FA00F3F581D4F82C3649
:103BE0001B7B002B00F0EF81B8F84A3AC3F3C00BFF
:103BF0000DAB3A460A99484600935B46FFF706FF2D
:103C00009FED738AC3B20F900BEE103AC0F30723F7
:103C10000AEE903AC0F307430CEE903A030E0DEE15
:103C2000103A9DF83430002B40F0D0819DF83530AB
:103C3000002B40F0CB81F8EE4B7A644AB0EE690A73
:103C400019AB314602F52070CDED197AF8EE6A7A9B
:103C5000CDED1A7AF8EE6C7ACDED1B7A72F0BCF8E5
:103C6000B0EE409A8DED140AF0EE608ACDED150AA3
:103C70009DF83630574C002B40F0AD8104F63C43A4
:103C8000B0EE691A1CEE901A96ED020AD3ED000A06
:103C900004F6687072F0BEF9B0EE40CA9DF8373095
:103CA000002B40F09B819AED000A30EE4A0A20F08A
:103CB000A3FFF0EE690A1DEE101A474871F0C0FE2E
:103CC000F0EE40BADAF80020444BC3F8802083EDD0
:103CD00021AA08F52363B0EE490A472093ED001AA4
:103CE0000C93F1EE410A20F0B3FF0C9BB0EE40AA1A
:103CF000482093ED001AB0EE680AF1EE410A20F078
:103D0000A7FF08F6342308F63828B0EE409A93ED62
:103D1000001A4920B0EE4C0AF1EE410A20F098FF5B
:103D200098ED001AF0EE408A4A20B0EE6B0AF1EEF0
:103D3000410A20F08DFF95ED007AD5ED017A04F669
:103D400028436AEE076A8DED148AF0EE40BA8DEDD5
:103D5000158ACDED106A69EE276ACDED116AD3EDB3
:103D6000006A04F62C4327EE267AD3ED006A9DF80C
:103D7000343067EEA67A8DED127ACDED137A9BBBC7
:103D80009DF8353083BBB0EE690A19ABB8EE4BBA7B
:103D900012AAF8EE6AAA10A911488DED19BACDED54
:103DA0001AAA71F005FF8DED140ACDED150A1BE07E
:103DB000A02C0024A4707D3F00D7233C50B21008F3
:103DC0002CE4100845E4100870540024D488002422
:103DD00000000000A07C0024808C0024A08C002423
:103DE000B0890024A06C00249DF83630002B40F0F0
:103DF000F88004F5436395ED000AB0EE691A1CEEF5
:103E0000901AD3ED000A8F4860EE200A28EE800A4F
:103E100072F000F9F0EE40AA14A98B48FEF748FDB5
:103E20009DF83730002B40F0DF8004F6444395EDD9
:103E3000010AB0EE691A1DEE101AD3ED000A83488C
:103E400060EE200A20EE2B0A72F0E4F8F0EE409AC1
:103E5000D4F82C361B7B7BBB19A97D488DED198AC4
:103E60008DED1A8A71F0CEFF9FED7A0A7A4872F0D2
:103E7000EDF89FED780A794871F00EFE19A978489F
:103E80008DED198A8DED1A8A71F0BCFF9FED710AD4
:103E90006C4872F0DBF86D489FED6E0A72F0D6F850
:103EA00004F6344393E807000B9B03F5FA6386E8B6
:103EB00007001B68CAF80030B9F1000F00F09780C6
:103EC000D4F82C3683ED368A0A9B002B00F09A80BA
:103ED000D4F82C3683ED358A002F00F09E80D4F87C
:103EE0002C3683ED388ABBF1000F00F0A080D4F8A7
:103EF0002C3683ED378A04F628439FED5A8A9FEDCE
:103F0000554AD3ED002A04F63443D6ED000AF0EE0C
:103F1000443A93ED001AB0EE443A62EE882A2AEE53
:103F2000082AF0EE441A21EE081A60EE880AB0EE74
:103F3000440A83F0F1FF04F62C439FED464A29EE34
:103F4000082AD3ED002A04F63843D6ED010AF0EE34
:103F5000443A93ED001AB0EE443A62EE882AF0EE4D
:103F6000441A21EE081A60EE880AB0EE440A83F083
:103F7000D7FF04F5436304F63C449FED364AD3ED86
:103F8000002A28EEC82A94ED001AF0EE443AD6ED45
:103F9000020AB0EE443A62EEC82AF0EE441A21EE6C
:103FA000481A60EEC80AB0EE440A83F0BDFF1DB0A7
:103FB000BDEC0C8BBDE8F08F4FF00109DDE501236E
:103FC000EFE5012702E64FF0010B11E6F0EE488A1B
:103FD000B0EE489A4CE69FED1FCA5FE6DFED1DBAD2
:103FE00077E6DFED1CAA17E7DFED1A9A30E79DF8B8
:103FF0003430002B7FF468AFD4F82C36149AC3F811
:10400000D82061E79DF83530002B7FF465AFD4F8F8
:104010002C36159AC3F8D4205EE79DF83630002B75
:104020007FF461AFD4F82C36C3ED38AA5BE79DF876
:104030003730002B7FF45FAFD4F82C36C3ED379ABE
:1040400059E700BF648A0024A02C0024DC8A0024E5
:10405000548B002400000000088C0024808C002475
:10406000B08900240000C8422DE9F04F2DED068BE9
:1040700091B0064688460593C74B039203F5A044CA
:10408000D3EDB9AAD4F82C26127B002A00F0508177
:1040900003F58043B3F84A5AC5F3400B05F0010A13
:1040A000C5F3800715F0080500D0012505ABDFF842
:1040B00000933A465146009358462B46FFF7A6FC1C
:1040C00099ED001A98ED000AF1EE410A07909A2046
:1040D00020F0BEFD4B46F0EE409A9B20B3EC011A57
:1040E00098ED010AF1EE410A049320F0B1FD049B22
:1040F000B0EE409A9C2093ED001A98ED020A4FF022
:104100000008F1EE410A20F0A3FD039B99ED021A8D
:10411000F0EE408A9D2093ED000AF1EE410A20F076
:1041200097FD96ED007AD6ED017A04F6284369EE04
:10413000876ACDF83080B0EE408ACDF83480CDED7E
:10414000086A69EE276ACDED096AD3ED006A04F6C4
:104150002C4327EE267AD3ED006A9DF8143067EEE3
:10416000A67A8DED0A7ACDED0B7AFBB99DF8153064
:10417000E3B99DF81C30B0EE6A0A0AAA08A907EE56
:10418000103A9DF81D3009F5975007EE903AB8EEB9
:10419000477A0EABF8EE677A8DED0E7ACDED0F7A99
:1041A00071F006FD8DED0C0ACDED0D0A9DF816306F
:1041B000002B40F0C18004F5436396ED000AB0EE99
:1041C0006A1A9DF81E10D3ED000A744860EE200AAA
:1041D00028EE800A71F01EFFB0EE40AA0CA96E48CE
:1041E000FEF766FB9DF81730002B40F0A88004F620
:1041F000444396ED010AB0EE6A1A9DF81F10D3ED04
:10420000000A674860EE200A20EE080A71F002FFFB
:10421000B0EE408AD4F82C361B7B8BB90EA96148CE
:10422000CDF83880CDF83C8071F0ECFD9FED5E0A52
:104230005A4871F00BFF9FED5C0A594871F006FF78
:10424000BBF1000F7ED0D4F82C36C3F8D880BAF179
:10425000000F00F08180D4F82C36C3F8D480002FF2
:1042600000F08580D4F82C36C3F8E080002D00F0F3
:104270008880D4F82C36C3F8DC8004F628439FED00
:104280004B8A9FED494AD3ED002A04F63443F0EE01
:10429000443A93ED001AB0EE443A62EE882A29EED1
:1042A000882AF0EE441A21EE081AF0EE440AB0EE25
:1042B000440A83F031FE04F62C439FED3B4A29EE7D
:1042C000082AD3ED002A04F63843F0EE443A93ED81
:1042D000001AB0EE443A62EE882AF0EE441A21EE5B
:1042E000081AF0EE440AB0EE440A83F019FE04F511
:1042F000436304F63C449FED2C4AD3ED002A28EE9C
:10430000C82A94ED001AF0EE443AB0EE443A62EE58
:10431000C82AF0EE441A21EE481AF0EE440AB0EE34
:10432000440A83F001FE11B0BDEC068BBDE8F08FAE
:104330000127BA46BB46B8E69FED1BAA4EE79FEDA4
:104340001A8A67E79DF81430002B80D1D4F82C36F8
:104350000C9AC3F8D8207AE79DF81530002B7FF42B
:104360007EAFD4F82C360D9AC3F8D42077E79DF8A9
:104370001630002B7FF47AAFD4F82C3683ED38AAB0
:1043800074E79DF81730002B7FF477AFD4F82C3604
:1043900083ED378A71E700BFA02C0024648A0024D3
:1043A000DC8A0024B0890024000000000000C8421C
:1043B000D076002470B5044610305DF0FDFFA025D6
:1043C0000A4B0B4E236160195EF0D0FA665130350E
:1043D000B5F5687FF7D104F5687060F097F820466E
:1043E00004494AF05DFB204670BD00BF9CED1008FB
:1043F00088ED1008A8E6100837B500F594410122B1
:10440000044604314DF0CCFA1E4A1368D9070AD489
:1044100004F581431C4920330B6004F58B4378334A
:10442000CB600123136004F5944002221649012554
:10443000543049F009FF002304F5DF51134AFD20F1
:104440000831CDE9005349F091FE114B012111488B
:104450001A68D2075FBF0F4A04F510541D6014603C
:1044600049F00EFF4AF00EFD0B4A04210B48138859
:1044700043F040031380002203B0BDE8304049F010
:1044800071BE00BF8C8E0024C4250024D48F110877
:10449000908E0024DC250024C4900024ACEB10088E
:1044A0000069C0F3401070470F299DBF302303FB04
:1044B0000100903000207047014B93F91E0A7047AD
:1044C000A06C0024024B93F8290600F0010070470D
:1044D000A07C0024014BD3F8B8037047A07C0024D3
:1044E000002910B517DB104CCBB294F8C0239A42C8
:1044F00011D3D4F8BC330122A4F5A040595C00F0DC
:1045000081FD94F8193638B99A0704D5074A13780B
:1045100043F00403137010BD9B07FCD5034A1378C6
:1045200043F00203F6E700BFA07C0024449000247F
:10453000022A10B50F4C12D13522A4F5A04000F08C
:1045400061FD94F819369B0705D50B4B1A7818B105
:1045500042F002021A7010BD42F00402FAE794F829
:104560001C268A42F7D15EF02BF9BDE810405EF0C0
:1045700015B800BFA07C002444900024064A92F89D
:10458000293692F8282603F00103134301D15DF088
:10459000FFBE0020704700BFA07C0024332901D05B
:1045A0005FF0A0B97047000008B50A68332A07D049
:1045B000382A08D10A790321FFF7BAFF012008BD84
:1045C0000A790121F8E7BDE808405EF003BE00006B
:1045D00030B5044689B004F51655684607F03AFA36
:1045E00004A8383507F036FA6946284603F07AF809
:1045F00078B104A9284603F017F950B104A9684618
:1046000007F056FA236800226946D3F8B8302046EE
:10461000984709B030BD000000F5005292F84C28D0
:10462000D2070BD400F5A042D2F82C26117B09B199
:10463000FFF7CEBF0368D3F8B430184770470000C7
:1046400010B586B0044602A8019107F003FA04F5FC
:10465000165002A9383003F045F830B1236802A99A
:10466000019A2046D3F8B830984706B010BD000034
:10467000F0B5044685B00F46154604F51656684653
:1046800007F0E8F969463836304603F0CDF810B93E
:10469000002005B0F0BD3946304602F055FE002836
:1046A000F6D0002DF5D004F50054284694F84C3887
:1046B00043F0020384F84C38EBE7000010B500F536
:1046C00094448AB00023D4ED0A7A2834F5EEC07AF7
:1046D000F1EE10FA44D9079300F51650089303AA97
:1046E000099306AB04A93830019307AB009305ABDF
:1046F00002F0C8FEDDED087A9DED077A87FE277A85
:10470000DDED097A87FE277AD4ED007AB4EEE77AF8
:104710009DED047A77EEA76AF1EE10FAF4EEC76A1F
:10472000ACBF01200020F1EE10FA0CD802309DED54
:10473000037AF4EEC77AF1EE10FA0CD8003818BFFD
:1047400001200AB010BDF4EEC77AF1EE10FA9CBF5A
:104750000130C0B2EBE7012894BF00200120F0E750
:104760000020EEE700F5A04210B592F82936044685
:1047700059071CD443F0040382F829364FF074FF24
:10478000012211214FF020FD094BD3F8E00003680E
:104790009B68984728B904F5804393F9253A032B81
:1047A00005D120460621BDE8104000F029BD10BD0E
:1047B000A08C002400F5A04008B590F829365A07CF
:1047C0000BD56FF3820380F829364FF04DFF00229E
:1047D0001121BDE808404FF0F7BC08BD2DE9F043BA
:1047E000054685B005F51658684607F033F9694661
:1047F00008F13808404603F017F8D8B105F5A04392
:10480000434C444FD3F82C361B7B43B105F59443FE
:10481000D3ED0A7AF5EEC07AF1EE10FA0DD82388BE
:10482000284623F4FF7323F0010323800023FB7346
:10483000FFF7C0FF05B0BDE8F083284601F080F81F
:10484000064618B9284601F03FF806462846FFF705
:1048500035FF814640B93EB12378002B41D16378C2
:1048600003F00103FB73E5E76378DB07F7D42378F4
:104870000133DBB2082B237006D12846FFF71EFF59
:1048800010B1404602F07EFE2378092B02D140464B
:1048900002F070FE2378092BE1D9238823F4FF73FB
:1048A00023F0010343F4857323804FF0DDFE0222E1
:1048B00010214FF089FC85F0DBFA6368C01A47F2DB
:1048C0003053984209D905F5A840134A02214430D3
:1048D00055F0F0FB85F0CCFA60602846FFF742FF08
:1048E000BDE7013B23702388C3F30803B3F5807F42
:1048F000B5D1637860F3000363704FF0B5FE4A46AC
:1049000010214FF061FC2846FFF754FFA7E700BFD6
:10491000948E002425900024B8ED100837B5044685
:1049200000F5165001A904F5A045383002F050FCFE
:10493000D5F83034834206D0C5F830044FF094FEE9
:104940003E214FF021FC04F5005395F9341493F8FF
:10495000E02893F9E038994213D0FF2A11D085F866
:1049600034344FF081FE95F8342418214FF02CFC9C
:1049700004F5A84095F934340421034A443055F035
:1049800099FB03B030BD00BFC8ED10082DE9F0431E
:10499000064695B085F06CFA002403AB06F5165870
:1049A00005460BAA019308F1380802AB08A9404656
:1049B000089400930EAB09940A940B940C940D94F4
:1049C0000E940F94109402F04BFDDFED437A0746EE
:1049D0009DED0A7AB4EEE77AF1EE10FA37DB9DED41
:1049E0000D7AB4EEE77AF1EE10FAACBF4FF00109A0
:1049F0004FF0000907AB1194129404AA019311AB74
:104A0000139406F5A044009305A906AB404602F0B6
:104A100039FD94F9A033002808BF002783B17FB186
:104A2000D4F82C361B7B5BB1B9F1000F08D0F7EE40
:104A3000007A9DED057AB4EEE77AF1EE10FA09D529
:104A400094F8383473B90023C4F83C340FE04FF0C5
:104A50000009CFE7D4F83C0420BBC4F83C54C4F8A8
:104A6000400404E0D4F8400420B9C4F8405415B020
:104A7000BDE8F083281A43F698239842E3D900252D
:104A800084F83854C4F840544FF0EEFD2A461D21F6
:104A90004FF09AFB06F5A840104A0221443055F029
:104AA00009FBD0E72D1AB5F57A7FE0D994F83834B0
:104AB000002BDCD1012584F838544FF0D5FD2A466F
:104AC0001D214FF081FB06F5A840054A0221443024
:104AD00055F0F0FACBE700BF00000034E0ED10081D
:104AE000FBED100810B504464FF0BEFD0022052175
:104AF0004FF06AFB04F5A840034A04214430BDE8A6
:104B0000104055F0D7BA00BF18EE100800F5A040CD
:104B100090F819369B065ABF90F81806C0F300109B
:104B20000120704738B5044603F0AAF84FF48041DD
:104B300002F01AF904F5A042054692F81936C3F3BB
:104B4000001181421CD060F3041304F5A84482F8DC
:104B50001936443460B14FF087FD02220B214FF02B
:104B600033FB084A20460221BDE8384055F0A2BA7E
:104B70004FF07AFD2A460B214FF026FB024AF1E75F
:104B800038BD00BF30EE10083BEE100800F5804342
:104B900070B593F90E3A0446B3B300F5A045D5F8C5
:104BA000A4658EB385F064F995EDEA0ADFED177A16
:104BB000861B9FED171A692020EE270ADFED150AE4
:104BC00020F046F8BCEEC00A10EE103A9E4209D220
:104BD00095F829369A0717D520460021BDE8704080
:104BE000FDF700BB10D995F829369B070CD4204659
:104BF0000121FDF7F7FA04F5A74001221221483000
:104C0000BDE87040FDF746BA70BD00BF00007A44B1
:104C10000000804F000000000B461146012B10B42D
:104C200004D0052B06D05DF8044B70475DF8044BAB
:104C300000F0E6BA00F5A740012214215DF8044B0C
:104C40004830FDF727BA0000F8B504464FF00CFDD8
:104C5000012205214FF0B8FA04F5804304F5A84677
:104C6000204693F9125A4436003D18BF0125FFF73C
:104C70004DFF98B11F4A04213046002555F01AFA1D
:104C800004F5A740012210214830FDF703FA294618
:104C900020460322BDE8F840FFF7BEBF04F5C04739
:104CA000D7F8E0000368DB6A984778B104F5A043C1
:104CB00093F8F92B52B193F9F83B012B06DC0E4A1D
:104CC00004213046012555F0F5F9E0E7D7F8E0007A
:104CD0000368DB6A984728B104F5A043D3F8A433EE
:104CE0001B0705D4054A0421304655F0E3F9CEE709
:104CF000034AE5E750EE10086BEE100899EE100835
:104D0000A8EE100870B5044615464FF0ADFC012220
:104D1000062104F5A8464FF057FA20464436FFF71F
:104D2000F5FE98B104F5A74001220721002548307F
:104D3000FDF7B0F9144A0421304655F0BBF9294675
:104D400020460422BDE87040FFF766BF04F5C0436B
:104D5000EDB2D3F8E0000368DB6A984768B104F568
:104D6000A043D3F8A4331B0707D535B1074A042164
:104D70003046012555F09EF9E1E7054A0421304609
:104D800055F098F9DBE700BFCCEE100873EE100881
:104D9000E9EE1008F8B5044685F060F8284B0546A2
:104DA000B4F8C6221988274E91420ED01A80264B9D
:104DB00018603378A3B1002434704FF055FC2246BC
:104DC0001321BDE8F8404FF0FFB933781F4FC3B946
:104DD0003B782BB11C4B1E4A1B68C31A934200D868
:104DE000F8BD0123337004F5A043D3F82C06037BF0
:104DF0000BB1FEF789F94FF037FC012213214FF078
:104E0000E3F93B78002BEBD03378002BE8D00E4A47
:104E100010491368EB1A8B42E2D904F5A0441560DF
:104E2000D4F82C26137B002BDAD0002313730A4A04
:104E3000D4F82C061371BDE8F840FEF73BB800BF6C
:104E40009E8E00249C8E0024A08E00249D8E002423
:104E500080841E0040420F0025900024F0B50446D7
:104E600000F5B94500F5A04785B0743504F5165630
:104E700097F838142846383682F040FF684606F026
:104E8000E9FD6946304602F02DFC029B20213046A8
:104E9000C7F8143C039BC7F8183C01F065FFD0B17C
:104EA000284604F5B84582F07BFFFDEEC07A0C354C
:104EB00004F50054022217EE901A284617EE906A65
:104EC00006F0CCFD94F84C38DB0706D401223146BD
:104ED000284606F0C3FD05B0F0BD0121284606F0C6
:104EE00097FE0028F2D0F6E70120704700207047B7
:104EF0000020704700207047002070470020704756
:104F000000207047002070479FED010A704700BFE6
:104F1000000000009FED010A704700BF0000000084
:104F200070470000104A0260104A02F150014260CE
:104F3000816001F59551C1600D49016102F628417A
:104F4000416102F62C41816102F6A811C16102F6AD
:104F5000AC11016202F51B6102F6B4124162826279
:104F6000044AC262704700BF74EF1008A4760024A0
:104F700058520024C02F0024042918D8DFE801F07B
:104F800003070B0F130000F5C2401430704700F503
:104F9000C1406430704700F5C2404430704700F5AE
:104FA000C2407430704700F5C34034307047002071
:104FB0007047000000F5C040D0F8E00003685B686F
:104FC0001847000038B500F5C0450446D5F8E000A4
:104FD00003685B6998470A4B04F5A042187492F87D
:104FE0001C26D5F8E000DA7003685B6A9847014632
:104FF00004F51550BDE83840283045F0DDBF00BF4E
:10500000259000242DE9F84F00F5A04A06460F46EA
:1050100091469AF81C368B4205D101258AF81D2647
:105020002846BDE8F88FFFF7A7FF044620B93046B1
:1050300025464CF071FEF3E7DAF82C3606F5A84861
:105040001B7B08F1440883F0010BEBB92368594638
:1050500020461B689847054680B306F5C04306F511
:10506000DF504A463946C3F8E04008308AF81C76DB
:105070008AF81D964EF0ACFC404600215CF0BAFB6D
:105080003046FFF79FFFCBE703689B689847E0B186
:105090001C4800F03FFC0546B8B9236820461B6A4F
:1050A0009847194A03460421404655F003F84FF04B
:1050B000DBFA3A460A214FF087F8B1E72368204629
:1050C0001B6A9847114A0346EDE70E4800F040FC82
:1050D0000028BBD106F5C043D3F8E0000368DB68C5
:1050E00098470028B2D023682046DB6898470546D9
:1050F0000028ABD1236820461B6A9847044A034620
:10510000D1E700BFA02C0024FCEE10084EEF1008E1
:1051100025EF10080148FFF775BF00BFA02C002441
:10512000234B70B593F8293605460C461646DB0727
:1051300005D5002363602360A360336070BD5DF01C
:105140003FFB037F002BF4D0EB699FED1A7A1B68BD
:10515000B3F90A3007EE903AF8EEE77AC7EE876ABD
:10516000C4ED016A2B6A1B68B3F90A3007EE903A66
:10517000F8EEE77AC7EE876AC4ED006A6B6A1B68CF
:10518000B3F90A305B4207EE903AF8EEE77AC7EEE1
:10519000876AC4ED026AAB6A1B68B3F90A3007EE8E
:1051A000903AF8EEE77AC7EE876AC6ED006AC5E77F
:1051B000A07C002400007A44002070470120704742
:1051C0000020704700207047004870475C5E11085F
:1051D00000487047BCEF10080020704743691A6808
:1051E0000023C2F8D43042691268C2F8D83042694C
:1051F0001268C2F8DC3042691268C2F8E0307047C9
:105200000A46002108B5FFF7FDFE034A137843F074
:105210000803137008BD00BF4490002401207047AC
:1052200000207047012070470020704700487047F9
:10523000FCB411080048704714F0100803207047B0
:10524000084B03F5B84203F51F533432103330B521
:10525000044600F1300507CA85E807001B680120F5
:10526000E36330BDA02C002430B52DED028B87B058
:1052700000230446584D01AA03A995EDB98A03936A
:1052800004930593FFF74CFF63689DED037AD3ED1C
:105290000E7A68EE277A27EE277A8DED037A9DED58
:1052A000047A67EE277ACDED047AD3ED0F7A28EEF3
:1052B000277ADDED057A67EE877ACDED057AD3EDB5
:1052C000107A93F9443028EE278ADDED017A27EE33
:1052D000888A8DED018A1BB903A92846FDF7D0FA0B
:1052E0003E4D94ED0C7AD5ED007AA5F63445636811
:1052F00077EE677A05F63842D3ED0E6A94ED0F0A21
:10530000F0EEE77AF4EEE67AF1EE10FA44BFDDED66
:10531000037A77EE877A94ED0D7A48BFC4ED0C7A64
:10532000D2ED007A05F63C42D3ED0E6A77EE677A4D
:10533000F0EEE77AF4EEE67AF1EE10FA44BFDDED36
:10534000047A77EE877A94ED0E7A48BFC4ED0D7A31
:10535000D2ED007AD3ED0F6A77EE677A2369F0EE2B
:10536000E77AF4EEE67AF1EE10FA42BFDDED057A67
:1053700077EE877AC4ED0E7AD3ED867A30EE670A3F
:105380001FF03AFC6368B0EEC00AD3ED107AB4EEB9
:10539000E70AF1EE10FA09D594ED0F0ADDED017A76
:1053A00030EE270A1FF028FC84ED0F0A002304F1D9
:1053B0003C0204F13001D5F830068DF808308DF844
:1053C00009308DF80A308DF80B30029BFEF734FB64
:1053D00007B0BDEC028B30BDA02C0024D488002483
:1053E000002070470120704701207047002070475F
:1053F000004870476CF010080048704774F01008BF
:10540000012070471FB5044600236A4601A9019395
:1054100002930393FFF784FE6369029A1B68C3F843
:10542000D4206369019A1B68C3F8D8206369009A85
:105430001B68C3F8DC206369039A1B68C3F8E0208B
:1054400004B010BD01207047002070470120704754
:1054500000207047004870475EB810080048704749
:105460005EB8100804207047012070477FB5002304
:105470000B4801AA03A90393049305930193002306
:10548000D0F830068DF808308DF809308DF80A30E4
:105490008DF80B30029BFEF7CFFA07B05DF804FBE6
:1054A000A07C002401207047002070470120704735
:1054B00000207047004870471CF1100800487047F2
:1054C00028F110080220704710B586B0002304466A
:1054D00001AA03A9039304930593FFF721FE6368D0
:1054E0009DED037AD3ED0B6ADDED047A27EE267A83
:1054F00093F9443067EEA67A8DED037ACDED047A08
:105500001BB903A91348FDF7BBF9636801AADDEDD8
:10551000057A03A993ED0C7A0F4867EE877A93ED2D
:105520000D7A0023D0F83006CDED057ADDED017A55
:105530008DF8083067EE877A8DF809308DF80A30DB
:105540008DF80B30029BCDED017AFEF78DFD06B094
:1055500010BD00BFA02C0024A07C002438B5044658
:105560005FF040F85FF0ACF9054604F5A0445FF049
:105570001BF95EF0BFFCD4F82C06FDF79BFC284617
:10558000BDE838405FF018B910B500F5A04414210B
:10559000D4F8AC035DF0FEF9D4F8B00314215DF04B
:1055A000F9F9D4F8B4031E215DF0F4F9D4F8B80386
:1055B0001421BDE810405DF0EDB9000038B5054696
:1055C0005DF0FEF85DF04AF805F5A044C4F8AC03C0
:1055D0005DF0F6F85DF04CF8C4F8B0035DF0F0F85B
:1055E0005DF050F8C4F8B4035DF0EAF85DF054F8EB
:1055F0004FF47A71C4F8B803D4F8AC035DF0C6F97F
:105600004FF47A71D4F8B0035DF0C0F94FF47A71B9
:10561000D4F8B8035DF0BAF94FF47A71D4F8B40352
:105620005DF0B4F92846FFF7AFFF94F8193643F060
:10563000080384F8193638BD08B55FF041F95EF00B
:1056400015FEBDE808405EF0C7BD000000F5A040B3
:10565000D0F82C06FDF758BD38B500F58043054657
:1056600093F9122A2AB900212846BDE83840FCF7F0
:105670009FBDB3F8143A00F5A0448B4219D994F8B1
:105680002936DA070FD45DF09BF8037F1BB9D4F8F5
:105690002C361B7B3BB194F8283601335BB2022BCE
:1056A00002DC84F8283638BD0323012184F828362B
:1056B000DAE794F82836013B5BB2002BF1DC0023DB
:1056C00084F8283694F82936DB07CCD4EBE70000C1
:1056D00038B50D46044684F0CBFB0C4B002D09DD9C
:1056E00004F5A044186094F819366FF3C30384F8E6
:1056F000193638BD1B68C01AB0F5C87FF9D904F552
:10570000A04494F8193643F00803F0E7A48E00246F
:10571000F7B5044684F0ACFB06465DF051F804F59D
:10572000A0455DF01FF8A8B395F81836204604F59B
:10573000C04743F0200385F81836D5F8B4331989EB
:10574000FFF78AFFD5F8B4332046B3F90A10FFF704
:10575000BFFFD7F8D8309FED307A6A46F31A01A917
:1057600004F5B84007EE903AD5F8B433F8EE677A0E
:10577000B3F90A3067EE877ACDED007A07EE903AFA
:10578000F8EEE77ACDED017A51F08EFAC7F8D860DD
:1057900003B0F0BD95F82936DB07F9D404F5C04312
:1057A000D3F8D800361A5CF0ABFE88BB5DF008F881
:1057B0009FED1A7AD0ED067A67EE877A9FED187A18
:1057C000F4EEC77AF1EE10FA77FE877AFCEEE77A0C
:1057D00017EE903AB342DBD804F5804393F9123ABE
:1057E000002BD5D05CF0ECFF037F23B9D5F82C3625
:1057F0001B7B002BCCD04EF037FF022211464EF01F
:10580000E3FC0121204603B0BDE8F040FCF7D0BC2A
:105810004FF47A73DEE700BF6F12833A00007A44D8
:105820000000C84238B500F5EE650446284604F08D
:105830006FFE94F8810750229FED087A04F5A0438B
:1058400002FB0055D5ED0B7A67EE877AFDEEE77A1D
:1058500017EE902AC3F8FC2B38BD00BF0000C842E9
:10586000FEF7B2B80148FFF795BA00BFA02C00249C
:1058700010B5838F044643B94CF09CFF92224FF43D
:1058800080114CF04FFF638FA387A08F10BD0000E5
:1058900038B500F5165504463835284600F0FCFCAE
:1058A00004F50053022204F51C7083F8D827FFF793
:1058B000DFFF014604F546601DF0F0FD2846BDE817
:1058C000384000F0EFBD000038B500F5165405462D
:1058D0003834204600F036FF08B9002038BD05F501
:1058E000A045D5F82C361B7B63B91021204601F06A
:1058F0003BFA0028F2D14FF400712046BDE8384051
:1059000001F032BA8021204601F02EFA0028E4D1BD
:105910001021F2E738B500F5A043054693F8293683
:105920005B070AD4FFF7D0FF044620B905F51650EF
:10593000383000F007FF204638BD0024FBE70000A8
:1059400000F5165008B5383000F0FCFE002008BD08
:1059500010B500F516543834204600F0F3FE50B16F
:105960000421204601F000FA28B120462021BDE89C
:10597000104001F0F9B9002010BD000038B500F565
:10598000A045044695F81836590719D5D5F82C3690
:105990001B7B2BB920460021BDE83840FCF7F2BB49
:1059A00000F5C043D3F8E0000368DB68984738B1DE
:1059B00095F819361A0703D595F82936DB07E9D586
:1059C00038BD000037B500F5DF55044601910835B4
:1059D00004F5A04428464DF043FF94F81836019989
:1059E00060F3C303284684F8183603B0BDE830409E
:1059F0004EF058BC072070470048704780F11008EF
:105A000037B505461148FFF733FF0190EC2006F04B
:105A10007FFC044610B10199FDF7ECF905F5A043B0
:105A2000C3F82C4634B905F58045094895F9601A44
:105A300005F0A0FF0749204649F02CFA012048F064
:105A4000C9FE03B0BDE8304049F01CBA102F002455
:105A500088F1100824AA100873B5044600F5155003
:105A6000283004F5EE6645F00FFA2046FFF7AAFA53
:105A700004F5AC40403005F031F904F5E850183039
:105A80005FF07EFD304604F0B5FB04F5A8404430DD
:105A900057F016FB2046FFF791FD2046FFF7B0FFB9
:105AA0006148FFF7E5FE082006F032FC18B14FF020
:105AB0007E530360436004F5A045C5F830065CF0F2
:105AC0007FFE992229215EF055F95CF079FE5CF0A9
:105AD00083FD2046FFF7B0FD95F8193604F5145004
:105AE00043F04003143085F8193662F0DDFF4F4B68
:105AF0004FF47A724E491B68986A0368DB6A9847CC
:105B0000042304F54A70C4F8C4330EF031FF07F0E3
:105B1000EDFA4FF40053436307F0E8FA08F02CF86D
:105B2000802301213046C4F8843704F011FE414B34
:105B300004F5DF500093404B0830019302AB13E9AA
:105B400006004DF035FD2046FFF7A2FE04F5805318
:105B50004FF40022C3F86C25D5F82C06FDF754F954
:105B600004F5A74001214830FBF7FAFF10B12046A9
:105B7000FFF76CFD04F51C763046FFF779FED5F88B
:105B80002C3607EE900A04F5B840D3ED390AF2EE50
:105B90000E1AB8EE670A4830B6EE001A51F07AFDD8
:105BA0003046FFF765FED5F82C3607EE900A04F56F
:105BB000B940D3ED390AF2EE0E1AB8EE670A0C308E
:105BC000B7EE001A51F090FB3046FFF751FED5F8C2
:105BD0002C3607EE900A04F5B940D3ED390AF2EEFF
:105BE0000E1A4030B1EE041AB8EE670A51F07CFB91
:105BF00004F580431A22204693F81F1AFFF702FA91
:105C000060B9212201212046FFF7FCF995F81936E9
:105C100043F0020385F8193602B070BD074A1378C5
:105C200043F008031370F1E7102F0024888E00243E
:105C300065580208A02C00246158020844900024F2
:105C4000836833B9C36823B94068003818BF01209E
:105C500070470120704700002DE9F0412DED048BC5
:105C600092B0044602AD284605F0F4FE94F8D43311
:105C7000002B70D004F58063D4EDF28A94EDF38AA2
:105C800094EDF49A0FCB85E80F0094F81034002BB4
:105C900061D094F8E833002B5DD02846D4F8D8833F
:105CA000D4F8DC73D4F8E063D4F8E443FFF7C8FF1A
:105CB000002855D12E4B01932D22002106A8E0F09B
:105CC000BBF8A3238DF8183095238DF8193046239F
:105CD0008DF81A3084F0D4F89FED260ADFED267A8D
:105CE00068EE808ACDF81F1028EE008ACDF81B00E0
:105CF00029EE000A68EEA78A28EE278A20EE270AF6
:105D0000FDEEE88ABDEEC88A18EE903AADF8233071
:105D100018EE103AADF825301EF02AFFBCEEC00A8E
:105D2000CDF83580CDF83970CDF83D6010EE103AE1
:105D3000CDF84140ADF82730019BCDF82930049BC8
:105D4000CDF82D30059BCDF831304EF08DFC2D2255
:105D500006A94DF065FC12B0BDEC048BBDE8F081E6
:105D600001AA0021284605F063FF0028A2D0A3E77E
:105D70005241C07FE02E65420000C84230B52DED93
:105D8000028B8BB0044624220D4601A80021E0F0CE
:105D900053F8A3239FED228A8DF8043095238DF8C4
:105DA000053048238DF8063084F06AF8D4ED847A03
:105DB0002B6867EE887A95ED020ACDF80F30CDF8A2
:105DC0000B1017EE903AD4ED857ACDF8070067EE08
:105DD000887ACDF813306B68CDF8173017EE903A0B
:105DE000CDF81B301EF090FE10EE103A94ED860AAE
:105DF00020EE080ACDF81F301EF086FE10EE103A95
:105E0000CDF8233094F824338DF827304EF02CFC55
:105E1000242201A94DF004FC0BB0BDEC028B30BD77
:105E2000E02E654230B5104689B00D461446FFF7A6
:105E300007FF28BB002301931822002102A8DFF0EE
:105E4000FBFFA3238DF8083095238DF809304923F3
:105E50008DF80A3084F014F8A368CDF80F1005937C
:105E6000E368CDF80B000693019B8DF81350079360
:105E70004EF0FAFB182202A94DF0D2FB09B030BD5A
:105E800001AA0021204605F035FE0028D2D0D3E734
:105E900010B590B0044604A805F0DCFD04A9204626
:105EA00001F020FC002846D001F0EAFE01A901F033
:105EB000EFF902A9204600F00FFD00283DD0DDEDEE
:105EC000027AF1EE677A03AA002104A8CDED027AE6
:105ED00005F0AEFE08B91A4B03931F22002108A853
:105EE000DFF0AAFFA3238DF8203095238DF8213011
:105EF0004A238DF8223083F0C3FF069BDDED017A43
:105F0000CDF82B30079BF1EE677ACDF82710CDF84E
:105F10002F30039BCDF82300CDF8333017EE903AA5
:105F2000CDF83730029BCDF83B304EF09DFB1F2261
:105F300008A94DF075FB10B010BDDFED027AC2E785
:105F40005241C07F5241C07F0023036043608360A1
:105F5000C360036143618361C361036270470000F2
:105F6000B02290F80C3302FB030390F8A12393F8BE
:105F7000E93012B1012B28BF0123184670470000F9
:105F80002DE9F04F05464FF0000A8BB00C4627F084
:105F9000ADFA05F5097085F820A24FF07E5783F021
:105FA0002BF84FF47A7305F5217085F88042A5F837
:105FB0007A320024C5F8607205F53179C5F864724B
:105FC00005F53A76C5F8687205F54E7B05F042FD99
:105FD00003234846C5F8AC42C5F8983205F27C4820
:105FE000C5F8B042C5F8B442C5F8B842C5F8BC42DD
:105FF000C5F8C042FFF7A8FF3046FFF7A5FF584697
:10600000C5F82C43C5F83043C5F83443FFF79CFF6F
:1060100005F57B70C5F85C43C5F86043C5F864437B
:10602000C5F86843C5F86C43C5F87043C5F87443B8
:10603000C5F87843C5F87C43C5F88043C5F8844368
:10604000C5F88843C5F8A443C5F8A843C5F8AC43D0
:10605000C5F8C043C5F8BC43C5F8B843C5F8C84344
:10606000C5F8CC43C5F8D043C5F8E443C5F8E043D0
:10607000C5F8DC43C5F8B473C5F8D87305F0EAFC7D
:1060800005F5806005F0E6FC05F2144305F5866031
:106090001C605C6005F584631C605C609C6005F0BE
:1060A000D9FC05F24443404605F254421C605C6052
:1060B0009C60764BC5F8543405F51073C5F8583418
:1060C00005F51173C5F85C3405F51273C5F8603435
:1060D00005F51373C5F8643405F25123C5F8683427
:1060E00005F51473C5F86C3405F58E631C605C60AF
:1060F0009C60FFF729FF05F59460FFF725FF05F584
:106100009A6305F2EC501C605C609C6005F2DC4315
:106110001C605C609C6005F59D631C605C609C601D
:1061200005F2F4431C605C609C6005F204531C6043
:106130005C609C6005F214531C605C609C6005F51B
:10614000A4631C605C609C6005F22C531C605C6066
:106150009C6005F5AA63C2F8EC70C2F8F0701C6090
:106160005C609C6005F25C531C605C609C6005F5A3
:10617000AD631C605C609C6005F274531C605C60E5
:106180009C6005F5B2631F605C6005F2B4531C604F
:106190005C609C6005F5B8631C605C609C6005F504
:1061A000BB631C605C609C6005F054FC05F2FC5312
:1061B000242251461C6040465C6005F204631C606A
:1061C0005C6005F20C631C605C60DFF035FE05F579
:1061D000C660C8F82070C8F81070C8F80070FFF7E3
:1061E000B3FE05F2546305F2AC601F609C605C6016
:1061F000DC6005F264631C605C609C6005F5CE6346
:106200001C605C609C6005F27C631C605C609C6050
:1062100005F5D1631C605C609C6005F294631C60B2
:106220005C609C60344605F015FC194B2846194902
:106230001D6048F035FC5146242258466E46DFF07A
:10624000FBFD05F52B7205F52E73C5F85873C5F8DF
:106250004873C5F8387307CA83E80700484695EDC8
:10626000B01AD5EDAF0A95EDAE0A1FF0BFF9494659
:1062700068461FF0E3F80FCE0FC40FCE0FC42846B8
:10628000336823600BB0BDE8F08F00BF68F41008DE
:10629000A88E002404F3100810B5044688B001F05D
:1062A0005BFD94F93E32012B02D1274805F080FBBB
:1062B000022B0AD1032304A904F1110084F83E3211
:1062C00001238DF8103049F0F7FB94F83E3204F2C8
:1062D000544084F8A83201F0FBFC94F93D32642B61
:1062E00030D1652304A904F23D208DF8103049F027
:1062F00021FC04A9204647F0BDFC18B304238DF807
:1063000018300023CDE9013303930F230593694629
:1063100004A847F031FE059B28B108AA009902EBBA
:10632000830242F8581C0133112B0593EFD97CF0FE
:106330003FFD9DED031ADDED020A65219DED010A89
:106340007CF0F4FC08B010BD98F1100870B500F5B1
:106350002B7600F52E758CB004463146284622F087
:1063600083FBE0B996E8070085E8070004F5317182
:1063700094EDB01AD4EDAF0A02AD94EDAE0A084622
:1063800001911FF033F9019902A81FF057F804F5A5
:106390003A740FCD0FC40FCD0FC42B6823600CB01F
:1063A00070BD000084B000F54E7004B01EF05ABFFE
:1063B00084B000F54E7004B01EF082BF13B50446E1
:1063C00000F5097140F2751201A819F0BDFA04F246
:1063D000544001F071FE204627F0C2FA01A819F0DE
:1063E000D5FA02B010BD0000F8B54B6801F11006F7
:1063F00007460C46C0F8103200F54E758B68C0F8A1
:106400001432CB68C0F818320FCE0FC50FCE0FC5AF
:1064100004F1440233682B6007F54B7307CA83E825
:10642000070004F1500207F5577307CA83E8070015
:1064300004F15C0207F55A73683407CA83E8070061
:1064400007F55D7394E8070083E80700384601F01C
:1064500097FD3846BDE8F84001F07ABD13B5044613
:1064600000F25440019003F0B3FA04F5C4610198BE
:10647000009102F059FE0099204602B0BDE810409C
:10648000FFF7B2BF4A78064BC2F340121A754A783A
:10649000C2F380125A750A78C2F300129A757047D7
:1064A0002590002413B5044600F5097140F24D32E1
:1064B00001A819F049FA002104F2544002F02AF828
:1064C00094F8783223B1204628F0F0F884F8780266
:1064D00001A819F05BFA02B010BD000038B590F8C1
:1064E000243305460C462BB1032B0BD095F8803294
:1064F000DB070CD405F2AC630FCB84E80F0095F8F2
:10650000BC0603E027F0AEFA0028EFD038BD00202B
:10651000FCE7000000F2544090ED3B0A7047000099
:1065200000F2544090ED3C0A7047000010B490F81F
:1065300024230C462AB1032A0AD000205DF8044B1C
:10654000704700F5BB6007C884E807000120F5E745
:106550005DF8044B27F042BA90F89C03431E584262
:106560005841704738B590F824330D468BB900F286
:10657000544001F009FE044610B90024204638BDFD
:1065800001F056FDD5ED007A27EE800A85ED000A70
:10659000F4E7D0EDE67AC1ED007A90F89443002C50
:1065A000EBD090EDE47ADFED076AB4EEE67AF7EE31
:1065B000006AF1EE10FA27FE267A67EE877AC1EDBF
:1065C000007ADBE70000003490F82433032B01D17C
:1065D00027F080B90020704790F82423032A01D1C6
:1065E00027F04ABB00F2544002F0E6B930B5054648
:1065F00085B00C469AB1032A1BD005F52B7022F00A
:106600006DFA01A920468DED010ACDED020A8DED4E
:10661000031A21F00BFB0123184605B030BD90F89A
:106620002036002BF8D000F254630FCB84E80F0023
:10663000E3E790F87832002BEED027F0E7FADCE7BA
:1066400090F82423FFF7D2BF7FB590F8242332B10E
:10665000032A4FF0000309D0039304930CE000F2E7
:10666000544007B05DF804EB01F0D8BD03A90393D3
:106670000493059327F024F99DED030ADDED040A48
:1066800007B05DF804FB000037B504460D4640F244
:10669000C75200F5097101A819F056F9204629469C
:1066A00027F00AFA94F82433032B0CBF0446002485
:1066B00001A819F06BF9204603B030BD10B52DEDDF
:1066C000028BB0F8C03682B004461B0730D5D0F834
:1066D000383401A99FED188A00F5157007EE903A3D
:1066E000B8EEE77A27EE087A8DED017A49F0D0F915
:1066F000D4F83C3401A904F5167007EE903AF8EE90
:10670000E77A67EE887ACDED017A49F0C1F9D4F8DD
:10671000343401A99FED097A04F5177007EE903A19
:10672000F8EEE77A67EE877ACDED017A49F0B0F9B5
:1067300002B0BDEC028B10BD95BFD6330AD7233C07
:1067400027F0EEB990F82403003818BF01207047F5
:1067500038B590F824230C46032A04D1012527F0EC
:10676000AFF8284638BD90F8A056002DF9D000F2B9
:10677000946393E8070084E80700F2E710B590F807
:10678000242303460C461AB1032A0BD0002010BD67
:1067900090F8A8060028FAD003F5C463D3F8843033
:1067A0000B60F4E727F0A2F8012084ED000AEEE781
:1067B00090F82433032B01D127F0E8B9002070476B
:1067C00030B590F8243387B005460C4623B1032B2F
:1067D00009D0002007B030BD00F2544007B0BDE83A
:1067E000304002F095BB0022002302A9CDE902232C
:1067F000CDE9042327F04CF80028EAD06946284662
:1068000027F052F80028E4D0DDE90223C4E9002390
:10681000DDE90423C4E90223DDE90023C4E90423FC
:10682000D8E7000010B586B0002200230C46694668
:10683000CDE90023CDE90223CDE90423FFF7C0FF12
:1068400088B19DED027B9DED005BF7EEC76BB7EE67
:10685000C55B9DED047B84ED005AC4ED016AB7EE83
:10686000C77B84ED027A06B010BD000090F82423A7
:106870001AB1032A05D00020704700F2544002F0FC
:1068800083BB27F005B800001FB5002200230C468B
:106890006946CDE90023CDE90223FFF7E7FF58B1B0
:1068A0009DED027B9DED006BB7EEC77BB7EEC66B2F
:1068B00084ED017A84ED006A04B010BD90F82423C1
:1068C0001AB1032A05D00020704700F2544002F0AC
:1068D00045BB26F0E9BF000013B50C466946FFF73B
:1068E000EDFF28B19DED007BB7EEC77B84ED007A0C
:1068F00002B010BD90F93E323BB990F8803213F0EF
:10690000010F14BF032000207047032070470000D0
:10691000F7B50446FFF7EEFF0546002862D00328CE
:1069200039D194F878326BB394F88032D8072BD5EC
:1069300001A9204627F0A8FABDF80430002B18BFA3
:10694000002594F8206206F0FD06012E4AD10023AE
:10695000032D019307D101A9204627F0A1FA204673
:1069600027F0BAF9064604F2544002F023FC08B9B5
:1069700094F821039DF80430D90703D55A0701D5AF
:106980009F0632D400252DE0204626F0E3FE0028A5
:1069900008BF0025D5E70025D3E713F0020F2EE04E
:1069A00094F9503223B99DF80430DB092FD0E9E780
:1069B000002EF8D00FF0D4FDFFF7D2FA022807D945
:1069C0009DF805309806DDD59DF80430D906D9D557
:1069D000FB6A93F89C30002BE5D118E0DA0601D46D
:1069E0001B0718D5284603B0F0BD0028FAD094F84C
:1069F0002123B4F9C036002ACFD013F0010FF1D112
:106A0000154B1F68FB6A93F89C30002BC8D19DF88A
:106A100004309C07E2D406F069FB06F063FA002814
:106A2000B0D10FF09DFDFFF79BFA0228AAD90FF015
:106A300097FDB02290F80C33F0EE007A02FB0300D1
:106A400090ED417AB4EEE77AF1EE10FA9AD59DF81E
:106A50000530DB09C6D195E7888E00242DE9F04783
:106A600090F8783292B00446002B00F093802046D4
:106A700027F08CFB2046FFF74BFF03287AD104F563
:106A80004E78002720464FF00C0A414600970197A8
:106A9000029727F091F86946204627F083F8009B7B
:106AA0002046C4F81032019BC4F81432029BC4F88B
:106AB000183201F065FA204601F04AFA1CF006FC93
:106AC0000546204626F0D6FE002803AA4FF0FF31E7
:106AD000AEBFC6B295F8049995F805692046A8BFDF
:106AE000B14603970497059726F00EFF03A804F517
:106AF0005D7721F0F3FF0AFB09500AFB065504F508
:106B0000577184EDD70A00F5DC60C4EDD80A05F5AD
:106B10005F7584EDD91A06AE21F0F0FF3A4684ED98
:106B2000CB0A4FF0FF31C4EDCC0A204684EDCD1ADC
:106B300026F0FEFE95E8070086E807003946304655
:106B400022F042F804F53172414609A81EF008FC13
:106B5000314609A81EF086FB09A9204684EDDA0A11
:106B6000C4EDDB0A84EDDC1A27F09AF909A9204666
:106B7000FFF788FC94F8C236002B3AD109A804F03C
:106B800069FF09A9204626F079FF90B3012384F814
:106B9000C2362EE0D0F87C321BB983F069F9C4F814
:106BA0007C02154B1B68D86A03685B68984788B1FC
:106BB00083F05EF9D4F87C32C01AB4F87A32984285
:106BC00004D9204627F072FD84F8780294F87832D0
:106BD0007BB14CE783F04CF9D4F87C32C01A41F217
:106BE00087339842E4D84DF03FFD4DF077FB002805
:106BF000DED112B0BDE8F087888E002490F82433EF
:106C000023B1032B4FF0000007D0704790F93E22CC
:106C1000032A04D10A70012070470870FBE7184668
:106C20007047000073B50D460DF107010446FFF7EC
:106C3000E5FF064628B19DF807302BB1032B09D09C
:106C40000026304602B070BD04F2AC630FCB85E87D
:106C50000F00F6E72946204626F004FF94F87862F4
:106C6000EFE7000037B50D460DF107010446FFF7C9
:106C7000C5FF28B19DF8072029462046FFF7B6FC3E
:106C800003B030BD37B50D460DF107010446FFF7DF
:106C9000B5FF28B19DF8073023B1032B11D0002098
:106CA00003B030BD04F224631B682B6004F5C56398
:106CB0001B686B6004F22C631B68AB6094F82006C1
:106CC000EEE72046294626F06DFF94F87802E7E7C4
:106CD00010B50446FFF70EFE18B1032807D00020B8
:106CE00010BD04F25440BDE8104001F021BA94F800
:106CF0007832002BF3D0204626F02CFD0028EED071
:106D000094F8203203F0FD03012BE9D194F8240319
:106D1000C31E58425841E3E710B50446FFF7EAFDA9
:106D200080B1032810D194F8780250B183F0A0F814
:106D3000D4F87C32C01A44F62063984294BF0020F5
:106D4000012010BD0120FCE70020FAE708B502464B
:106D5000FFF7D0FD032804D1104627F0A1F8012049
:106D600008BD0020FCE7000013B50C4601A9FFF7A1
:106D7000EDFF20B1019B1C4214BF0120002002B096
:106D800010BD000030B585B00446019102F032FF1D
:106D90000199054610B9002005B030BD019102F0FF
:106DA000F9FE01990028F6D0284602F0F7FE0028E7
:106DB000F1D0B4F8C0365907EED494F82133002B43
:106DC000EAD00B4A1268D26A92F89C506DB103A9BE
:106DD0002046FFF7BBFF30B19DF80E309A07DBD598
:106DE000C3F38000D8E72846D6E71846D4E700BFAB
:106DF000888E002410B4BDF8044001945DF8044B63
:106E000026F0E2BF10B4BDF8044001945DF8044BD5
:106E100026F076BF26F0AEBF90F840245AB100F2BB
:106E200034439FED057AD3ED007AF8EEE77AA7EECA
:106E3000C70A27F003B870470AD7233C10B50446A9
:106E4000FFF758FD032804D12046BDE8104026F086
:106E5000DDBD002010BD00002DE9F04190F8243385
:106E60008CB000270646032B0C4615460097019769
:106E7000029719D126F0FEFC6A4680464FF0FF319A
:106E8000304626F055FDB8F1FF3FA76067602760E8
:106E90000DD11CF01BFA2B46224690F805191AF06A
:106EA0008DFF0CB0BDE8F0814FF0FF38EBE71CF030
:106EB0000DFA2B4622465FFA88F11AF07FFF95ED16
:106EC000000A684621F046FE03A920468DED051A0A
:106ED0008DED030ACDED040A21F076FE06F5317240
:106EE00006F54E7103A81EF03BFA214603A81EF0DA
:106EF000B9F9DFED077A84ED021A84ED000AC4EDDA
:106F0000010A95ED007AA7EE271A84ED021AC8E768
:106F10000AE81C41DFED0B7A20EE270A1FB50C466C
:106F20001946094BBDEEC00A1868084B8DED020AE0
:106F3000CDE900429DF81820C06A18F007FF04B0A0
:106F400010BD00BFE02E6542888E0024ACF1100811
:106F50002DE9F0472DED028B92B000254FF07E5ABF
:106F600004460F4600F54E7106A89046CDF818A0CD
:106F700009950895079520F019F906F0B7F805F07E
:106F8000B1FF81462046FFF7B5FC032803D094F8F3
:106F90002433032B4FD100269FED548ADFED548A12
:106FA0002379F2B2934247D90AAA71B22046CDF8AA
:106FB00028A00D950C950B9526F008FE0AA906A8A9
:106FC00020F064FEB4EEC80AF1EE10FA0DDD3B4687
:106FD000484ACDF8008048492046FFF79BFF002033
:106FE00012B0BDEC028BBDE8F0870AA906A8039594
:106FF0000495059520F034FE03A90EA88DED0E0A28
:10700000CDED0F0A8DED101ACDED111A20F09CFB7D
:10701000B9F1000F0DD09DED050AB0EEC00AB4EE37
:10702000E80AF1EE10FA04DD3B46344ACDF8008060
:10703000D1E70136B4E7002394F8806216F001002E
:1070400001D0012BCCD104F5C6610AA8CDF828A047
:107050000D950C950B9520F0A9F80AA906A820F02B
:1070600015FEDFED227AB4EEE70AF1EE10FA05DD47
:107070003B46204ACDF800802149ADE72046FFF786
:1070800039FC03282DD1204626F002FE94F88032E8
:10709000DB0728D438BB0AA906A8039504950595F3
:1070A00020F0DEFD03A90EA88DED0E0ACDED0F0A2E
:1070B0008DED101ACDED111A20F046FBB9F1000F3D
:1070C00011D09DED050ADFED0A7AB0EEC00AB4EEEC
:1070D000E70AF1EE10FA06DD3B46084ACDF80080DB
:1070E000CAE70020D2E701207AE700BFC2B8323EEB
:1070F000C2B8B23ED8F11008E3F11008C3A31008DB
:10710000E8F110082DE9F743154604468846019337
:10711000FFF7DEFD019A074638B928482946284B73
:107120000068C06A18F012FE019A294620460192B2
:10713000FFF70EFF064668B32046FFF7DBFB94F926
:107140003E1243B2019A994207D01E4B1B48294672
:107150000068C06A18F0FAFD1CE094F824338342FA
:1071600007D0019205F0C2FF05F0BCFE019A00288D
:10717000EBD12046FFF7BEFB18B103280FD0124B0E
:10718000E4E7134641462A4604F2544000F0E4FF87
:1071900000B107B90026304603B0BDE8F08394F88B
:1071A0007892B9F1000F01D1084BCFE71346414661
:1071B0002A46204626F0DEFAEAE700BF888E002441
:1071C000ECF11008F8F1100828F2100817F2100876
:1071D00090F82433032B01D126F078BE00207047AD
:1071E00013B5044600F5097140F6783201A818F08D
:1071F000ABFB204626F0CEFB01A818F0C7FB02B07F
:1072000010BD000008B50246FFF774FB10B103285B
:1072100006D008BD02F25440BDE8084000F05CBF53
:107220001046BDE8084026F047BE00000B46114658
:1072300010B42BB1032B09D000205DF8044B70472C
:1072400000F254405DF8044B00F052BF5DF8044B6F
:1072500026F014BC13B504460A46FFF74BFB014663
:1072600020460192FFF7E2FF70B9084B019A1B68B4
:10727000DB6A93F89C0038B194F82413204602B0DE
:10728000BDE81040FFF7D2BF02B010BD888E0024C9
:1072900070B590F8943286B004460D46DB070CD4E6
:1072A00003F0A2FB5022437C02FB0300D0ED0B7ADB
:1072B000F1EE677AC5ED007A41E002A804F0CAFB5E
:1072C00069462046FFF7FAFAE8B90FF049F994F950
:1072D00050320646022BE3D1FEF742FE0228DFD9E8
:1072E000B02396F80C039FED177A03FB0066D4F8E1
:1072F0008832D6F8F8209B1A07EE903AF8EEE77A33
:1073000067EE877AD6E702A92046FFF7A3FF002899
:10731000DBD0D4F88822039BDFED0A7A9B1A07EEB4
:10732000103AB8EEC77A9DED006B27EE277AB7EEDC
:10733000C77A36EE477BB7EEC77B85ED007A06B09D
:1073400070BD00BF0AD7233CF0B587B00C46064697
:1073500000F5097140F6DD3201A818F0F5FAA368CE
:1073600053B9E36843B9636833B9002701A818F03B
:107370000DFB384607B0F0BD204604F08DFC002818
:10738000F3D002AD94E80F0085E80F0000212846F5
:1073900004F03EFC07460028E7D096F89432DB075D
:1073A00004D44DF061F919214CF0EEFE06F5217C74
:1073B00095E80F008CE80F0096F89432304643F0C1
:1073C000010386F8943200F013FE58F0AFFD462119
:1073D0005AF010FA58F0AAFD45215AF00BFA084B62
:1073E000A2681B68DB6A1A61E2685A6162689A6186
:1073F00024F022FF0028B9D022F046FBB6E700BFF8
:10740000888E002438B5144B04461B68DD6A2B684F
:1074100028465B689847F0B12B690BB96A69D2B10D
:10742000C4F88C3200226B6904F52170C4F89032E4
:10743000A96904F013FB94F8943223F0030343F09A
:10744000030384F8943258F071FD044A0621BDE824
:10745000384052F02FBE38BD888E00243CF2100810
:1074600013B504460193FFF745FA0328019B05D1A4
:10747000204602B0BDE8104026F0D2BB002002B08A
:1074800010BD000010B588B004460593FFF732FA2E
:107490000328059B4FF000000AD10690079006A82C
:1074A00002900B9801900A980090204626F0C6FBA7
:1074B00008B010BD13B504460193FFF71BFA03286B
:1074C000019B05D1204602B0BDE8104026F0C4BBA8
:1074D000002002B010BD000038B5044602F08AFB5F
:1074E0000546D0B194F82433032B03D095F84E41D0
:1074F000204638BD204626F07DFAFF280446F5D008
:107500000146284602F04AFB0028EFD021462846D3
:1075100002F040FB0028E9D0EAE70446E8E7000073
:1075200008B590F82433032B05D01BF0CFFE90F95B
:107530000409C0B208BD26F09DF9431CF9D1F4E757
:1075400008B590F8243383B1032B03D1BDE808407C
:1075500026F088B94BF02EF940F64C524FF48011CA
:107560004BF0E0F84FF0FF3008BD1846FCE7000094
:10757000FFF7D6BF90F82433032B01D126F070BF5C
:107580007047000090F82433032B01D126F062B835
:107590007047000026F0C6B826F0DEB910B50446E4
:1075A00029F078FC2046FEF757FB2046BDE8104046
:1075B000FEF76EBC90F824330BB1032B01D126F0FB
:1075C00073BB00207047000090F824231AB1032AEF
:1075D00007D00120704790F95002003818BF0120F1
:1075E000704726F06DBB000010B590F840348AB0AB
:1075F0000446002B62D1B0F8C036DB065ED590EDB4
:10760000957ADFED2F7AB0EEC77AB4EEE77AF1EE35
:1076100010FA11D590ED967AB0EEC77AB4EEE77A0B
:10762000F1EE10FA08D590ED977AB0EEC77AB4EE85
:10763000E77AF1EE10FA41D42046FFF7C5FF0028A3
:107640003CD1D4ED976ADFED1F7A9FED1F6A66EE9D
:10765000A76A94ED967AD4ED957A27EE067A009093
:1076600067EE867A06A8FDEEE66ABDEEC77AFDEE05
:10767000E77A16EE903A17EE102A17EE901A04F0F9
:1076800007FA06A92046FEF7FFFFB8B158F04EFCF6
:1076900094ED977A0D4A0621B7EEC77A8DED047BFB
:1076A00094ED967AB7EEC77A8DED027B94ED957ADC
:1076B000B7EEC77A8DED007B52F0FCFC0AB010BD2E
:1076C000000000340000C8428096184B54F21008A5
:1076D00090F824330BB1032B01D126F029BF0020F1
:1076E0007047000000F57B7330B504460D460FCBA4
:1076F00085E80F0094F8FC0330BD00007FB5064616
:1077000068460D4604F0A6F996F89432DB0703D4D8
:107710000024204604B070BD69463046FFF7E2FF02
:1077200004460028F4D0694606F5217004F0A0FB59
:1077300085ED000AC5ED010A85ED021AE9E70000B2
:1077400000F56072034610B50C4607CA84E80700CE
:1077500093F88C0310BD000000B52DED028B85B0B1
:10776000B0EE408A9FED120A01A98DED010A8DED60
:10777000020A8DED030AFFF7E3FFA0B1DDED010A78
:107780009DED020AF1EE600AB1EE400ADBF0AEFCBC
:10779000DFED087AA8EE670A05B0BDEC028B5DF854
:1077A00004EBDAF0CBBC05B0BDEC028B5DF804FB5A
:1077B0000000000035FA8E3C10B52DED028B90EDE7
:1077C000800A0446FFF7C8FFB0EE408A04F56070F7
:1077D00021F040F820EE080ABDEC028B10BD00003D
:1077E000D0F898330B6090F894037047D0F8A0332A
:1077F0000B6090F89D03704700F56972034610B561
:107800000C4607CA84E8070093F8B00310BD0000D7
:1078100000F56D7330B504460D460FCB85E80F00BB
:1078200094F8C40330BD000000F5866330B504460B
:107830000D460FCB85E80F0094F8400430BD0000E2
:1078400000F24442034610B50C4607CA84E807001C
:1078500093F8500410BD00002DE9F04305460E4694
:1078600017462DED028B8BB0FFF736FE01468046A2
:107870002846FFF787FA0446002846D002F0BAF9F6
:10788000414602F08DF986ED000A95F93C32002B55
:1078900038DD0EF065FEFEF763FB012832D90EF0ED
:1078A0005FFEB02290F80C33B7EE008AD5EDE47A93
:1078B000DFED598A02FB030095F93C32F4EEE87AD9
:1078C000D0ED410A07EE103A96ED000A40F20E4064
:1078D000F1EE10FAB8EEC77A67FE887A20EE270A32
:1078E00037EE201A70EEC70A1DF0B2F9D5EDE47A32
:1078F000F4EEE87AF1EE10FA67FE887A80EE277AE5
:1079000086ED007A01233B7003E095F8203333B90C
:10791000387020460BB0BDEC028BBDE8F0834FF011
:10792000000995F82433CDF80490CDF80890CDF8EF
:107930000C9043B1032B10D0CDF81090CDF81490DB
:10794000CDF818907CB902233246414605F25440E6
:107950003B7001F073FB0446DBE701A9284626F0E3
:107960003DF80446E8E795F82433002BEBD004A952
:107970002846FFF765FF04460028E4D001A904A8C3
:1079800021F0D2F807A8CDED080A8DED091A8DED8A
:10799000070A21F0FDFC04A8B0EE408A21F0F8FCB3
:1079A00095F93C32002B2EDD07EE903A40F2544020
:1079B000F8EEE77A70EE670A37EE801AB0EE480A02
:1079C000F5EEC00AF1EE10FA48BFDFED140AF4EE4E
:1079D000410AF1EE10FA30FE811A1DF039F9B0EECD
:1079E000408AD5EDE47A03239FED0B7AF4EEC77A53
:1079F000B7EE007AF1EE10FA67FE877A88EE277A02
:107A000086ED007A7FE7B5EEC08AF1EE10FA48BF46
:107A10009FED028AE5E700BF00000034000000008F
:107A200038B50446FFF77CFD054694F826338342BB
:107A300004D01BF04BFC29461AF07AF82046FFF7D9
:107A40006FFD84F8265384F825032046FFF768FD70
:107A500084F827032046FFF773FD04F5607184F86E
:107A600028032046FEF762FD84F88C0300F0E0FA5C
:107A700004F5677284EDE40A04F566712046FFF7A9
:107A8000EBFE04F5687184F894032046FEF76AFD66
:107A900004F5697184F89D032046FEF795FD04F511
:107AA0006D7184F8B0032046FEF7CAFD04F57271CB
:107AB00084F8C4032046FFF7E5F804F5767184F8EE
:107AC000D4032046FFF7CEF804F57B7184F8E80371
:107AD0002046FEF703FD04F5806184F8FC03204690
:107AE000FFF7A0F884F810042046FEF7ADFD04F27D
:107AF000144004F5836380ED000AC3ED000A20F012
:107B0000A9FE04F21C4304F58461204604F22C42D1
:107B100083ED000AFFF7A0F904F586612046FFF720
:107B200099FB80B194F840349BB90123204684F836
:107B3000403400F05DFA58F0F9F9452159F05AFE49
:107B40002046FEF7BBFD94F8403413B92046FFF7FA
:107B50004BFD04F244412046FEF7FAFD84F8500440
:107B600038BD000037B50D46044600F0F5F81DB9E4
:107B70001BF0ACFB1AF04CFA4FF4EA7204F50971F1
:107B800001A817F0E1FE94F881322BB92046FFF7E7
:107B900039FC012384F88132224B1D68A86A0368EE
:107BA0009B6998472046FEF7D1FB2046FEF756FC1E
:107BB000204600F059FA2046FEF750FF286B30B1FE
:107BC0000368D4EDD80ADB6894EDD70A9847D4F857
:107BD0001C0208B1A3F040FB204600F079F82046D3
:107BE000FEF796FE94F8A83284F8240383420ED060
:107BF00084F8A80298B10C4D0C4B032808BF1D4611
:107C000058F094F92B460A4A062152F053FA2046BE
:107C1000FFF706FF01A817F0B9FE03B030BD054D10
:107C2000EEE700BF888E002419BE1008E3F11008AB
:107C300080F21008E8F11008D0EDE47AB7EE000AFF
:107C40009FED047AF4EEC77AF1EE10FA27FE800A6F
:107C5000704700BF00000034D0EDE47AB7EE000AB0
:107C60009FED067AF4EEC77AF1EE10FA67FE807A9D
:107C700067EEA77A80EE270A704700BF0000003445
:107C8000014B1868704700BFA88E002470470000A1
:107C900070470000704700000020704700207047C8
:107CA0000120704703681B6E1847000000207047D2
:107CB0000020704700207047002070477047000088
:107CC0000020704700207047002070477047000078
:107CD0007047000008B51BF0F9FA90F8040908BDD8
:107CE00030B59FED1B1A0C46DFED1A0A05462D2014
:107CF0002DED028B87B091ED000A8DED011ACDEDCF
:107D0000000A1CF0A5FF9DED011AF0EE408ADDEDA2
:107D1000000A2E2094ED010A1CF09AFF9DED011A35
:107D2000B0EE408ADDED000A2F2094ED020A1CF02F
:107D30008FFF03A905F52B70CDED038A8DED048A25
:107D40008DED050A47F0DAFF07B0BDEC028B30BDC0
:107D5000C2B8323EC2B832BE10B5044682F088F8CE
:107D6000D4F80C331BB1C21AB2F57A7F12D30A4A87
:107D70001268D26A92F89C2002B15BB9C4F80C0375
:107D800094F83D421BF0A2FA80F8F74805F0AEF9EE
:107D900080F8294010BD00BF888E00242DE9F043F3
:107DA0002DED028B87B091ED007AD1ED037A0C4670
:107DB0008DED047AB0EEC77A15461E46DDF84C907C
:107DC000B5EEC07ACDED057ADDE91087F1EE10FA57
:107DD00006DCF0EEE77AF5EEC07AF1EE10FA02DD9D
:107DE00004A820F0ABFDB7EE001A6B20FFEE000AEE
:107DF0009DED050A1CF02CFFB7EE001AFFEE000AFD
:107E00006C2089ED000AB7EE008A9DED040A1CF093
:107E10001FFF04A888ED000A20F000FD002852D0C2
:107E20000023C9F8003088ED008AD4ED067A67EEA9
:107E3000A77AF4EEC87AF1EE10FA4ADB0023336039
:107E400085ED008AB7EE001A7C20DFED3E0A96ED44
:107E5000000A1CF0FDFEB7EE001A86ED000AFFEEE8
:107E6000000A7D2095ED000A1CF0F2FE85ED000A67
:107E7000D4ED067A129BF1EE677ADFED336AC3ED3B
:107E8000007A96ED007AF0EEC77AF4EEE67AF1EE3B
:107E900010FA2BD503AB02AA01A920461DF006FC5F
:107EA0009DED018AB0EE480ADAF048F985ED000A46
:107EB000B0EE480ADAF048FF87ED000A07B0BDECE3
:107EC000028BBDE8F08304A820F094FC0028A7D121
:107ED000ABE738EE670A1CF0DFFD86ED000A94ED93
:107EE000087AC7EE007AC5ED007AABE794ED076A31
:107EF000C6EE077AC7ED007A96ED007AB0EEC77A43
:107F0000B4EEE67AF1EE10FAC4D495ED007ADFED26
:107F10000F6AB0EEC76AB4EE666AF1EE10FAB9DC29
:107F2000B4EE477AF1EE10FAB4D6B0EEE77AB4EEDA
:107F3000667AF1EE10FAADDCF4EE677AF1EE10FA43
:107F4000BCD7A7E70000000000000034FFFF7F7FE0
:107F50001FB500F51D7300F5187200F54E710393FF
:107F600000F51C73029300F51B73019300F51A735F
:107F7000009300F51973FFF711FF05B05DF804FBDE
:107F80009FED196AD0ED846ADFED187A66EE866A95
:107F900090ED860A20EE060A26EEA77AC0ED7E6AEC
:107FA00010B5BDEEC77A044680ED817A90ED857AF2
:107FB00027EE067A67EE275A80ED7F7A60EE277A01
:107FC000FDEEE55AFDEEE77AC0ED825A17EE903AE3
:107FD000002BBCBF03F50C43A033C0F80C321CF0DF
:107FE00093FD84ED800A10BDE02E65420000C8427A
:107FF0001FB50E4B04461B68B3B1684603F02AFD5B
:1080000069462046FFF710FC20B16A460021204651
:10801000FDF708FF94F89432DB0705D504F52172CB
:1080200001212046FDF7FEFE04B010BD4C93002454
:1080300008B502F0D9FCBDE8084001F017BF000008
:108040007FB51BF043F990F8051907B05DF804EB14
:1080500019F088BF10B5044680F8101381F008FFAE
:10806000C4F8140310BD000010B590F81033044696
:1080700053B181F0FDFED4F81433C01AB0F57A7F05
:1080800084BF002384F8103394F8183353B181F07F
:10809000EFFED4F81C33C01AB0F57A7F84BF0023FA
:1080A00084F8183310BD000000F5C2700B4607C8F5
:1080B00083E80700012070470023C0F89C30C0F817
:1080C0009830C0F89430C0F8A830C0F8A430C0F898
:1080D000A030C0F8AC30704770470000024B0B6016
:1080E0004FF07C5313607047000048427047000017
:1080F00000F5CC7010B50C460FC884E80F00204680
:1081000003F09CFC30B1FFF7BBFD00F521700FC8F8
:1081100084E80F00204603F091FC80F00100C0B21B
:1081200010BD000010B5044604F0FAF8204610BD5A
:1081300010B5D0F8903104465BB181F099FED4F8C7
:108140009031C01A41F28833984294BF0020012038
:1081500010BD0120FCE7000013B5009303680192F5
:10816000DB6D98470446DDE9002128B90448054B3A
:108170000068C06A17F0EAFD204602B010BD00BFDB
:10818000888E0024ECF1100813B50446019101F02B
:1081900031FD019A23680146DB6B08B190F84E115E
:1081A000204602B0BDE810401847000090ED007A6C
:1081B000DFED0F7AB0EEC77AB4EEE77AF1EE10FA9F
:1081C00014D590ED017AB0EEC77AB4EEE77AF1EE0D
:1081D00010FA0BD590ED027AB0EEC77AB4EEE77ADA
:1081E000F1EE10FA4CBF01200020704700207047CC
:1081F0000000003410B501F0FDFC044658B190F8C1
:108200004E1101F0C7FC30B194F84E112046BDE884
:10821000104001F0C3BC002010BD00002DE9F04368
:10822000002504462DED028B8FB0036802A99B6BDD
:10823000039504950595069502959847064638B12D
:10824000FFF7F6FEDDED027A27EE800A8DED020AD9
:108250000EF086F9FDF784FE0746002E50D0DDEDC6
:10826000027A0BA9D4ED706A204694ED717A2368E6
:1082700027EE877A0B9567EEA67A0C950D9509ADDA
:108280008DED097ACDED0A7A5B6B98470BA92846EC
:1082900020F028FA012F8DED030ACDED040A40F2FB
:1082A000B3800EF05DF9B02590F80C33DFED5A7A0B
:1082B00005FB030090ED428A28EE278AB0EE480ABB
:1082C000D9F03CFFF0EE408AB0EE480ADAF03CFD0F
:1082D0008DED0C0ACDED0B8A0EF042F990F80C33BF
:1082E00005FB030009AD90ED410A0BA820F01AFA36
:1082F00005A88DED050ACDED060A96BB03C885E0FD
:108300000128CED89DED020AB5EEC00AF1EE10FAB2
:108310007FDD07AED4F8C421D4F8C03130460792CF
:10832000089320F029FA23680BA90B9520460C9599
:108330000D955B6B9847DDED077A9DED0B7A09ABE8
:1083400077EE877A9DED0C7ACDED077ADDED087A30
:1083500077EE877ACDED087A96E8030083E803008C
:1083600049E02369B7EE008A04F5D47904F5DC7698
:1083700093ED000A03AF04F5D87838EE408A20F078
:10838000D1F98DED090A4846CDED0A0AB0EE480A4A
:1083900020F0C8F90BA92846CDED0C0A8DED0B0A8B
:1083A00020F0A0F93146C4ED6B0A384684ED6A0A24
:1083B00020F0A8F98DED090AB0EE480A4046CDED4F
:1083C0000A0A20F0AFF90BA928468DED0B0ACDED76
:1083D0000C0A20F087F984ED6C0AC4ED6D0A97E869
:1083E000030086E803004946404620F07BF98DED06
:1083F000090ACDED0A0A9DED090ADDED0A0A0FB062
:10840000BDEC028BBDE8F083DDE9030185E80300E4
:10841000F1E709950A95EEE735FA8E3C10B590F82C
:108420004613044604F072F97C23C0B203FB0044F7
:10843000D4F8A40010BD0000044B026F1B68DB6A77
:108440005A60426F9A60826FDA607047888E0024AB
:10845000F0B58FB004461AF039FF002302AA90F855
:10846000041902930546039304F19407049301ABA6
:1084700019F044FCD8B39DED010AB5EEC00AF1EE47
:1084800010FA34DD04F1B00602A820F073FB39467F
:1084900084ED2C0A3046C4ED2D0A84ED2E1A20F00E
:1084A00079FB04F17C01304620F028FB04F18801BF
:1084B00005A88DED050ACDED060A8DED071A20F011
:1084C0001DFB08A88DED080A9DED010ACDED090AF6
:1084D0008DED0A1A20F03EFB0BA904F128008DED6A
:1084E0000B0ACDED0C0A8DED0D1A1DF001F995F872
:1084F00004090C23394603FB005000F5DC6020F032
:10850000FDFA84ED2C0AC4ED2D0A84ED2E1A0FB06D
:10851000F0BD00007B4B2DE9F04700251F680446A5
:108520000E462DED028BC0F89C508AB0C0F89850D2
:1085300004F12809C0F89450C0F88450C0F8805065
:10854000C567C0F89050C0F88C50C0F88850C0F88B
:10855000B850C0F8B450C0F8B050F86A03685B680F
:10856000984700284CD081F083FC42F20F73984268
:1085700046D8FB6A484693ED010A84ED1C0AD3ED08
:10858000020AC4ED1D0A93ED031A84ED1E1A1DF0B4
:108590002DF857F0CBFCDFED5C7A94ED1E6A0621D6
:1085A00094ED1C7A26EE276A584A27EE277AB7EE12
:1085B000C66A8DED046B94ED1D6A26EE276AB7EE50
:1085C000C77AB7EEC66A8DED007B8DED026B51F078
:1085D00071FD94ED1E8AB0EE480AD9F0AFFD84ED2E
:1085E000710AB0EE480ADAF0AFFB84ED700A81F050
:1085F0003FFCC4F894010AB0BDEC028BBDE8F087E3
:10860000A6B194ED1C0AB4EE400AF1EE10FA0DD6B4
:10861000D4ED1D0AF4EE600AF1EE10FA06D694EDE0
:108620001E1AB4EE411AF1EE10FA67D71AF04EFE98
:108630004FF00C0A90F80539B2EE028AF2EE068A83
:1086400007460AFB030307AE4FF0150803F55F73F7
:1086500093E8070086E80700304620F099FEB4EE64
:10866000C80AF1EE10FA11D508F1FF3818F0FF082A
:1086700015D1304620F08CFEF1EE047AB4EEE70A14
:10868000F1EE10FA1CDC2567656731E0304620F01A
:108690007FFEB4EEE80AF1EE10FAE5DCE9E73846D1
:1086A00019F04AFA384619F0B3FC97F805390AFB75
:1086B000037303F55F7393E8070086E80700CBE7D1
:1086C000DDED098A9DED088A68EEA80A9DED070A8E
:1086D000E8EE080AF1EEE00ADAF008FD84ED1D0A82
:1086E000F1EE680AB1EE480ADAF000FD84ED1C0AEA
:1086F0009FED071AD4ED1D0A94ED1C0A48461CF0A4
:1087000075FF66E7888E0024E02E6542F4F31008BA
:10871000000000000021FFF7FDBE000037B5044651
:1087200008461546019120F033FEB7EE007AB4F802
:10873000E8300198C7EE007A94ED397A0133A4F855
:10874000E83037EE277A84ED397AB0EE007AF4EE2D
:10875000C77AF1EE10FA06D5B6EE007AF4EEC77AD3
:10876000F1EE10FA0DDC9FED0E7AF4EEC77AF1EE21
:1087700010FA13D59FED0B7AF4EEC77AF1EE10FAEA
:108780000CDDB0EE670A20F0E5F90120C5ED010A25
:1087900085ED000A85ED021A03B030BD0020FBE72D
:1087A00000247449BD37863570B500F1280600F104
:1087B00034050446294630462DED028BB6EE008A7C
:1087C0008AB020F043FA284620EE088AB0EE480A24
:1087D00020F0C0F907A93046CDED080A8DED091A41
:1087E0008DED070A20F0A0F98DED010AB0EE480AE0
:1087F0003046CDED020A8DED031A20F0ABF907A942
:1088000028468DED070ACDED080A8DED091A20F0F6
:108810008BF904A901A88DED040ACDED050A8DEDB3
:10882000061A20F027FA324601A920468DED070AE4
:10883000CDED080A8DED091AFFF770FF58B981F0E8
:1088400017FB0121C4F890012046FFF763FE0AB030
:10885000BDEC028B70BD2A4604A92046FFF75EFFDF
:108860000028ECD004F1400207A92046FFF756FF8C
:108870000028E4D0EBE7000030B50D4604462DEDAE
:10888000028B284683B091F8461303F03FFFC1B234
:108890007C2000FB015104F1280094311CF03EFDC6
:1088A00068468DED000ACDED010A1FF0D3FFDFED24
:1088B0001C7AB4EEE70AF1EE10FA05D59FED190A1D
:1088C00003B0BDEC028B30BD684620F037F8684637
:1088D0001FF0A4FF0028F1D194ED4E8A284604F041
:1088E00091F9F0EE400AB0EE480A1CF067F880B942
:1088F000284604F087F9B0EE408A84ED4E0AD9F09C
:108900001DFC84ED4F0AB0EE480ADAF01DFA84ED42
:10891000500A04F59E7168461FF058FFD0E700BF6B
:1089200000000034000000009FED0C7AB4EEC70A8E
:10893000F1EE10FA0BD4DFED0A7AB4EEE70AF1EEAD
:1089400010FA07DCC0EE077AB0EE670A7047F7EE60
:10895000007AF9E7F2EE047AF6E700BFF3665F3FCC
:1089600058A00B411C3008B51FF074FFF1EE007ADF
:10897000B4EEE70AF1EE10FA97BFF1EE027A9FED3E
:10898000050A37EEC00ADFED047A98BF20EE270A09
:1089900008BD00BFCDCCCC3DCDCC4C3E08B58369E5
:1089A00093F9000038B10DF0DBFDFDF7D9FA01288D
:1089B00094BF0020012008BDF8B52DED028B0546BF
:1089C00004F094FB04F08EFA0446B8B3FFF758F9AC
:1089D00090F8213393B32846FFF7E0FF064668B3CB
:1089E0000DF0BEFDB02790F80C33F0EE087A07FBCF
:1089F000030090ED417AB4EEE77AF1EE10FA1DD45F
:108A000095ED1E8A0DF0ACFD90F80C33DFED1E7A6B
:108A100007FB030090ED420A98EE270A1CF08AF843
:108A2000B0EEC00ADFED197AB4EEE70AF1EE10FA03
:108A300008DC344681F01CFAC5F880012046BDEC04
:108A4000028BF8BD05F5C27020F0A2FCB0EE408AA2
:108A50000DF086FD90F80C339FED0D7A07FB0303B4
:108A6000D3ED417A67EE877AB4EEE78AF1EE10FA39
:108A7000DFD581F0FDF9D5F88041001BB0F5FA6F24
:108A80008CBF00240124D9E7E02E65420000344267
:108A9000CDCC4C3F0A4B1B6810B5DB6A044693F8FB
:108AA0009C305BB981F0E4F9D4F89431C01A44F6F3
:108AB0001F6398428CBF0020012010BD0020FCE7FE
:108AC000888E0024F8B52DED068B04460DF048FD88
:108AD000054604F00BFB064606F0D2FC002840F0E9
:108AE000AB802046FFF768FF002800F0A8803046E2
:108AF000FFF794FCD4F8F430984200F01A81304625
:108B0000FFF78CFCD4F8F430DFED8F7AC31A3046CF
:108B100008EE903AF8EE688A68EEA78AFFF77EFCC6
:108B200094F8BC30C4F8F400F3B9304604F0ECF922
:108B3000D0B104F1280796F846233046394604F0B0
:108B400065F8D4ED1D0AB0EE401A384694ED1C0AC3
:108B50001CF04CFD0023C4F89030C4F88C30C4F8ED
:108B60008830012384F8BC3020463146FFF784FE6C
:108B700095F80C03B0EE408A05EB0015D5F8B83037
:108B8000C4F8F83004F1B000D4ED129A20F000FCE3
:108B90006368DFED6E7A68EE299A93ED007AB0EEA5
:108BA00040AAB4EEE77AF1EE10FA01D5C3ED007AEF
:108BB0002046B0EE4A0AFFF7B7FE636820EE299A16
:108BC00093ED000A29EE009AFFF7CCFE204629EE2D
:108BD000009A84ED249AFFF75DFF38B1B2EE007A77
:108BE000D4ED247A67EE877AC4ED247AF0EE007A29
:108BF000F4EEE78AF1EE10FA10D5DFED557AB4EE17
:108C0000E7AAF1EE10FA09D5DFED527A69EEA79ADC
:108C1000D4ED2A7AE9EEA87AC4ED2A7AB0EEC88AB1
:108C20009FED4D0A94ED3C7ADFED4C7A28EE008AF8
:108C3000A7EE278A84ED3C8ABDEC068BF8BDFFF7D2
:108C40001FF890F82133002B73D02046FFF7A6FEC3
:108C500000286ED095F80C2305EB0213D3F8B8105A
:108C6000D4F8F8308B4264D0B026F0EE087A06FBD8
:108C7000025292ED417AB4EEE77AF1EE10FA58DB47
:108C8000CB1AC4F8F8109FED361A08EE903A95F812
:108C90000C3394ED1E0A06FB0353F8EE688ADFEDF1
:108CA000317AD3ED429A68EEA78A69EE819A39EE5D
:108CB000C00A1BF0A1FFB0EE409ADAF045F894F834
:108CC000BC30B0EE408AF3B1F3EE047AF4EEE78AFA
:108CD000F1EE10FA17DC95F80C03F2EE027A06FBBF
:108CE000005595ED417AB4EEE77AF1EE10FAFFF611
:108CF00049AFB0EEC99ADFED1C7AB4EEE79AF1EE17
:108D000010FAFFF63FAFB0EE691AD4ED1D0A94EDEC
:108D10001C0A04F128001CF069FC9FED148A012351
:108D200084ED248A84ED238A84ED228A84F8BC3081
:108D300028E7BDEC068B04F188009FED0D0ABDE825
:108D4000F8401FF05BBF00BFBD378635CDCC4C3D32
:108D5000C2B8B23E0AD7233CCDCC4C3ECDCC4C3F22
:108D600035FA8E3C6F12833A1904863F00000000EA
:108D7000EC51783F0C2303FB010130B501F1C00336
:108D80008BB0144604AD93E8070085E8070094E82B
:108D9000070083E807002846FFF708FA07AB58B139
:108DA00094E8070083E807009DED070ADDED080A57
:108DB0009DED091A0BB030BD95E80700F2E7000001
:108DC00010B52DED028BDFED0E8AB0EE408A044621
:108DD00060EEA88AB0EE680AD9F0B0F920EE480A31
:108DE00084ED610AB0EE680AD9F0AEFF20EE480AC1
:108DF0000023BDEC028B84ED620AC4F88C3110BDF7
:108E000035FA8E3CF0B52DED028BD0F84831044692
:108E100085B00D468B60D0F84C31CB6001F0E4FD9D
:108E200006460DF09DFBA369074693F90030022B1F
:108E300053D1FDF795F802284FD997F80C33B0229B
:108E400002FB0373D3F8F8100022284602F006FE56
:108E500094ED561A94ED550A2846B7EEC11AB7EEAE
:108E6000C00A03F0D9F994F85C3183B39FED258AE9
:108E700080F0FEFF01AA97F80C13064638468DEDE8
:108E8000018A0CF0A1FAD4F85001F0EE480A9FEDE7
:108E90001E0AB6EE001A361A40F23C4007EE906AFF
:108EA000F8EE677A27EE800A1BF0D2FEDDED017A3C
:108EB00004F5907030EE270A8DED010A1FF032FCA8
:108EC0002846B7EEE01AB7EEC00A03F0A5F994F809
:108ED0005C0105B0BDEC028BF0BD707C502303FB40
:108EE000006696ED0B8AFEF7CBFED0EDA27A9FEDE1
:108EF000077AF8EEE77AE8EE077AFDEEE77A17EE02
:108F0000901AA1E7000000006F12833A0000C842E7
:108F100030B589B004460D46684602F09BFD6946AF
:108F20002046FFF7E5F818B90024204609B030BD07
:108F300004A802F08FFD204604A9FFF763FF044652
:108F40000028F1D004A9684602F0CCFF85ED000BA3
:108F500085ED021B85ED042BE7E7000010B586B018
:108F6000002200230C466946CDE90023CDE9022307
:108F7000CDE90423FFF7CCFF18B1DDE90423C4E9F0
:108F8000002306B010BD000070B586B0002200239B
:108F90000C466D462946CDE90023CDE90223CDE9F3
:108FA0000423FFF7B5FF064618B195E80F0084E8E3
:108FB0000F00304606B070BDF8B52DED028B0646A9
:108FC0000F46154600F016FE0446A0B1394600F0E3
:108FD000E1FD80B12046394600F0E0FD044650B185
:108FE00000F008FE394600F0DBFD85ED000A204662
:108FF000BDEC028BF8BDFEF743FE90F82033B7EED0
:10900000008A7BB13046FFF7C9FC044650B1D6ED6B
:109010005F8AFFF70DF8C8EE007A67EEA87AC5ED13
:10902000007AE4E7D6ED5F8AFFF702F8C8EE007A2F
:10903000002467EEA87AC5ED007AD8E770B52DED6B
:10904000048B1646FFF7B8FF054670B3FEF718FE0F
:1090500090F93C424CB30DF083FAFCF781FF0128F4
:1090600023D9E4B207EE904AB8EE678A0DF078FA99
:10907000B02290F80C3396ED009A02FB0300D0ED7D
:10908000418AFEF7D5FF40F2654029EE000A38EE2E
:10909000281A78EEC80A1BF0DBFDB0EE408AFEF716
:1090A000C7FFC8EE007AC6ED007A2846BDEC048BF7
:1090B00070BD000038B50D460DF052FA0446FCF7BD
:1090C0004FFF022885BF94F80C03B023002003FB58
:1090D000004081BF00F58E7007C885E807000120B9
:1090E00038BD000030B585B000230D4601A90193BD
:1090F00002930393FFF7DEFF044620B1039B2B602E
:10910000204605B030BD01F06FFC417C01F022F932
:1091100004460028F4D001F067FC00F05BFFB1EEDC
:10912000400A85ED000AEBE7F8B5036F00F14C0744
:109130000C4605464B6001F11006436F8B60836F50
:10914000CB600FCF0FC60FCF0FC63B6805F12801CC
:1091500004F1340033601EF029F82346012203F89D
:10916000442B05F1B00207CA83E8070005F1940219
:1091700004F1500307CA83E8070005F11C0204F15B
:109180005C0307CA83E8070004F174012846FFF76F
:1091900091FF04F1840184F880002846FFF7A2FFC4
:1091A00004F18C0184F888002846FFF72BFE84F830
:1091B0009C00F8BD08B503F099FFBDE8084003F036
:1091C00091BE000010B504461FF070FD50B904F1C7
:1091D0000C001FF06BFD28B904F11800BDE8104029
:1091E0001FF064BD012010BD38B500F1280504460C
:1091F0002846FFF7E7FF28B120460121BDE83840A7
:10920000FFF788B9B7EE007AD4ED107AF4EEC77A9A
:10921000F1EE10FA06D5BFEE007AF4EEC77AF1EE61
:1092200010FA12DC2046FFF7BFFA2846FFF7CAFF04
:109230000028E1D1D4ED107AB2EE047AF0EEE77AAC
:10924000F4EEC77AF1EE10FAD6DC38BD10B504465C
:1092500020F09EF82046BDE810401FF0E3BC00005F
:109260002DE9F04F044600274FF0000804F1FC0BF5
:1092700004F1280A2DED028BABB0B0EE408A5E46B9
:1092800009970A970B97FFF71DFC1AF01FF8054680
:1092900095F86D335FFA88F1032BA8BF03238B4247
:1092A0003AD92846019118F03BFB019980B312ABE3
:1092B00015AA284615971697179718F07FFD9DED6C
:1092C000120AB5EEC00AF1EE10FA21DD15A81FF062
:1092D00051FC21A950468DED210ACDED220A8DEDDC
:1092E000231A1BF0BFFF8DED180AB0EE480A18A82C
:1092F000CDED190A8DED1A1A1FF02CFC21A930466C
:109300008DED210ACDED220A8DED231A1FF042FCCE
:1093100008F101080C36BBE70C2395F805195046F7
:1093200003FB015101F55F711BF09CFF84ED070AFF
:1093300094ED4B0AC4ED080A30EE088A84ED091A50
:1093400084ED4B8A0DF00CF90646FEF799FC90F877
:10935000213320460393FFF721FB80B13046FCF711
:10936000FFFD02280BD996F80C23B023616903FB9B
:10937000026391F9001093F81A01884264DA94EDBF
:109380004B7ADFED857AB4EEE77AF1EE10FA65D428
:1093900094ED5F8AFEF72EFF58B100F02BFC90F899
:1093A0004E1100F0FDFBB0EE408AFEF741FE20EECC
:1093B000088A236CB0EE480A626B21A8A16A239345
:1093C000229221911FF0C6FB04F5C27109A88DED10
:1093D000090ACDED0A0A8DED0B1A1FF0DBFB80F0B8
:1093E00047FD0023019084F844312046FFF7D6FA68
:1093F00000286AD096F80C23B02101FB0262D2F853
:10940000FC30C4F8483196F80C3301FB0363D3F801
:109410000031C4F84C3180F02BFD0123C4F8500119
:10942000C4F85471C4F8587184F85C31D4F8303100
:10943000002B5DD1019B04F59074236109AB93E887
:10944000070084E8070009E006EB0212D2F8B82012
:1094500001920199D4F830218A4204D12BB0BDEC9D
:10946000028BBDE8F08F03F58E730DF1240C93E8A9
:10947000070094F844318CE807001BB904F5907399
:1094800083E807000123604604F5C27184F8443183
:109490001FF04AFB21A904F14C008DED210ACDED0E
:1094A000220A8DED231A1BF00BFFB5EEC00A8DEDDD
:1094B000210ACDED220A8DED231AF1EE10FAD8BF64
:1094C0009FED340A84ED5F0A8FE794ED4B7AD4ED7B
:1094D000557ADDED096AE6EE877ADDED0A6AC4EDBC
:1094E000557AD4ED567AE7EE267AC4ED567A9DE7A2
:1094F000D4ED4B7A244BF5EEC07A0C970D970E9372
:10950000F1EE10FAAAD9214B9FED217A1B6867EE84
:10951000877ADB6AB7EE007A93F89C30C7EE278A29
:109520000293002B4AD094F8443113B9039B002BCB
:1095300042D0E36804F5907109A893ED008A1FF00A
:10954000F3FA8DED210A21A828EE888ACDED220AB2
:109550008DED231AB0EE480A1FF0FCFA18A90CA8EA
:10956000CDED190A8DED180A8DED1A1A1FF012FBB8
:109570000CA8FFF76BFE0CA81FF0B2FBF0B180F057
:1095800077FCC4F8900169E7000080BF888E002452
:109590000AE81C4100000000CDCC4C3ECDCC4C3F35
:1095A000CDCC4C3D920A06BF920A063FC2B8B23EED
:1095B000728A0E3C5B821839039B0293242200219D
:1095C00018A80DF18408DCF037FC2422002121A822
:1095D000DCF032FC4FF0000905F62B131FED138A67
:1095E0004FF0FF37059395F86D335FFA89F1032B40
:1095F0001A46A8BF03228A427AD98B4204916BD9BA
:10960000059B13F80930002B66D0B0EE680A584667
:109610001FF0F4FA029B0499002B64D00C222AABB1
:10962000204602FB0933A3F12402069304925A4612
:10963000FFF7A0FB069B03ED090A049BC3ED010A9B
:1096400083ED021A4046FEF7B1FD002844D14046A2
:10965000FFF7FCFD40461FF043FB00283CD10C23E4
:109660000CA9404603FB09F22AAB13440792A3F16D
:109670004802069304921FF0FDFA069B0CA940468F
:1096800003ED120A049BC3ED010A83ED021A1FF0D9
:10969000DDFA2AAB079A03EB890303ED1B0A18AB2B
:1096A00098181FF075FE7A1C04D0B4EEC08AF1EE53
:1096B00010FA03DDB0EE408A4FFA89F72AAB03EBCC
:1096C000870353ED1B7AF5EE407AF7EE007AF1EE60
:1096D00010FA48BFB0EE678A09F1010908F10C08D9
:1096E0000BF10C0B7FE79BE8070088E80700A9E770
:1096F0007B1C3FF444AF204684F83471FFF75CF9DB
:1097000060B12046FFF74AF9002840F033812AAAC9
:109710000C2303FB0723002243F8402C18AA07EB75
:10972000470895F8043902EB880895F86C239A42AB
:1097300040F23B812B4493F82839002B00F035810F
:1097400095F8053995F86D239A4240F22E812B4405
:1097500093F82B39002B00F028810C232AAA4146CC
:10976000504603FB07271BF0ABFD07ED120A47ED40
:10977000110A07ED101A40461FF098FA002840F031
:10978000208140461FF0ACFA002840F01A815FEDBE
:109790007E7A04F1B00094ED3B7A28EE278A5FEDE3
:1097A000817AA7EE278A84ED3B8A1FF0F1FDA3683A
:1097B0005FED857AB0EE408A93ED007AB4EEE77AF9
:1097C000F1EE10FA00F101812046B0EE480AFFF7F1
:1097D000ABF840461FF0BEF9A3688DED150A15A839
:1097E000CDED160A8DED171A93ED000A1FF0B2F9B0
:1097F000204684ED1F0AC4ED200A84ED211AFFF7EC
:1098000049F928B1B2EE000A04F17C001FF0F6F924
:10981000039BB3B33046FCF7A3FB012831D996F87C
:109820000C03B023F0EE087A03FB006696ED417A54
:10983000B4EEE77AF1EE10FA23D595F805090C237A
:10984000F1EE0C7A03FB005595EDDF7AB4EEE77A82
:10985000F1EE10FA15DBD4ED1D7A1FEDAE7AF4EEC1
:10986000C77AF1EE10FA0CDD1FEDB17AF4EEC77A8B
:10987000F1EE10FA05D5B6EE000A04F17C001FF0F7
:10988000BDF95FEDB67AB4EEE78AF1EE10FA22D5B3
:109890001FEDB90A40461FF05DF912A88DED120ABE
:1098A00094ED4B0ACDED130A8DED141A1FF052F909
:1098B00015A904F1A0008DED150ACDED160A8DED68
:1098C000171A1FF067F9D4ED2B7A94ED4B7A77EEE7
:1098D000877AC4ED2B7AF1EE047A94ED2B7A002589
:1098E000B4EEE77AF1EE10FA3BDB19F0EFFC5FED36
:1098F000CF7A94ED2B1A40F2C93094ED280A21EE6C
:10990000271AF1EE410A8DED031ACDED020A1BF084
:109910009FF940F2CA309DED031ADDED020A84ED95
:10992000280A94ED290A1BF093F940F2CB309DED03
:10993000031ADDED020A84ED290A94ED2A0A1BF0D0
:1099400087F904F1A00104F1940084ED2A0A1FF0C4
:1099500021F9C4F8A850C4F8A450C4F8A050C4F821
:10996000AC502422002104F1FC00DCF065FAC4F8BC
:109970002C515FE5E368F7EE000A93ED000A1BF057
:109980001DF800283FF4C3AE94ED1C0AB0EEC00AE7
:10999000D9F0DAF90C232AAA03FB072353ED107A36
:1099A00027EE800A03ED100AB8E60C232AAA03FB6F
:1099B0000727002347F8403C47F8443C47F8483C19
:1099C000D9E62046FFF710FCD9E5C3ED007AFBE6A7
:1099D000F0B52DED108BA1B0044619F077FC00F620
:1099E000141390EDDE8AD3ED007AF4EE487AF1EEAE
:1099F00010FA48BFB0EE678ADFED5B7AB4EEE78A13
:109A0000F1EE10FA0CDD2422002104F1FC00DCF060
:109A100013FA0023C4F82C3121B0BDEC108BF0BD3B
:109A2000204616ADFEF714FD2046FEF7BDFEB0EE53
:109A3000480A204604F14C06FFF712FC2046FFF7C7
:109A4000D3FBFEF71DF904F1280100F53A7216A8C0
:109A50001BF086FC0FCD0FC60FCD0FC62B6804F18F
:109A6000740204F1700104F14C00336004F17803D6
:109A70001BF01CFE94ED1E8AB0EE480AD8F05EFB87
:109A800084ED710AB0EE480AD9F05EF9204684ED03
:109A9000700AFEF7D1FCFEF7F3F804F5CC71FDF780
:109AA000C3FE80F0E5F9D4F8C831C31A632BB3D9EB
:109AB000C4F8C8014AF0D8FD054680F0E1F9DFEDB1
:109AC0002B7A94ED1E0A074694ED1C8A0E4694EDFF
:109AD0001D9A20EE270A28EE278A29EE279A1BF0E6
:109AE00013F8D4ED5FAAB0EE40AA94ED3BBAB7EEFE
:109AF000C88A94ED3CCAB7EEC99A94ED61DAB7EE24
:109B0000CBBA94ED62EAB7EECCCA94ED63FAFEF7F5
:109B10008FFA8AEE807A164B164A28460193164B26
:109B20001649B7EECDDA0093B7EECEEA144BB7EE96
:109B3000CFFAB7EECAAA8DED12FB8DED10EB8DEDCD
:109B40000EDB8DED0CCB8DED0ABB8DED08ABB7EECA
:109B5000C77A8DED069B8DED147B8DED048BCDE9E1
:109B600002764AF0B7F957E7CDCC4C3EE02E65427D
:109B70000BC910082BF4100861C91008E8F110088F
:109B800020F4100870470000002070477047000064
:109B90000020704700207047002070470020704769
:109BA0009FED010A704700BF000000009FED010A11
:109BB000704700BF000000007047000000207047A1
:109BC0007047000010B50446143000F019F804F195
:109BD0002C0000F015F804F17000A1F059FD04F11B
:109BE000F400A1F055FD4FF0FF332046C4F8543186
:109BF00010BD0000014B1868704700BFAC8E0024F8
:109C000070470000094A0123D2ED057AD8B2F4EE7C
:109C1000C07AF1EE10FA02DD0138C0B270470133AC
:109C20001432082BF0D10720704700BF0CF5100844
:109C30000C4B1422DFED0C6AF0EE407A02FB003090
:109C400090ED047A90ED010AB0EEC76AB4EEE66AD0
:109C5000F1EE10FA5EBFD0ED006A77EEE67AA7EE7D
:109C6000270A70470CF510080000003410B50446B0
:109C70003648F0EE407A012103462DED068B90ED3B
:109C8000077ACAB2F4EEC77AF1EE10FA23DD013A90
:109C9000D2B2142101FB023393ED027A87EE870AD8
:109CA000DFED2B7AB4EEE70AF1EE10FA19DA48F09C
:109CB00081FDA7224FF4801148F034FD637C5022CF
:109CC000D4ED467A02FB034393ED0B0A30EE270AEC
:109CD000BDEC068B10BD013114300829CFD107220D
:109CE000D7E793ED049A93ED008AB0EEC97AD3EDED
:109CF000019ADFED188A9FED18AAB4EEE77AF1EE2B
:109D000010FA12D568EEE98AD8F042FDF0EE487AF2
:109D100088EE8A7AE0EE077A9FED107A67EE876A1E
:109D200077EE677A86EEA70AD2E768EEC98AC8EEB0
:109D30008A0AD8F04BFE89EE897AF7EE007A30EE87
:109D4000670AF0EE487AE7EE007AE5E70CF51008CE
:109D500000000034CB868F430AE81C413CFEC14A18
:109D6000DFED257A254920EE277A30EE270A08B55F
:109D700087EE005A2DED028BB0EE450AFFF742FF49
:109D8000142303FB001140B2FFF752FFDFED1C7AF2
:109D9000D1ED045A91ED038AB0EEE57AB4EEE77A9C
:109DA000DFED187AF1EE10FA12D520EE270A9FEDBA
:109DB000167AC7EE007A91ED000A35EE400A27EEDA
:109DC000800AD8F041FC20EE080ABDEC028B08BDE9
:109DD00065EEA75ADFED0D7AC7EEA50AF7EE007A19
:109DE00070EEA70AD1ED017A80EE270AF1EE600A43
:109DF000D8F0ECFDE7E700BF3CFEC14A0CF51008C7
:109E000000000034CB868F430AE81CC10AE81C41DD
:109E100008B5FFF7A5FFDFED087A9FED087AB4EEED
:109E2000E70ADFED077AF1EE10FA20FE270AC7EE07
:109E3000007AB1EEE70A08BD00000034CDCC9C3FAB
:109E4000BC77E93610B52DED028BF0EE608A044642
:109E5000FFF70CFFB0EE408A2046B0EE680AFFF72D
:109E600005FF30EE480ABDEC028B10BD427C50214C
:109E7000D0ED467A01FB020292ED0B0A30EE270A82
:109E8000FFF7C6BF38B52DED088BB0EE409A0546FA
:109E9000F0EE609A1524B0EE408ADFED1DAA9FED2A
:109EA0001DAA9FED1DBA013CA4B25CB3F0EE490AB5
:109EB0002846B0EE480AFFF7C5FF70EE698AF0EE5B
:109EC000490A284638EE2A0AFFF7BCFFB0EEE87AC6
:109ED00070EE697AB4EECA7A77EEE87AF1EE10FAAB
:109EE00010D468EEAA8A40F26310B0EE4B1AF0EE7E
:109EF0004A0A88EEA70A38EE400A1AF0A9FEB0EE28
:109F0000408AD0E7B0EE480ABDEC088B38BD00BFF0
:109F1000CDCCCC3D0AD7233C0024744900234360B8
:109F20008360C360036143618361C361002380F880
:109F30002030704790F82020531C00EB8202DBB2E7
:109F4000062B80F8203082ED010A84BF002380F8C0
:109F5000203070470022A2F0C5BE00004FF0FF3352
:109F600010B543610023044600F5967040F8D03CDC
:109F700040F8CC3C40F8C83C40F8803C40F87C3C81
:109F800040F8783C40F8303C40F82C3C40F8283C05
:109F90000C4B0360002380F82030FFF7BFFF0A4B13
:109FA00004F5C870C4F82C317FF026F8074B204622
:109FB00007491C6044F074FDD4F814312046C4F8FD
:109FC000183110BDF0F6100800F71008B08E00240C
:109FD000ACF7100800F5967008B54CF017FDDFEDF2
:109FE000027A20EE270A08BD00007A4490ED5D0A4F
:109FF000DFED057AB0EEC07AB4EEE77AF1EE10FA52
:10A0000048BF90ED5E0A70470000003410B504466A
:10A0100080ED490A7FF02CFFC4F8280110BD000034
:10A0200073B5D0F8283104460E4663B17FF020FFA7
:10A03000D4F82831C01A42F20F73984203D894ED35
:10A04000490A02B070BD114B1D687DB195F84E11E3
:10A050002846FFF7A3FD48B101AA95F84E112846FE
:10A06000FFF792FD10B19DED010AEAE75021DFED07
:10A07000087A01FB064494ED0A0AB4EEE70AF1EE11
:10A0800010FA58BFB0EE670ADBE700BFAC8E0024C1
:10A0900000000C4208B561B10378022B02D90648D2
:10A0A0007FF0B6FE5A1C027000EB83004160012075
:10A0B00008BD0846FCE700BFACF510082DE9F843E1
:10A0C00005460E469146002400F13C082B7CA34235
:10A0D00011DD00234A463146012015F091FA502344
:10A0E00007460021634358F8030015F099FA8742A8
:10A0F00004D00134EAE70020BDE8F8830120FBE743
:10A1000070B50B46064614469AB111469847054667
:10A1100028B9236820465B68BDE8704018470146AF
:10A120003046FFF7B7FF20B92B6828465B68984791
:10A13000EFE770BDF0B50D4685B011461A460446EE
:10A14000CDE90213FFF7BAFF034698B90A4804277E
:10A15000006840680668DDE90212CDE90037074B68
:10A160003668B04702462946204605B0BDE8F040B3
:10A17000FFF7C6BF0022F6E7888E0024801A06008B
:10A180001A4B1B682DE9F0470546D0F884915868B2
:10A190004FF0010A164C036804F1E4089B689847E5
:10A1A00095F921310646002BA4BF01269E40236865
:10A1B00019EA030F07D000270AFA07F3334206D142
:10A1C0000137202FF8D10C344445F0D10BE0237A2D
:10A1D000FAB261682846FFF7ADFF2B78032B02D057
:10A1E0002B7C032BECD1BDE8F08700BF888E0024C8
:10A1F000CCF810087FB5D0ED457A01239FED4B7A5E
:10A200000446F0EEE77A0376F4EEC77AF1EE10FA40
:10A210000AD400F58A70002303A90190039345F046
:10A220001FFC019844F000FE00230322E363C4F8FE
:10A230008C30C4F8DC3020460192A2F04BFF01467E
:10A240002046FFF727FF2378032B35D0237C032BF1
:10A2500032D0019A013A12F0FF02ECD17623344950
:10A2600020460192FFF766FF2378032B24D0237C3E
:10A27000032B21D07723019A2D492046FFF75AFF5F
:10A280002378032B18D0237C032B15D07723019A36
:10A2900028492046FFF74EFF2378032B0CD0237C60
:10A2A000032B09D094F92121002A07DA2046FFF771
:10A2B00067FF2378032B0ED104B070BD7723D2B291
:10A2C0001B492046FFF736FF2378032BF4D0237C6D
:10A2D000032BEBD1F0E7237C032BEDD0D4F88431B2
:10A2E000DA0403D5637E0BB9012363760025637E10
:10A2F000EAB2EB40DB0703D40135082DF7D1DBE7E9
:10A300003820019202F004F8064618B1019A21465D
:10A31000A4F0B2F931462046FFF7BCFE2378032BA8
:10A32000CAD0237C032BE7D1C6E700BF000000346E
:10A3300031E30C0859C70C08054B1B682BB1416968
:10A340004A1C02D0184649F0ADBF0020704700BF3C
:10A350004C93002402290BD8502303FB010191F8F0
:10A36000390030B191F83A0018B191F83B007047CC
:10A37000002070472DE9F04704467FF079FD42F256
:10A3800010730027D4F87C614FF0500942F2107A24
:10A39000861B9E4288BFC4F87C01FDB2237CAB4281
:10A3A0001CD929462046FFF7D5FF70B109FB0548A7
:10A3B000D4ED460A204698ED0D0AD8ED097A30EE24
:10A3C000270AFFF75FFD88ED0C0A564504D909FB03
:10A3D0000540303044F028FD0137DEE7617C20463F
:10A3E000FFF71EFE84ED5E0ABDE8F08770B50446F7
:10A3F0002DED028B86B07FF03BFDD4F81C31054675
:10A40000C31AB3F57A7F3FD394ED467A9FED3A8A2B
:10A41000F0EEC76A394BD4ED457A1B68F4EEC86A92
:10A42000DB6AF1EE10FA93F89C6022D5F0EEE76A51
:10A43000F4EEC86AF1EE10FA1BD502A801F00AFB8F
:10A4400016BBFDF71DFC02A9FDF7EEF9E0B1DDED4D
:10A45000037A9FED2B7AF8EEE77A67EE877AB0EE13
:10A46000E77AB4EEC87AF1EE10FA11D4C4ED467A68
:10A4700011E077EE676AB7EE006AF0EEE66AF4EE96
:10A48000C66AF1EE10FA1CDC06B0BDEC028B70BDA2
:10A490001C4BC4F81831C4F81C51FDF7F1FBFCF754
:10A4A0009FFE2046FFF766FF55F040FD94ED467A8B
:10A4B000154A0621B7EEC77A8DED007B4FF0FAFD05
:10A4C000E2E7F0EEE76AF4EEC86AF1EE10FADBD4E8
:10A4D000002ECBD004F58A7084ED457A44F0A4FCBC
:10A4E00055F024FD094A012106B0BDEC028BBDE800
:10A4F00070404FF0DFBD00BF00000034888E0024A4
:10A500000AD7233C6F12833AEDF51008C8F51008FE
:10A510002DE9F0412DED048B84B0044640F27232F7
:10A5200000F5C87103A8002515F00EFAD4ED437AA2
:10A53000D4ED446A50229FED806A37EEE67A637C60
:10A5400002FB0343B0EEC77AB4EEC67AF1EE10FA1E
:10A55000C1BF9FED7A7A67EE877A9FED797AE6EE52
:10A56000877AC4ED447A93F83970E9B223788B4244
:10A5700006D904EB81030135586800F0A3FAF4E72B
:10A580004FF000089FED6F9ADFED6F8ADFED6F9A55
:10A590005FFA88F5237CAB4271D9502303FB054356
:10A5A00093F83920002A3FD0D3ED0C7AF4EEC97A23
:10A5B000F1EE10FA0BDBF4EE677AF1EE10FA06D644
:10A5C000F0EEE77AF4EE687AF1EE10FA04DD50234B
:10A5D00003FB05435A6A1A63502606FB054696EDAF
:10A5E000098AD6ED0D0A96F8383038EE208AF3B98C
:10A5F00029462046A4F012FB78EE400A204696ED4C
:10A600000C0AC6ED1A0AFFF71DFCD4ED467A30EEAF
:10A61000670AB4EE400AF1EE10FA18D75023002270
:10A6200003FB054383F83A2008F10108B0E7012B4A
:10A6300003BFD6ED0C0AD4ED5C7A30EEC88A96EDF5
:10A640000B0A04BF88EE297A87EE270AE1E7F0EECD
:10A65000C07A502101FB0545F4EE687AF1EE10FA5C
:10A66000D7BF0123002385F83A30D4ED447ACEBF1A
:10A6700085F83A3037EE800A85ED0B0AD4E7627C24
:10A6800020461146FFF766FE48B1502104F596704A
:10A6900001FB0242D16992ED0B0A4CF099F994F951
:10A6A0002011267C002907DBB14205DACAB2204618
:10A6B0001146FFF74FFE68B900226274D5B2AE4270
:10A6C00009D9294620460132FFF744FE0028F5D07B
:10A6D000657400E062742046FFF788FE2046FFF7AD
:10A6E0002BFE10B12046A3F0CDFA637C502505FB6C
:10A6F000034393F83930BB4216D049F0B5FF4FF60B
:10A70000FF7149F0CFFD78B1607C05FB004494F8FF
:10A710003930002B14BF00220422019249F0A4FF1B
:10A72000019A122149F050FD03A815F02FF904B049
:10A73000BDEC048BBDE8F0810AD7233C0AD7A33CCB
:10A7400048E17A3F00000034FFFF7F7F0020194678
:10A750002DE9F04F04460F4687B0007C04F13A0320
:10A7600000220121D5B25033A84205D9013203F8A5
:10A770004F1C03F8501CF5E7744B1E68F06A036821
:10A780005B68984740B155F0D1FB714A062107B08C
:10A79000BDE8F04F4FF08EBC23781BB1237C0BB18A
:10A7A00063681BB955F0C2FB6A4AEFE755F0BEFB80
:10A7B000694A06210A254FF07DFC002303A904F510
:10A7C0008670039345F04CF97FF052FB804620469B
:10A7D000FFF79EFE7FF04CFBA0EB0800B0F5FA7F80
:10A7E00002D95E4801F0E4F8B06A0A2103685B68A8
:10A7F0009847617C2046FFF7ADFD0028E7D0B06A9E
:10A80000013D642103685B68984715F0FF05DBD1C3
:10A81000534B05951B888DF80650ADF80430CDE9F3
:10A82000035505257FF024FB80462046FFF770FE88
:10A830007FF01EFBA0EB0800B0F5FA7FD1D8617C59
:10A840002046FFF787FD0028EFD094F810B00DF1F7
:10A850000C08A14601AA4FF0000A5FFA8AF18B4565
:10A8600016D92046FFF776FD50B1D8ED007A99ED64
:10A87000097A137877EE877A0133C8ED007A13707E
:10A880000AF1010A08F1040809F150090132E4E76C
:10A89000B06A013D642103685B68984715F0FF05C5
:10A8A000C0D1A9464FF05008237C5FFA89F6B34225
:10A8B00026D906AB334413F8143C33B908FB0646DB
:10A8C00086F83B3009F10109EEE7002FFAD006AA1D
:10A8D00007EE903A2046D4ED460A02EB8602F8EEE7
:10A8E000E77A12ED030A80EE270AFFF7CBFA08FB9E
:10A8F000064002A98DED020A303045F0B1F8E1E7DB
:10A9000000264FF05008DFF860902046617CFFF78A
:10A9100087FB84ED5E0A237CF7B2BB420FD908FBAC
:10A92000074393F83B3043B1013555F0FFFA7B1CE8
:10A930004A46EDB206214FF0BDFB0136EBE70DB9FB
:10A9400008484FE707B0BDE8F08F00BF888E0024AD
:10A9500008F6100833F6100860F6100876F61008AE
:10A96000BC9F1008B2F6100890F6100808B5037CDA
:10A97000022B02D903487FF04BFA5A1C0274184686
:10A9800008BD00BFD4F6100838B50246057C002487
:10A99000E1B28D4206D910460134FFF7DBFC0028F6
:10A9A000F6D138BD281E18BF0120FAE770B50D4654
:10A9B00009780446072906D8027E437E22B901227F
:10A9C0008A401343437670BD002BFCD000262278CA
:10A9D000F3B29A42F7D904EB83032946013658684B
:10A9E0000368DB689847F2E7014B1868704700BFBF
:10A9F000B08E00247047000073B5436805460C46CE
:10AA00001B7C8B4242D900F10801212201A814F0DD
:10AA10009BFF7FF02DFA6A68502303FB0423D9695A
:10AA2000411AB1F5FA7F33D2196A401AB0F5FA6FBC
:10AA30002ED2D3ED097A9FED177AF0EEE77AF4EE95
:10AA4000C77AF1EE10FA54BF0120002050269FED86
:10AA5000127A06FB04F31A4482F8390069680B4441
:10AA6000D3ED0A7AF4EEC77AF1EE10FA06D49FED30
:10AA70000B7AF4EEC77AF1EE10FA04DD06FB04114E
:10AA8000002381F8393001A814F080FF02B070BDB6
:10AA90000020DBE700000034000048C3000048430A
:10AAA000044B10B50446C0E9003108307EF0A4FA2A
:10AAB000204610BDB8F910084368502000FB013152
:10AAC000CA63704713B50368044601919B689847B1
:10AAD0002368019920461B6902B0BDE81040184761
:10AAE000F8B52DED028B4368F0EE408AB0EE608A37
:10AAF00005461B7C0C468B421FD950277FF0B8F9C6
:10AB00006B68F0EE680A674306463B4493ED090A1A
:10AB100019F054FFA0B96B68502202FB04331E6287
:10AB200050216B684C432344C3ED098A6B6823446E
:10AB300083ED0A8A69680C44E661BDEC028BF8BDBE
:10AB40006B68F0EE480A3B4493ED0A0A19F036FFB1
:10AB50000028E0D0E4E70000B0EEC07ADFED297A0B
:10AB6000B4EE677AF1EE10FA49DCB4EE400AF1EE89
:10AB700010FA44D6436893F9803163B190ED087AB6
:10AB8000DFED217AF0EEC76AF4EEE76AF1EE10FA33
:10AB900003D580ED080A01232BE077EE407ADBB283
:10ABA00037EE006AF0EEE77AC7EE866A9FED176A25
:10ABB00007EE903AF8EE677A26EE866AB4EEE76A18
:10ABC0009FED136AF1EE10FA15DDF2EE047A436A96
:10ABD000013366EEA76A43620023C6EE267AF7EEDB
:10ABE000006A27EE800A76EEE76AA7EE260A80ED75
:10ABF000080A18467047F0EE467A0123EFE7002373
:10AC0000F7E700BFFFFF7F7F0000003400004843EC
:10AC1000CDCCCC3D0020704700207047002070470D
:10AC2000704700000020704790F836007047000021
:10AC300090F83B00704700000120704700207047EB
:10AC4000022070477047000010B5044601F068FB11
:10AC5000204610BD90F8A835934207D902F5B0728E
:10AC600050F8220010B103689B6A18470020704713
:10AC70002DE9F3416E46054604460F4600F5C878B7
:10AC800086E80C00114B45F8043B28462C3500F0B3
:10AC90007BFDA845F9D104F2AC53C4F8A47596E83D
:10ACA000030083E80300089B20460949C4F8B43533
:10ACB00043F0F6FE074B1A6812B107487FF0A8F878
:10ACC00020461C6002B0BDE8F08100BFFCFB10080C
:10ACD000C4FA1008B48E0024CCF910082DE9F04F06
:10ACE0002DED028B90F8A83583B00446002B64D17B
:10ACF0007F2200F5C87500F5B067061D99469FEDE7
:10AD0000B18A80F8B8255FFA89FA1C22FF2128460B
:10AD1000DBF092F885F864A096F926B0ABF1030356
:10AD20001C2B2AD8DFE813F01D001D002900290084
:10AD30004E009800A500B200C100CE005A00680085
:10AD40008C007000290029007F002900E8002900FC
:10AD5000F500DB000301290010011E012B01290071
:10AD60001D00442001F0D4FA804620B133462A4623
:10AD70002146A4F08DF9C7F80080386850B1E96E1B
:10AD8000C5F868B031B1904B43F8291044F082F80F
:10AD900044F078F80AF1010A57F8040B5FFA8AFACE
:10ADA00020B103689B68984784F8A8A509F10109B8
:10ADB00070352C36B9F1090FA5D103B0BDEC028B6B
:10ADC000BDE8F08F7C2001F0A3FA80460028D2D0A5
:10ADD00033462A462146A6F08BFCCCE7482001F0FA
:10ADE00097FA80460028C6D0032300932A463346AC
:10ADF0002146A6F09FFEBEE7482001F089FA804672
:10AE00000028B8D00623F0E77C2001F081FA8046C4
:10AE10000028B0D033462A462146A6F069FC6B4B89
:10AE2000C8F80030A7E77C2001F072FA80460028BD
:10AE3000A1D033462A462146A6F05AFC644BEFE7E0
:10AE4000442001F065FA8046002894D033462A4613
:10AE50002146A6F0F5FD8EE7E82001F059FA80467C
:10AE6000002888D000232A4621460096A4F0E2FD5F
:10AE700081E7382001F04CFA804600283FF47BAF90
:10AE800033462A462146A5F0B7FB74E7302001F08F
:10AE90003FFA804600283FF46EAF33462A462146EB
:10AEA000CDF800A0A7F01CF965E7542001F030FAB6
:10AEB000804600283FF45FAF33462A462146A5F07E
:10AEC00079FC58E75C2001F023FA804600283FF423
:10AED00052AF33462A462146A5F0C2FD4BE7582023
:10AEE00001F016FA804600283FF445AF33462A4663
:10AEF0002146A5F009FD3EE7782001F009FA8046D9
:10AF000000283FF438AF33462A462146A5F046FED6
:10AF100031E72C2001F0FCF9804600283FF42BAFEC
:10AF200033462A462146A4F05BFA2A4B78E74820AC
:10AF300001F0EEF9804600283FF41DAF33462A4663
:10AF40002146A7F03FF916E7282001F0E1F98046F5
:10AF500000283FF410AF33462A462146A4F040FAB9
:10AF60001D4B5DE75C2001F0D3F9804600283FF4DB
:10AF700002AF33462A462146A3F042FFFBE6A0205B
:10AF800001F0C6F9804600283FF4F5AE33462A4664
:10AF90002146A4F025FA114B08F1880088ED1D8A9E
:10AFA000C8F800304FF6FF7388ED1E8AA8F82E30DF
:10AFB000A8F8703088ED1F8A88ED208A7EF01CF892
:10AFC000D9E600BF0000C07FB88E002470FA1008D8
:10AFD00078BD130888BF13087CB8130830BE130867
:10AFE00090F8A8358B4283BF702303FB010090F8D3
:10AFF000E10100207047000090F8A8358B4283BF24
:10B00000702303FB010090ED6B0A9FED010A70476E
:10B010000000000090F8A8358B4206D901F5B07108
:10B0200050F8210008B1A4F0EDB99FED010A704776
:10B030000000000010B490F8A8450A468C4214D9CC
:10B0400001F5B07450F824407CB1E468246A6406C9
:10B0500003D55DF8044BFFF7DDBF702101FB020350
:10B0600093ED6B0A5DF8044B70479FED010AF9E719
:10B070000000000090F8A8358B420BD901F5B071A3
:10B0800050F8210038B1C3681B6A1A4214BF01206E
:10B09000002070470020704770B590F8A83504462E
:10B0A0000E461546934201D8002070BD02F5B073DC
:10B0B00050F823000028F7D003689B6998470028C0
:10B0C000F2D0702202FB0544D4F8B0313360ECE7D3
:10B0D00070B590F8A83504460E461546934201D83F
:10B0E000002070BD02F5B07350F823000028F7D09F
:10B0F00003689B6998470028F2D0702202FB054440
:10B10000D4ED6D7AF4EE677AF1EE10FAE8D6C6ED7A
:10B11000007AE6E770B590F8A83504460E46154665
:10B12000934201D8002070BD02F5B07350F823009F
:10B130000028F7D003685B6998470028F2D0702296
:10B1400002FB0544D4F8B8313360ECE790F8A83539
:10B1500093420ED902F5B07350F823305BB17023DF
:10B1600003FB020292F8F00130B1D2F8EC310B602F
:10B1700070470020704718467047000008299DBF9F
:10B180002C2303FB0100406800207047474B1B68DD
:10B190002DE9F04F2DED028BDB6A87B0044693F862
:10B1A0009C30002B7DD04FF00009DFF814A1DFF8B0
:10B1B00014B19FED3F8A5FFA89F594F8A835AB4248
:10B1C0006FD905F5B07354F82300002853D00368F5
:10B1D0005B6B98477023074603FB054393F8E03108
:10B1E000834248D2032857D8DFE800F04502484F91
:10B1F000304E4FF0000854F099FE94F8A8256B1CCF
:10B200000421AA4289BF7022B0EE487A02FB0542AF
:10B2100092ED6B7A702202FB0545B7EEC77A524673
:10B2200095ED6D6A0096B7EEC66A8DED027B8DEDE9
:10B23000046B4EF03FFF012384F8B9358BF80B30D7
:10B2400085F8E071D4F8B4354BB3002255B25957A4
:10B25000481C03D0414502F10102F7D194F9B835F9
:10B26000AB4208DBD4F8B03542463146D4F8AC05E1
:10B27000984784F8B85509F101099CE72C230E4E34
:10B2800003FB054393F92D80B5E72C230B4E03FBFD
:10B29000054393F92E80AEE70026B046ABE71D4686
:10B2A000DCE707B0BDEC028BBDE8F08F888E002490
:10B2B00000000000F9F910087AB61308F0F9100838
:10B2C00008FA1008259000240020704790F8A8354F
:10B2D0008B4207D901F5B07150F8210010B1036815
:10B2E000DB6918470020704708299CBF702303FBC7
:10B2F000010000F5C8707047F8B504460E461546C3
:10B300001F46FFF7E3FFD0B10D2D19D8082E9CBFC3
:10B31000702101FB06444FF6FD7104F5C87434F842
:10B320001520531E9BB28B420AD807EE902A9FED40
:10B33000057AF8EEE77A67EE877AC7ED007AF8BD0E
:10B340000020FCE76F12833A90F8A835934207D9A2
:10B3500002F5B07250F8220010B103685B6A18471A
:10B360000020704790F8A8358B420DD901F5B073D5
:10B3700050F8233043B1702303FB0101012081ED1C
:10B38000740A81F8CC01704700207047F8B500249A
:10B3900002460E462C272546E1B292F8A8358B428C
:10B3A00010D901F5B07352F823304BB107FB0123DC
:10B3B0009B689E4204D11046FFF7D4FF2843C5B2D4
:10B3C0000134E9E72846F8BD0B46114690F8A82558
:10B3D0009A4207D903F5B07350F8230010B10368FF
:10B3E000DB6A1847002070472DE9F04F002493B026
:10B3F00005460E46174621462F2206A8059405F558
:10B40000B069DAF019FD05F12A0A4FF02C0B05F5A9
:10B41000FC730BFB04F259F8040BE5B21AF90210A5
:10B4200030B951B90134092CF3D14FF0010813E0C0
:10B43000702262439A58914212D001351448154B3C
:10B440004FF000080068EDB201933246009539468E
:10B45000114BC06A14F07AFC404613B0BDE8F08F7F
:10B4600005A933220393A4F0ADF805A98046039BF8
:10B470000028D7D10135064801913246EDB2006867
:10B48000054B39460095C06A14F060FCE4E700BF44
:10B49000888E00246507110830FA10082DE9F04F56
:10B4A00006468DB00027DFF87C90DFF87CA0DFF83F
:10B4B0007CB096F8A835FCB2A3422ED9702505FBC6
:10B4C000046595F8E83133B395F8E91119BB4FF0ED
:10B4D0000108202204A8444489F81980DAF0ACFC61
:10B4E0004AF2104307EE904A03AA4C215046F8EE68
:10B4F000E77AADF828302423CDED037A4EF0D0FB67
:10B5000054F014FD9BF80030054A042100944EF0DD
:10B51000D1FD85F8E9810137CBE70DB0BDE8F08FAB
:10B5200040FA1008259000243C9400242027002491
:10B53000304B2DE9F04F1E6885B0044646B1D0F877
:10B54000A415304648F0AEFE10B1304647F050FD2D
:10B550004FF000084FF02C0A4FF0700B7EF088FC83
:10B5600001905FFA88F594F8A835AB4239D904EB1D
:10B570008507D7F8800588B30AFB05430BFB05490F
:10B5800093F92A20D9F8F8118A4227D132B30268F8
:10B59000D2689047D7F880050268126B904799F8F7
:10B5A000E12112B1019BC9F8E431BEB1D4F8A41570
:10B5B000304648F077FE88B17EF062FC02460B46CA
:10B5C000CDE902102946D7F88005A5F00FFE2946DF
:10B5D000D7F88005DDE90232A5F07EFE08F101080A
:10B5E000BFE72046FFF7D2FD204605B0BDE8F04F8B
:10B5F000FFF754BF4C9300242DE9F0474FF00008AB
:10B6000004468946012647464FF0700A2DED028B0D
:10B61000B0EE408A94F8A8355FFA88F5AB421AD9A3
:10B6200029FA05F3DB070AD505F5B07354F82300B2
:10B6300078B10368B0EE480A9B6B984706400AFB56
:10B64000054508F1010895F8E0319F4238BF1F46D3
:10B65000E0E70646F3E727B97F23A4F8B835034BA4
:10B66000DF723046BDEC028BBDE8F08725900024E8
:10B6700090F8A8358B4207D901F5B07150F8210038
:10B6800010B10368DB6B1847002070470B4611466A
:10B6900090F8A8259A4207D903F5B07350F8230013
:10B6A00010B103681B6C18477047000070B5044662
:10B6B0000E460025E9B294F8A8358B4205D93246EA
:10B6C00020460135FFF7E2FFF4E770BD2DE9F843AE
:10B6D000024690F8A855002400F12A062C2700F510
:10B6E000FC784FF07009E1B28D420FD907FB04F3EB
:10B6F00009FB04F0F35658F80000834209D11BB14E
:10B700001046FFF76DFC10B10134ECE70120BDE8F5
:10B71000F8830020FBE7000010B590F8A825044648
:10B720008A4217D9702202FB010393F8E031022B01
:10B7300003D004D9032B18BF0023184610BDFFF710
:10B7400097FF48B92046FFF7C1FF00280CBF06232A
:10B750000123F2E70023F0E70623EEE70B4611464C
:10B7600090F8A8259A4207D903F5B07350F8230042
:10B7700010B103685B6C184700207047014B1868D4
:10B78000704700BFB48E002410B50446024943F050
:10B7900087F9204610BD00BF84FC100800F120038B
:10B7A0004022002110B504461846DAF045FB9FED13
:10B7B0000C1ADFED0C0A9FED0C0A69F0C3FE0023A2
:10B7C00004F1600084F8403084F85C3065F01CFBC4
:10B7D000064B204606491C6043F062F9204610BD26
:10B7E00000008C42295C8F3D00004842DC8E002422
:10B7F00094FE10082DE9F3410546B7EE000A002239
:10B80000022142F057FD2846A6F01EFF65F0DAFC43
:10B81000234B04461E68F06A03685B6A98470B4630
:10B82000022102462046009165F004FBB5F99270B2
:10B83000002F13DDD6F82C80BCB2D8F8003040467B
:10B840005B68984728B198F84D3013B1C92FA8BF4D
:10B85000C824B06A214603685B689847202200210B
:10B8600095F9910019F05CFAC4B266F04FFE66F0EB
:10B8700095FD70B9B06A013405210368E4B25B68D4
:10B880009847072CF1D9074802B0BDE8F0417DF098
:10B89000EBBC072CF7D885F8914002B0BDE8F081E9
:10B8A000888E002484FD100810B50446A6F03AFEE8
:10B8B0002046BDE81040A6F065BE00002DE9804896
:10B8C0001446284B012293B005460E464FF000085F
:10B8D000DFF89490DFF894A0DFF894B01A707EF04F
:10B8E000C7FAD9F80030A0EB08020746039341F2EB
:10B8F00087339A421FD903985346342205A9B84684
:10B90000CDE90056C06A14F021FA214605A8049436
:10B910007DF09AFC03985B46342205A9CDE90056D8
:10B92000C06A14F013FA049454F000FB049B05AAB7
:10B9300002214EF0A7FB54F0F9FA53F0C7FF54F080
:10B94000F5FA56F019FB0A2105A813F0E3FF039B53
:10B950000521986A03685B68984705A813F0E6FF1D
:10B96000BDE700BFE08E0024888E0024ED91110811
:10B970000DDA13080FB400B595B0002116AA05A87A
:10B98000049152F8043B03923C220193DAF054FAFA
:10B99000054A4021019B04A87DF0FEFB039A04A9FF
:10B9A0000248FFF78BFF00BF9CFD1008B2FD100896
:10B9B0000FB407B504AA034852F8041B0192FFF71D
:10B9C0007DFF00BFC4FD10080A2938B518D10E4B01
:10B9D000C4881B68B0F90650D86A14F0040302D179
:10B9E00090F89C2062B90368DB699847012802D16E
:10B9F00005F0010038BD022804D1C4F34000F9E786
:10BA00000020F7E70120F5E7888E0024014B186835
:10BA1000704700BFDC8E002438B504460025E2895B
:10BA2000ABB2A0689A4205D950F823000135D4F092
:10BA300083FAF4E7D4F080FA204638BD1022044996
:10BA400008B5DAF09FF9B0FA80F0400908BD00BFF0
:10BA5000E48E002410220021DAF0EEB90378022AE5
:10BA6000416023F00D03037008D0032A0AD0012A95
:10BA700003D1DBB243F0010303707047037843F056
:10BA80000803F9E7037823F0050343F00503F3E720
:10BA900073B504460E4615460193FFF7DBFF2046BB
:10BAA000069A0199C4E90265FFF7D8FF02B070BD9C
:10BAB0004B68436003780A7862F3000303700B78E5
:10BAC0000278C3F3800363F382020270D2B20B7870
:10BAD000C3F3C00363F3C3020270704700784207E8
:10BAE00004D4030704D400F001007047032070471A
:10BAF00002207047F0B587B004461546FFF7EEFF09
:10BB000088420F46064605D163682B600126304601
:10BB100007B0F0BD00230328019301D0032913D1FE
:10BB200045F038FF08B90026F1E7012301AA2146B4
:10BB300045F098FC0028F6D0DDED017A9FED337AD0
:10BB400067EE877ACDED017A032E32D8DFE806F072
:10BB5000020916246468032FE5D8DFE807F02C2ECD
:10BB60003C49FCF78DF890F89432DB07DBD564682C
:10BB7000FCF786F8D0F888321C44ECE702A8FFF7FF
:10BB800069FFFCF77DF802A9FBF74EFE0646002888
:10BB9000BDD06468039BEFE7D4ED017A9DED017A97
:10BBA000F8EEE77A77EE877AFDEEE77A17EE904ABD
:10BBB000D1E70024CFE72C60A8E7FCF761F890F804
:10BBC000946216F00106AED0FCF75AF8D0F888322D
:10BBD000E41A2C609BE702A8FFF73CFFFCF750F843
:10BBE00002A9FBF721FE0646002890D0039BEFE751
:10BBF00007EE904A9DED017AF8EEE77A77EEC77A84
:10BC0000FDEEE77AC5ED007A80E700BF0000C8428C
:10BC100073B501AA05460E46FFF76CFF044620B136
:10BC2000324601992846FFF719FF204602B070BD41
:10BC300013B5144601AAFFF75DFF48B1DDED017AA7
:10BC40009FED047AF8EEE77A67EE877AC4ED007A22
:10BC500002B010BD0AD7233C07EE900A9FED0C0AF4
:10BC6000F8EEE77A08B527EE800AD6F067FADFED3E
:10BC7000097AB4EEE70AF1EE10FA02DDB7EEC00A77
:10BC800008BD9FED010BFBE700000040E17A843F17
:10BC900050E0EF300AD7233C10B50446806819F015
:10BCA00093FA20B1E068BDE8104019F0A1BA10BDC8
:10BCB00073B5856804460E461DBBC36823B98B68FF
:10BCC00001258360CB68C360636873B92378DB07A1
:10BCD0000BD52046FFF702FF01AA01463046FFF7C9
:10BCE00009FF10B1019B054663602046FFF7D4FFB2
:10BCF00020B9B3680125A360F368E360284602B069
:10BD000070BD0025E0E700000D4B83424FF00003BB
:10BD10008B4106DA00F1255000F5311000F5E050B6
:10BD20007047084B98424FF0FF3371EB0303BEBFDF
:10BD300000F1564000F5130000F52440704700BFA5
:10BD400000D2496B002EB69490EA010F01D4401A3C
:10BD50007047C317401A63EBE1710D4B83424FF0FC
:10BD600000038B4106DA00F1255000F5311000F593
:10BD7000E0507047074B98424FF0FF3371EB0303DD
:10BD8000BEBF00F1564000F5130000F52440704797
:10BD900000D2496B002EB69470B52DED028B84B0A5
:10BDA00004460D466846FFF755FEFBF769FF6946F6
:10BDB000FBF73AFD064628B3A368029ADFED148A22
:10BDC0009B1A039907EE903AF8EEE77A67EEA87AA5
:10BDD000C5ED007AE068FFF7B7FF08EE100AA0682B
:10BDE000B8EEC88A024428EE288A02EBD2725010BC
:10BDF000B7EEC88AFFF730FF28EE000BB7EEC00B96
:10BE000085ED010A304604B0BDEC028B70BD00BF69
:10BE1000F67C8E3F002337B50C4601AA0221054669
:10BE20000193FFF767FE10B9002003B030BD214633
:10BE30002846FFF7B1FF0028F6D0DDED017AF8EED5
:10BE4000E77AC4ED027AF0E708B5FFF7E3FF08BD33
:10BE500038B50D46FFF7DEFF044620B19FED030A1B
:10BE600028461CF0CBFE204638BD00BF0AD7233C35
:10BE7000F0B50D4606462DED028B8C6889B0D0E9F1
:10BE80000271E868FFF760FF08EE100AE019E41B92
:10BE900000EBD0704010FFF7DFFEB8EEC86ADFEDB0
:10BEA0000F4A736826EE246A6A689FED0D1A9B1A82
:10BEB000B7EEC66A07EE903A26EE006BB8EEE75A88
:10BEC00007EE904AF8EEE75AF7EEC60B25EE011A98
:10BED00025EEA40A09B0BDEC028BF0BD8262363CAF
:10BEE0000AD7233CF0B50D4606462DED028B8C6833
:10BEF0008DB0D0E90271E868FFF726FF08EE100A5E
:10BF0000E01900EBD0704010FFF7A6FE73686A6876
:10BF1000B8EEC87ADFED107AB0EE401B9B1A02EE45
:10BF2000103AE31BB8EEC22A00EE103AB8EEC00A8F
:10BF300022EE272ADFED097A27EE277A20EE270A5C
:10BF4000B7EEC22AB7EEC77AB7EEC00A27EE011BDA
:10BF50000DB0BDEC028BF0BD0AD7233C8262363CAB
:10BF6000F0B52DED028B8BB00D460021074605AADA
:10BF70000691FFF7BFFD002190BB0023CDE90533FB
:10BF8000D7E90261AC68E868FFF7DEFE08EE100A48
:10BF9000A019A41B00EBD0704010FFF75DFEB8EEB7
:10BFA000C86ADFED134A9FED131A26EE246ADDE915
:10BFB0000532B7EEC66A9B1A07EE903A26EE006B82
:10BFC000B8EEE75A07EE904AF8EEE75AF7EEC60BDE
:10BFD00025EE011A25EEA40A0BB0BDEC028BF0BDD4
:10BFE00006AA2846FFF786FD0028C6D0C8E700BF8E
:10BFF0008262363C0AD7233C38B50C4602462DED0A
:10C00000028BC168E068FFF79FFE9568A46808EEA0
:10C01000100A6019641B00EBD0704010FFF71CFE83
:10C0200007EE904AB8EEC81BB8EEE77B87EE006BD0
:10C03000BDEEC60B10EE103A5B4200EE103AB8EEC1
:10C04000C00BD6F0BBFF9FED087B30EE070BB5EEC3
:10C05000C00BF1EE10FA03D59FED057B30EE070B18
:10C06000BDEC028B38BD00BF00000060FB21F93F32
:10C0700000000060FB2119400B4630B52DED028B0E
:10C080008C6885B0D0E90251D868FFF75DFE08EEF4
:10C09000100A6019641B00EBD0704010FFF7DCFD44
:10C0A000B8EEC86A9FED095A07EE904A26EE056A77
:10C0B000F8EEE75AB7EEC66A26EE006B25EE850A63
:10C0C000F7EEC60B05B0BDEC028B30BD8262363C8C
:10C0D0000B4630B52DED028B8C6889B0D0E902514A
:10C0E000D868FFF731FE08EE100A6019641B00EBF8
:10C0F000D0704010FFF7B0FD07EE904AB0EE401B45
:10C10000B8EEE76BB8EEC87B9FED050B27EE007B22
:10C1100026EE000B27EE011B09B0BDEC028B30BDF3
:10C120000000004050CC863F84B004B0FFF7D0BF81
:10C1300010B52DED048B84680B468A68111B2244D0
:10C1400009EE101AC168D86802EBD272FFF7FCFD45
:10C1500008EE100A5010B8EEC99BB8EEC88BFFF776
:10C160007BFD28EE000B20EE000BA9EE090BBDECC9
:10C17000048BB1EEC06B9FED020B26EE000B10BDE1
:10C180000000004050CC863F094B984206DDC0F1CC
:10C19000D64000F5930000F5A4407047054B984247
:10C1A000BEBFC0F1144000F5360000F538507047AE
:10C1B00000E9A43500175BCAF8B52DED048B9FED9F
:10C1C000149BB0EE418B076806460D4620EE090B26
:10C1D00028EE098BFDEEC07B17EE904A04EBD4707D
:10C1E00007EB6000FFF738FD88EE007B3819FFF79A
:10C1F000CBFF306051EC170BF4F71EFC2B68C01816
:10C2000041EBE371FFF780FD2860BDEC048BF8BDC6
:10C21000000000404075564000F10C010830FFF767
:10C22000CBBF000000B52DED068B9FED109B83B0BA
:10C23000B0EE418B20EE099B0190B0EE490BD6F099
:10C24000ABF8B0EE40ABB0EE490BD6F0E5F820EE1F
:10C25000081B01982AEE080B03B0BDEC068B5DF8B5
:10C2600004EBFFF7D9BF00BFAFF30080000000A0D0
:10C2700046DF913F10B52DED0A8B9FED1ECBB0EE42
:10C28000409B0446B0EE42AB21EE0CBB29EE0C9B6A
:10C29000B0EE4B0BD6F080F8B0EE408BB0EE490B11
:10C2A000D6F07AF8B0EE40CBB0EE490BD6F0B4F849
:10C2B00028EE001B204628EE0C8B21EE0A1B28EEF0
:10C2C0000A0BFFF7A9FFB0EE4B0BD6F0A5F820EE56
:10C2D0000A0B63689FED092BBDEC0A8B20EE020B65
:10C2E000BDEEC00B10EE102A1344636010BD00BFFA
:10C2F000AFF30080000000A046DF913F0000000087
:10C30000000059400148FFF7A5BB00BFE48E0024A0
:10C310000121884238BF0846D3F00ABEFFF7F8BFB4
:10C3200008B1D3F009BE7047FFF7FABFF8B506466B
:10C330000F46144622B92546D3F0FEFD2846F8BD27
:10C3400010461EB9BDE8F840D3F0B2BDD3F0B0FD41
:10C3500005460028F2D0BC422246314628BF3A4664
:10C36000D9F020FD3046D3F0E7FDE7E737B5089D6B
:10C370000446084611461A46036801959DF81C506C
:10C3800000951D68069BA8472060204603B030BD7D
:10C3900090F9253013B190F8440370471846704760
:10C3A00000214FF0FF33002210B54363044600F133
:10C3B0004003016041608160C16080F8291000F590
:10C3C0000C70D9707C3343F8742C43F8702C43F80C
:10C3D0006C2C43F8682C43F8642C43F8602C43F829
:10C3E0005C2C43F8582C43F8542C43F8402C43F869
:10C3F0003C2C43F8382C43F8342C43F8302C43F8C9
:10C400002C2C43F8282C43F8242C43F8202C43F8F8
:10C41000102C43F80C2C43F8082C9842D1D121461B
:10C4200004F5177007F042FF044B1A6822B904495B
:10C4300020461C6042F034FB204610BDF48E0024E0
:10C44000D801110873B5D0F84032044601919942E1
:10C4500013D0D0F84432994218D0D0F848328B42E9
:10C4600016D102200AE0D4F8383253B3D4F83C3263
:10C470004BB34FF0030002B070BD002094F826309B
:10C480008342F8D8431C84F82630F4E70120F5E70E
:10C49000D0F83462002EE6D194F845233546B60034
:10C4A0009AB1A319C3F83412A319019A2846C3F804
:10C4B000402294F82630AB429CBF6B1C84F8263097
:10C4C000D9E70126E8E70226E6E704F50D7001A9A1
:10C4D000304443F0D3FBE7E738B504460D4643F05C
:10C4E00043FB291D201D43F03FFB05F1080104F12A
:10C4F000080043F013FC05F1140104F1140043F0AB
:10C500000DFC05F1200104F1200043F007FC05F1CA
:10C510002C0104F12C0043F0BBFA05F1300104F1C9
:10C52000300043F0C3FB05F13C0104F13C0043F053
:10C53000F5FBAB6BA3636B6B636338BD2DE9F04315
:10C5400000F14007A1B000230025064600F5107851
:10C55000B9468DF807500393049305930693079308
:10C56000089309930A930B931093119312931393C7
:10C57000149315931693179318931C931D931E935E
:10C5800058F8043BF3B1326F934222D0D6F8EC2036
:10C59000934220D0D6F86821934213D10221EBB206
:10C5A00099420FD0C1EB411101A809EB810421464A
:10C5B000FFF792FF39462046FFF78EFF01A9384664
:10C5C000FFF78AFF01357C37032DD9D121B0BDE8B3
:10C5D000F0830021E3E70121E1E700002DE9F047C6
:10C5E00004460E461546804607464FF0000A31467F
:10C5F0002046FFF727FFBA6F5FFA8AF9B2420ED1E1
:10C60000C3B2022B0BD87C2202FB0A44012084F81F
:10C61000433084F8420085F80090BDE8F0870AF1C5
:10C62000010A7C37BAF1030FE1D1002731462046D9
:10C63000FFF708FFD8F870205FFA87F912B9C3B284
:10C64000022B19D9013708F17C08032FEED13146AE
:10C650002046FFF7F7FEC2B2C2EB421304EB83039E
:10C6600093F8427067B9022A0BD8012083F843205F
:10C6700083F842002A70D0E77C2000FB0744C5E71E
:10C6800000274FF07C0904F1420A31462046FFF7AB
:10C69000D9FE034609FB07F05FFA87F81AF8002075
:10C6A00012B9DBB2022B09D90137032FEDD194F86F
:10C6B000271004290BD914487DF0AAFB044401205B
:10C6C00084F8433084F8420085F80080A5E704F53B
:10C6D0004477002057F8043BC2B2B34208D19142DC
:10C6E00002D8531C84F8273003322A70002094E7C4
:10C6F00033B9481CC43184F8270044F82160F3E7BB
:10C7000001300528E6D1F1E7F4FF1008C9B200EBCB
:10C710008101D1F8403253B1426F93420AD0D0F830
:10C72000F020934208D0D0F86C21934206D04FF00D
:10C7300003007047002070470120704702207047B7
:10C740002DE9F8430F469146044600F5BA7894F86F
:10C75000425035B97C344445F9D100252846BDE81E
:10C76000F88300234A463946012012F049FF064665
:10C770000021206F12F054FF8642EBD1EEE700005B
:10C78000012303FA01F1D0F80C3319420AD14AB15E
:10C7900090F82430032B1FBF591C063380F8241057
:10C7A00040F823207047000038B505460C4609B90B
:10C7B000002038BD084612F043FF0328F8D105F5E4
:10C7C000497305F54E7253F8041BA142F0D09A420A
:10C7D000F9D1AB6F9C42EBD0D5F8F4309C42E7D056
:10C7E000D5F87001001B18BF0120E2E738B50546F7
:10C7F0000C4679B1084612F023FF03280AD105F54B
:10C800004472002352F8041B8C4204D1C43300222A
:10C8100045F8232038BD0133052BF3D1FAE700009A
:10C820002DE9F04FD0F80C5389B0044615F400659B
:10C8300025D1E8B203F0B6FC024618B10B21204620
:10C84000FFF79EFF94F82730052B02D00135082D05
:10C85000EFD1B4F84E329B0711D594F8455375B912
:10C8600004F510763068B14612F0EAFE03285FFA4C
:10C8700085FA06F1040605D00135032DF2D109B081
:10C88000BDE8F08F51462046FFF740FF7C23C0B241
:10C8900003FB004090F84270002FEDD104F50D73BA
:10C8A000A9F10C090493314B0293029B20465FFAD5
:10C8B00087FBD3F80C804146FFF776FF0390F8B171
:10C8C00053F034FB56F8043C294A012100932B46CF
:10C8D0004DF0F0FB002307A94846079343F0CEF93B
:10C8E0000023584646F8043C03F05CFC07A970B1ED
:10C8F00002460B212046FFF743FF4146FFF776FF34
:10C90000029B01371033032F0293CED1B4E7A34625
:10C9100004F5BA73DBF87020904517D19BF84320DB
:10C920000593524516D900230793049B03EB82001D
:10C9300043F0A4F99BF843200023039804EB820200
:10C9400007A9C2F84032059B8BF843A00BF17C0B82
:10C950005B45DFD10028D3D007A94846CDF81C801D
:10C9600043F08CF946F8048CCAE700BF288F0024F6
:10C97000100011082DE9F043044685B000F510764B
:10C9800000257C27DFF87080B14656F80C3CE9B2F0
:10C990000436D9F80020934219D1C3B12046FFF7DD
:10C9A000B5FEC0B207FB004090F842307BB903A946
:10C9B000A9F10C00039343F061F953F0B7FA56F86C
:10C9C000043C4246012100932B464DF073FB013598
:10C9D000032DD9D104F1700504F5F274296821B949
:10C9E000AB6813B1284641F061F97C35A542F5D119
:10C9F00005B0BDE8F08300BF3C00110838B505461E
:10CA0000FFF7C6FC28B3134B1B68DB6A93F89C3016
:10CA1000FBB9114C7DF02CFA2368C01AB0F57A7F6F
:10CA200017D37DF025FA2060D5F80C4314F4006488
:10CA30000FD1E0B203F0B6FB024618B10B21284635
:10CA4000FFF79EFE95F82730052B02D00134032C0A
:10CA5000EFD138BD888E0024F88E002438B5044606
:10CA60001546FFF753FEC0B2022808D87C2329469A
:10CA700003FB0040BDE83840543043F03FB938BDB7
:10CA800038B504461546FFF741FEC0B2022808D863
:10CA90007C23294603FB0040BDE83840603043F06A
:10CAA0002DB938BD37B50D4604468DED010AFFF7A7
:10CAB0002DFE022D07D8C0B27C2301A903FB004044
:10CAC0006C3042F0CDFF03B030BD000038B50546F4
:10CAD000FFF71CFEC4B2022C13D8C4EB441440353B
:10CAE0000021A40004F10800284441F0DFF804F11B
:10CAF000340104F1300029442844BDE8384043F0B3
:10CB0000BDB838BD70B505460E461446FFF7FEFDAC
:10CB1000C3B2022B0DD87C2000FB035394E807001E
:10CB2000483383E8070031462846BDE87040FFF7E8
:10CB3000CDBF70BD37B504461546FFF7E7FDC0B25F
:10CB4000022809D87C230DF107018DF8075003FB5B
:10CB50000040443043F008F803B030BD1FB590F9F1
:10CB60003030044623B390F925300BB36846FEF706
:10CB700071FFFBF785F86946FAF7B4FDC0B1DDED4A
:10CB8000037A01239FED0B0AF8EEE70ADDED027A46
:10CB900084F84133F8EEE77AC0EE800A87EE800A27
:10CBA00007F0DAFDDFED047A20EE270A84ED0B0AA8
:10CBB00004B010BD8096184B35FA8E3C38B505464A
:10CBC0000C46FFF7E5FB40B12C4494F9300220B14C
:10CBD00095F92800033818BF012038BD70B590F8CA
:10CBE000264006465CB100252C46E9B23046FFF7E8
:10CBF000E5FF08B10134E4B20135032DF5D120463B
:10CC000070BD000090ED0B0A7047000038B50C466F
:10CC1000D1ED066A11460546FFF778FDD4ED087A96
:10CC2000C3B27C2094ED076AB7EE007A00FB035391
:10CC3000D3ED270AA6EEE67AD3ED265A26EE600A51
:10CC400093ED255A67EEA00AA5EEA70AF0EE607AEA
:10CC5000E5EE867AB1EE400A67EEE60AE5EE070AEF
:10CC6000D6F044FA40F658009FED061ADFED060AAA
:10CC700017F0EEFFD5ED0B7ABDE8384030EE270A0D
:10CC800017F0BABFDB0F4940DB0F49C02DE9F04177
:10CC900090F8263004460D468B4202D20020BDE8B3
:10CCA000F081FFF733FD04F14006C0B2C0EB401045
:10CCB00006EB800008301CF06BFBB0EEC00ADFED25
:10CCC000147AB4EEE70AF1EE10FAE7D429462046CA
:10CCD000FFF71CFDC5B27C2000FB05477B6F002BD6
:10CCE000DCD0032DDAD000FB0560D7F8708030303F
:10CCF00041F0A2FFD7E91C32934201D1984505D0FB
:10CD00007C2000FB0544C4F87080C7E70120C6E71B
:10CD1000000000342DE9F74F04460E46174600F593
:10CD2000107A4FF0000B5AF8049B5FFA8BF8B9F1B8
:10CD3000000F26D041462046FFF740FF08B341468A
:10CD40002046FFF7E3FC7C23C0B203FB004090F8D1
:10CD500042505DB908F101031B4A39463046DBB247
:10CD60007CF01AFA284603B0BDE8F08F5AF8102C70
:10CD7000914506D0154A3946304600257CF00CFA1C
:10CD8000F0E70BF1010BBBF1030FCCD14FF0000822
:10CD90005FFA88F194F826308B420DD92046019134
:10CDA000FFF774FF054620B901992046FFF706FFFB
:10CDB00020B908F10108EBE70125D3E7044A394619
:10CDC00030467CF0E9F9CDE76400110879001108DC
:10CDD0009E0011082DE9F04106464FF000082DEDA8
:10CDE000048B82B090F84613FFF790FC06F14007E1
:10CDF000C5B27C209FED2F8A00FB0575DFED2E8AE2
:10CE00009FED2E9A54355FFA88F496F82630A342A7
:10CE10004DD921463046FFF7D1FE10B908F101087F
:10CE2000F1E721463046FFF771FCC4B27C2000FBDD
:10CE30000474D4ED157A5434F0EEE77AF4EEC87A3F
:10CE4000F1EE10FA0ED5D4ED017AF0EEE77AF4EEB9
:10CE5000C87AF1EE10FA05D5002002B0BDEC048BC3
:10CE6000BDE8F081294620461CF0A2FAB4EEE80A9B
:10CE7000F1EE10FAF0DC294620461BF0F7FCB4EE88
:10CE8000C90AF1EE10FAE7DC214628461BF03AFC0D
:10CE900068468DED000ACDED010A1BF0DBFCDFEDED
:10CEA000087AB4EEE70AF1EE10FAB7DDD4E7012014
:10CEB000D3E700BF00000034DB0FC93F920A863F72
:10CEC00000004843022910B5044608D8FFF71EFCAD
:10CED0007C23C0B203FB004494F8410010BD002045
:10CEE000FCE7000013B590F8461304460191FFF7E4
:10CEF000E9FF30B10199204602B0BDE81040FFF7CC
:10CF00005DBE02B010BD0000F7B50446FFF740FA61
:10CF10000546002873D094F846132046FFF7D2FF49
:10CF200094F84133064613B92046FFF717FE002553
:10CF30002046FFF763FD94F82420EBB29A4207D90C
:10CF40000633013554F8230003689B689847F2E7DD
:10CF50007CF08EFF0027224604F5BA7140F2F315EB
:10CF6000D2F8A0307C32C31AAB428CBF002301231D
:10CF700002F83B3C914247EA0307F1D194F928308B
:10CF8000032B07D194F84033002B3BD0D4F83C035B
:10CF9000002849D167B1636B013309D047F064FBC6
:10CFA000616B47F07FF918B147F05EFB46F078F906
:10CFB00094F93032002B3AD194F93132CBBB94F949
:10CFC000323213B1022384F8463394F846132046D4
:10CFD000FFF778FF8642054611D047F045FB4FF634
:10CFE000FF7147F05FF950B1002D14BF00220422F9
:10CFF000019247F039FB019A032147F0E5F82846F2
:10D0000003B0F0BD0123042084F84033FFF780F91A
:10D01000054610B1214607F0F9F994F92830C4F813
:10D020003C53032BB2D0B5E707F0FEF9B2E700237B
:10D03000C9E70123C7E7000070B504460E46FFF7B5
:10D04000A7F90546C8B131462046FFF75FFBC0B2DD
:10D05000022812D87C239FED0A7A03FB0044D4ED0A
:10D060001B7AF4EEC77AF1EE10FA06D4B7EE087A1E
:10D07000F4EEC77AF1EE10FA00DD0025284670BD07
:10D08000ABAA2A3F70B5D0F80C5304460E4615F4EF
:10D0900000350DD190F844335BB90A78072A07D8D8
:10D0A000012303FA02F290F84333134380F8433329
:10D0B00070BD94F82420EBB29A42F9D90633314678
:10D0C000013554F823000368DB689847F1E7000056
:10D0D00038B5054670242B591BB10021281940F0A2
:10D0E000E5FD7C34B4F5F27FF5D138BD014B18680D
:10D0F000704700BFF48E002410B50446006810B1DC
:10D1000003685B689847204610BD000010B50446D0
:10D11000006810B103685B689847204610BD0000A6
:10D1200010B50446006810B103685B689847204654
:10D1300010BD000030B50C2289B000210546FFF774
:10D14000FFFA0446F8B10023CDE904330022059B21
:10D1500007A811460793CDE9052203F009FF07212F
:10D1600002462846FFF70CFB07A8FFF7D9FF06A8E1
:10D17000FFF7D6FF05A8FFF7C9FF14B104A8FFF712
:10D18000C5FF09B030BD0423064902460968CDE950
:10D190000103054B05A800930C234968FFF7E6F847
:10D1A000D4E700BF888E0024801A06002DE9F04FD6
:10D1B000D0F80C538DB004460F4615F4807B16460C
:10D1C00098469DF858909DF85CA060D1FFF7B8FA9A
:10D1D000054600283FD0CDE906BB069B4FF0000B6B
:10D1E0004246394620460493CDE905BBFFF7A8FA2D
:10D1F000064600283DD0CDE90ABB0A9A002308A9BB
:10D2000004A808924A46CDE90933534600F0B0FF1E
:10D21000074608A8FFF784FF09A8FFF781FF0AA8BF
:10D22000FFF774FF16B10BA8FFF770FF04A8FFF714
:10D2300077FF05A8FFF774FF06A8FFF767FF15B192
:10D2400007A8FFF763FF3A46082120460DB0BDE866
:10D25000F04FFFF795BA04230E493A460968CDE925
:10D2600001030D4B06A8009333464968FFF77EF88B
:10D27000B3E7042307493A460968CDE90103064BA1
:10D280000AA8009343464968FFF770F8B5E70DB068
:10D29000BDE8F08F888E0024801A06002DE9F04F3B
:10D2A00001249146D0F80C238BB08C40984606465A
:10D2B0000F4614409DF850309DF854A09DF858B08A
:10D2C00035D11A4641460593FFF73AFA059B0546C4
:10D2D00000B3CDE90844089A0023514606A80692F7
:10D2E0005A46CDE90733C847044606A8FFF718FF9A
:10D2F00007A8FFF715FF08A8FFF708FF15B109A851
:10D30000FFF704FF2246394630460BB0BDE8F04F28
:10D31000FFF736BA04220749CDE90102096808A8D7
:10D32000054A009242464968FFF720F8D3E70BB060
:10D33000BDE8F08F888E0024801A0600B14B2DE9DD
:10D34000F04F1D68044689B0002668684FF0010858
:10D350004FF0080ADFF8B49203689B6898470746C5
:10D3600008FA06F33B4240F06F820136202EF7D1D7
:10D37000686800264FF001094FF006080368DFF8DF
:10D380008CA2DB689847074609FA06F33B4240F057
:10D390006D820136202EF7D1686800264FF0010813
:10D3A0004FF0080A0368DFF868929B6898470746C1
:10D3B00008FA06F33B4240F06A820136202EF7D18C
:10D3C000686800264FF001084FF0080A0368DFF88C
:10D3D00044929B689847074608FA06F33B4240F0A0
:10D3E00066820136202EF7D16868002601274FF0AB
:10D3F0001A0903689B689847804607FA06F313EA00
:10D40000080F40F064820136202EF6D168680026AD
:10D410004FF0010A4FF01A090368B046DB689847DD
:10D4200007460AFA06F33B4240F06C820136202E92
:10D43000F7D1686800264FF0010ADFF8DC91036835
:10D44000B046DB68984707460AFA06F33B4240F0CD
:10D4500074820136202EF7D1686800264FF0010A49
:10D46000DFF8B4910368B046DB68984707460AFACC
:10D4700006F33B4240F071820136202EF7D16868F6
:10D4800000264FF001084FF0020A0368DFF8889188
:10D490009B689847074608FA06F33B4240F06D82C6
:10D4A0000136202EF7D1686800264FF001084FF0B2
:10D4B000020A0368DFF860919B689847074608FAFC
:10D4C00006F33B4240F076820136202EF7D16868A1
:10D4D00000264FF00108DFF844910368B2469B68CC
:10D4E0009847074608FA06F33B4240F0738201363C
:10D4F000202EF7D1686800264FF0010ADFF81C9152
:10D500000368B046DB68984707460AFA06F33B42D1
:10D5100040F070820136202EF7D1686800264FF067
:10D5200001084FF0060A0368DFF8F4909B689847FB
:10D53000074608FA06F33B4240F06C820136202E83
:10D54000F7D1686800264FF0010ADFF8D49003682D
:10D55000B046DB68984707460AFA06F33B4240F0BC
:10D5600069820136202EF7D1274B0027DFF8B4B0AF
:10D570004FF00C0A0793686800264FF00109036812
:10D580009B689847804609FA06F313EA080F0FD004
:10D5900007AB5A4607212046CDE9019AFB5C009370
:10D5A000F3B2FFF77BFE94F82730052B00F05B8188
:10D5B0000136202EE7D10137042FDCD16868002620
:10D5C0004FF00108DFF860900368B2469B68984707
:10D5D000074608FA06F33B4240F03C820136202E13
:10D5E000F7D1686800264FF0010ADFF83C90036825
:10D5F000B046DB68984707460AFA06F33B4240F01C
:10D60000398213E0888E00240C0D0E0F250A0308C2
:10D610007D210308A5230308B11303087D11030826
:10D62000FDE00208710F0308890C03080136202E63
:10D63000E2D1686800264FF00108DFF86C930368B8
:10D64000B2469B689847074608FA06F33B4240F00B
:10D6500021820136202EF7D1686800264FF0010A9A
:10D66000DFF844930368B046DB68984707460AFA38
:10D6700006F33B4240F01E820136202EF7D1686847
